:020000040800F2
:100000005C38002063050008AD040008650A02089A
:10001000B1040008B3040008B504000800000000A3
:10002000000000000000000000000000B70400080D
:10003000B904000800000000BB040008BD0400086B
:10004000BF040008C1040008C3040008C504000878
:10005000C7040008C9040008CB040008CD04000848
:10006000CF040008D1040008D3040008D504000818
:10007000D7040008D9040008DB040008DD040008E8
:10008000DF040008E1040008E3040008E5040008B8
:10009000E7040008E9040008EB040008ED04000888
:1000A000EF040008F1040008F3040008F504000858
:1000B000F7040008F9040008FB040008FD04000828
:1000C000FF040008010500080305000805050008F5
:1000D00007050008090500080B0500080D050008C4
:1000E0000F05000811050008130500081505000894
:1000F00017050008190500081B0500081D05000864
:100100001F05000821050008230500082505000833
:1001100027050008290500082B0500082D05000803
:100120002F050008310500083305000835050008D3
:1001300037050008390500083B0500083D050008A3
:100140003F05000841050008430500084505000873
:1001500047050008490500084B0500084D05000843
:100160004F05000851050008530500085505000813
:1001700057050008590500085B0500085D050008E3
:080180005F050008610500089D
:10020000DECEA5ED02003078463430370000000025
:1002100000000000000044433231365F3134313099
:100220000000000000004170706C69636174696FC8
:100230006E00000000000000000000000000000050
:100240000000000000000419BB00DAF7DECEA5EDC7
:100250000200307846343037000000000000000013
:10026000000053504C6174436F6E74726F6C6C6518
:1002700072004170706C69636174696F6E00000098
:10028000000000000000000000000000000000006E
:0802900000000000FE00DAF797
:1002980001000208100000002500020818000000F4
:1002A800790102081700000009060208170000007B
:1002B8000509020803000000410F020806000000BB
:1002C8000114020809000000A11C02080200000035
:1002D800AD1D0208110000003122020810000000C4
:1002E800ED230208FF000000D12B02080C000000DB
:1002F800D93002080000000015330208050000008C
:1003080051590208120000004D5D02080A00000061
:10031800256302080A000000E56D020814000000C9
:100328003D78020808000000F57F02080700000079
:100338009D86020810000000AD8A02081300000024
:10034800559C020813000000D5C9020816000000D9
:10035800652E030816000000693003081700000026
:1003680079680308160000004969030817000000AF
:08037800F97C030815000000E8
:100380002F49072291438D462E492F480A1A06D03D
:100390000722914381F30988022282F314882B48B3
:1003A0002B492C4A00F039F82B482C492C4A00F0F4
:1003B00034F82C482C492D4A00F02FF82C482D49B0
:1003C0002D4A00F02AF82D482D492E4A00F025F834
:1003D0002D482E492E4A00F020F82E482E490022A2
:1003E00000F026F82D482E49091A082903DB0022BF
:1003F0000260043001601F481F49884205D002682E
:10040000043003B4904703BCF7E700208646EC466F
:1004100000200021234A9047FEE7884207D0521A65
:1004200005D0037801300B700131013AF9D17047E2
:10043000884202D002700130FAE770471A487047CC
:100440005C3800205C4000205C38002058EE030837
:1004500088010020FC0100200000020800000208C2
:10046000B0BB030858EE0308880100208801002073
:10047000BC050008BC050008BC050008BC05000858
:10048000BC050008BC050008B0BB0308B0BB0308EE
:1004900058EE0308FC010020103500205C350020D8
:1004A0005C3500204D410208FFFFFFFFFEE7FEE73D
:1004B000FEE7FEE7FEE7FEE7FEE7FEE7FEE7FEE714
:1004C000FEE7FEE7FEE7FEE7FEE7FEE7FEE7FEE704
:1004D000FEE7FEE7FEE7FEE7FEE7FEE7FEE7FEE7F4
:1004E000FEE7FEE7FEE7FEE7FEE7FEE7FEE7FEE7E4
:1004F000FEE7FEE7FEE7FEE7FEE7FEE7FEE7FEE7D4
:10050000FEE7FEE7FEE7FEE7FEE7FEE7FEE7FEE7C3
:10051000FEE7FEE7FEE7FEE7FEE7FEE7FEE7FEE7B3
:10052000FEE7FEE7FEE7FEE7FEE7FEE7FEE7FEE7A3
:10053000FEE7FEE7FEE7FEE7FEE7FEE7FEE7FEE793
:10054000FEE7FEE7FEE7FEE7FEE7FEE7FEE7FEE783
:10055000FEE7FEE7FEE7FEE7FEE7FEE7FEE7FEE773
:10056000FEE71348854600F022F84EF68850CEF29A
:100570000000016851F47001016000BF00BF00BFBE
:10058000F1EE100A50F04070E1EE100A4FF000005A
:1005900080F314884EF63C71CEF20001086850F0EA
:1005A00040700860034804490160FFF7E9BE7047E6
:0C05B0000000022008ED00E00000000840
:020000040801F1
:1000000000000000000000000000000000000000F0
:1000100000000000000000000000000000000000E0
:10002000000000000000000000000000000004EAE2
:100030000F018600003D8601003D680120830042DB
:10004000F430F10B000E496E697469616C69736973
:100050006E672E2EF00400C000F411F40300790046
:100060000000F10A0006F10A0101F00201C085F169
:100070000A0001F00104C085095E8302A1F00001BD
:10008000C0008302DE8302C78304B5F10A0001F1D8
:100090000A0100F00200C000F10A0003F10A0101A8
:1000A000F00201C000F10500F00300C000F10B00F8
:1000B0000156F00400C0001E0000145D0B00CB4A86
:1000C000077108F42D00007D800085F419830387F3
:1000D000F00001C000F10B0010456E7465722059EC
:1000E0006561723A2020202020F00400C000F10B4E
:1000F00000023230F00400C0008F13028301B3818C
:100100000079830387F00001C000F10B000C456EFD
:10011000746572204D6F6E74683AF00400C0008FF1
:1001200013038301B38100CD830387F00001C00076
:10013000F10B000A456E746572204461793AF0044F
:1001400000C0008F13048301B3810102800154F4C5
:1001500019800128F41AF4114A00F420830387F06F
:100160000001C000F10B0010456E74657220486FED
:10017000757220283234293AF00400C0008F130031
:100180008301B381014F830387F00001C000F10BAD
:10019000000E456E746572204D696E757465733A14
:1001A000F00400C0008F13018301B381015CF412DD
:1001B0008000795E690020F10A0001F10A0100F077
:1001C0000200C000171301D001D801E001F502219F
:1001D000F41B83035780024AF41D83035780024AAD
:1001E000F10A0001F10A0102F00200C000F41B83D1
:1001F000035780024AF41DF303004783033EF41DB6
:10020000F10B00022028F00400C000F10200F00110
:1002100001C000F10B00022920F00400C0008002A0
:100220004AF41F83036FF10B00022028F00400C082
:1002300000F42FF423F303001583033EF10B0002B7
:100240002920F00400C00080024A830393F4028C4A
:100250000802658C0902805D0A029B5D0B029E68A4
:10026000002080024D17130271027602710276029D
:100270007BF4288001B7F4298001B7F42A8001B704
:100280001713028C0291028C02910296F4388001BD
:10029000B7F4398001B7F43A8001B74A00094A013E
:1002A00009F41300F41B870002B7F41D870002B79E
:1002B000F421877F02B7094A00F41C4A00F41E4A61
:1002C0007FF422F4140009F10A0001F10A0105F09B
:1002D0000200C000F411F416F00400C00009F10A95
:1002E0000000F10A0100F00200C000F419F423F349
:1002F00003001583033EF10B000120F00400C00051
:10030000F41F01890A0311F10B000120F00400C061
:1003100000F10200F00101C000F10B000120F00427
:1003200000C000F41DF303004783033EF10B0003FC
:10033000203230F00400C000F41B83035709F3118E
:1003400002F30BF30900F31103F30A0000F31F009B
:1003500000F00400C0000901890A0366F10B0001E6
:1003600030F00400C000F10200F00101C0000901FA
:10037000890A037EF10B000120F00400C000F102A5
:1003800000F00101C00009F40270084A0F52820314
:10039000875E09F40661002003A29948000084806A
:1003A00003A79920000082F40270084A0F528103CB
:1003B000BBF437F61C03A76900200968002009096F
:1003C000F00002C08509F10200F00100C08509F1CA
:1003D0000200F00101C08509F10A0000F00101C02E
:1003E0008509F10200F00104C08509F10200F00165
:1003F00005C08509F10200F00106C08509F102017E
:10040000F10200F00201C08509F10201F10200F0E1
:100410000202C085F10102F1010109F00500C08569
:10042000F1010009F00501C085F1010009F00502A4
:10043000C085F101004AFE525609F00503C085F15E
:10044000010009F00504C085F1010009F00600C0B3
:1004500085F10101F1010009F00601C085F10100FB
:10046000F1010109F00602C085F10101F101000965
:10047000F00608C085F10101F1010009F00603C092
:1004800085F10101F1010009F00606C085F10101C5
:10049000F1010009F10200F00607C085F10101F148
:1004A000010009F00702C085F1060009F00703C04A
:1004B00085F1060009F00704C085F1060009F0087F
:1004C00000C085F10103F10102F10101F101000910
:1004D000F00400C085F10102F1010109F00401C03E
:1004E00085F10103F10102F10101094D6F6E5475AF
:1004F0006557656454687246726953617453756ECA
:100500000000000300060009000C000F00124A6101
:100510006E4665624D61724170724D61794A756EC9
:100520004A756C4175675365704F63744E6F7644BE
:1005300065630000002300260029002C002F0032F4
:1005400000350038003B003E00410044FFFFFFFF44
:10055000FFFFFFFFFFFFFFFFFFFFFFFFFFFFFFFFAB
:10056000FFFFFFFFFFFFFFFFFFFFFFFFFFFFFFFF9B
:10057000FFFFFFFFFFFFFFFFFFFFFFFFFFFFFFFF8B
:10058000FFFFFFFFFFFFFFFFFFFFFFFFFFFFFFFF7B
:020000040802F0
:1000000000B583B04FF0000100914FF0F60301936B
:1000100008464FF007024FF0010303F0F7FB03B06F
:1000200000BD00BF10B54FF002004FF0F80116F010
:1000300023FF40F2B104C0F602044FF003004FF07A
:100040000001224604F0E6FB4FF0010040F2A5015A
:10005000C0F60201224604F0DDFB4FF0000001462D
:10006000224604F0D7FB4FF008004FF0090102468A
:1000700012F022FE4FF000004FF001014FF003029A
:1000800001F084FC4FF0010049F69A11C3F6996122
:1000900002F022FB4BF6E430C0F6030008F092FFBA
:1000A00010BD00BF08B54FF00A0001F0AFFA08BD5F
:1000B00008B521B94FF0030017F0E8FD08BD01298C
:1000C00004D14FF0010017F0E1FD08BD022903D172
:1000D0004FF0000017F0DAFD08BD00BF11B1012993
:1000E00016D108E040F28811C2F200010B781370BB
:1000F0004FF00000704740F21000C4F202000168A7
:1001000081F01003C3F3001010704FF0000070472F
:100110004FF01400704700BF11B1012928D11AE037
:1001200042F63C01C4F200010B6813F4004F42F6A2
:100130003C00C4F2000001684FEAC1534FEAD350BB
:1001400008BF404207EE100AF8EEC70AC2ED000AE7
:100150004FF00000704740F2FC10C2F20000D0EDFA
:10016000007AB8EE670A82ED000A4FF0000070478F
:100170004FF01400704700BF30B585B04FF0010557
:1001800000954FF00304019402954FF000004FF0EA
:1001900005012246034601F049F9009501940295B4
:1001A0004FF0000021462246034601F03FF94FF48C
:1001B00000504BF62441C0F6030140F20422C2F283
:1001C00000020BF0A5FB05B030BD00BF38B51446EA
:1001D0004FF000031370002940F0838040F20020AC
:1001E000C2F20000016800297ED142F62402C4F266
:1001F00000024FF0CA0515604FF05303136042F63A
:100200000800C4F20000016841F40025056003689D
:1002100043F4000101604FF0FF00106043F6400519
:10022000C4F202052A6842F001032B604BF65841E4
:10023000C0F60301086840F20003C4F2000318602E
:100240004FF0000540F20402C4F2000215604BF6C4
:100250000841C0F60301086840F20802C4F2000237
:10026000106040F22002C4F2000215604BF6044117
:10027000C0F60301086840F21C01C4F200010860E6
:100280004BF60C40C0F603000168116040F22C02EE
:10029000C4F200024FF0FF30106040F22801C4F2B7
:1002A00000010D801A8842F0010018804BF61040C2
:1002B000C0F603004FF0070140F29932C0F6020287
:1002C00007F000FF40F20023C2F2000318604FF075
:1002D000010140F28812C2F200021170217028461A
:1002E00038BD4FF0140038BD4FF0000038BD00BFDE
:1002F00070B508F0B3FB054643F2D30440F2100694
:10030000C4F2000608F0AAFB401BA04209D940F243
:100310008813C2F200034FF0050119704FF000007E
:1003200070BD07F0DBFE336803F010018AB2002ACB
:10033000E8D040F24000C4F20000006870BD00BF89
:1003400030B583B005460C464FF0F60001A94FF0DA
:10035000020203F0AFFDBDF80430C3F340222A705F
:100360004FEAC3514FEAD153236003B030BD00BF01
:1003700000B583B04FF0000360F3492361F3080335
:1003800002A820F8043D4FF002014FF0F60203F0FE
:100390002DFE03B000BD00BFF8B54FF000000146D0
:1003A00001F08EFE40F24003C4F200031B68FFF729
:1003B0009FFF0646002800F0F980FFF799FF0746E7
:1003C000002800F0F380861B304617F01BFE044621
:1003D0000D4687A3D3E9002318F076FA002862D1EE
:1003E0002046294684A3D3E9002318F089FA00287F
:1003F00059D140F2FC10C2F200000660FFF778FF0E
:100400000546002800F0D280C71BBE4294BFC6EB51
:100410000703C7EB0603012B66D940F2FC11C2F2B9
:1004200000010F60FFF764FF0446002800F0BE8063
:10043000461BB74294BFC7EB0603C6EB0703012B6D
:100440004FD940F2FC12C2F200021660FFF750FFD3
:100450000546002800F0AA80041BA64294BFC6EB04
:100460000403C4EB0603012B3ED940F2FC17C2F291
:1004700000073C60FFF73CFF0746002800F096802D
:10048000461BB44294BFC4EB0603C6EB0403012B26
:1004900029D940F2FC13C2F200031E60FFF728FFC7
:1004A000014640B982E040F28813C2F200034FF0E7
:1004B000020119707AE0C01BB04234BFC0EB0601E4
:1004C000C6EB000101290FD940F2FC12C2F2000272
:1004D000106040F28813C2F200034FF0020119705D
:1004E00064E03E4600E02646304617F08BFD0246AB
:1004F0000B4643A1D1E9000117F0AAFE17F06CFEEC
:1005000017F04EFE4FF000024FF00003C4F2E0037C
:1005100017F0E4FF3AA3D3E9002318F095F84FF061
:1005200000024FF00003C4F2400317F0D7FF17F0AA
:1005300053FE044618F000FA0546204617F030FE38
:1005400018F01EFF4FF000024FF00003C3F6E073F7
:1005500017F080FE17F0EAFD0446B0F5007F07D3E0
:1005600040F28810C2F200004FF0040202701DE059
:10057000003518BF01250DB1C0F50074284621468D
:1005800001F09EFD28462146FFF7F2FE38B940F201
:100590008813C2F200034FF00301197006E040F225
:1005A0008810C2F200004FF00002027042F62400F0
:1005B000C4F200004FF0CA0202604FF05303036020
:1005C00042F60802C4F2000211686FF3D3411160D1
:1005D00013686FF3D75313604FF0FF02026040F2CD
:1005E0000020C2F200004FF000010160F8BD00BF22
:1005F0000000000053126341000000004D136341EE
:1006000000000000D012634108B54FF440504BF693
:100610005C41C0F6030140F21822C2F200020BF066
:1006200077F908BD70B582B00C461646684611468B
:100630004FF0080219F09CFC009809F079FD40F297
:100640001023C2F200031860019809F071FD014601
:1006500040F21420C2F2000001600B2C00F2DD8099
:10066000DFE804F00613202D3A4754616EA2AFBCB8
:1006700040F21020C2F20000006818F03FFD40F286
:100680002423C2F200031860B4E040F21024C2F246
:100690000004206818F0E0F940F22422C2F20002BF
:1006A0001060A7E040F21023C2F20003186818F0AF
:1006B000CBFD40F22421C2F2000108609AE040F232
:1006C0001020C2F20000006818F0F6FB40F224226D
:1006D000C2F2000210608DE040F21021C2F200016F
:1006E000086818F0BBFB40F22424C2F2000420602A
:1006F00080E040F21022C2F20002106818F000FC04
:1007000040F22423C2F20003186073E040F210208C
:10071000C2F20000006818F0CBFE40F22424C2F2BE
:100720000004206066E040F21023C2F20003186863
:1007300018F02EFE40F22421C2F20001086059E0B8
:1007400040F21025C2F20005286817F029FD044682
:100750000D464FF000024FF0000318F099F860B119
:10076000204629464FF000024FF00003C3F6E07325
:1007700017F070FD17F0B2FC0BE0204629464FF051
:1007800000024FF00003C3F6E07317F061FD17F0AD
:10079000A5FC07EE100AF8EEC77A40F22422C2F256
:1007A0000002C2ED007A25E040F21020C2F2000003
:1007B000006818F01DFE40F22421C2F2000108601A
:1007C00018E040F21024C2F20004206818F08EFAFB
:1007D00040F22423C2F2000318600BE040F2102123
:1007E000C2F20001086818F0C7F940F22422C2F2F0
:1007F0000002106040F22421C2F20001086809F0F2
:100800006DFC00904FF000040194304669464FF0B3
:10081000080219F0ADFB204601E04FF0140002B0D1
:1008200070BD00BF4BF69043C0F603031A684EF646
:100830000C50CEF200000260FEE700BF08B5FFF7E3
:10084000F1FF00BF51E8002FBFF35F8F41E80003C5
:10085000012B3FF4F7AF1046704700BF13461A460E
:100860002DE9F00F0B460C460D460E460F46884606
:1008700089468A468B46092AC0F00780A0E8F80F0F
:10088000A2F10902092ABFF4F9AF4FF0080303FBF4
:1008900002F2144B1A44974600F020B800BF00BF84
:1008A000046000F01BB800BF80E8300000F016B80C
:1008B00080E8700000F012B880E8F00000F00EB898
:1008C00080E8F00100F00AB880E8F00300F006B814
:1008D00080E8F00700F002B880E8F00FBDE8F00F04
:1008E0007047134698080208EFF311804FF080011B
:1008F00081F3118870474FF0000000BF80F311882A
:10090000704700BF30B440F20003C0F6000340F26D
:100910008812C0F60002D01A4FEAA001B1F5C47FD8
:1009200004D81346264A9A4201D324E0FEE7254D17
:10093000254C601B20F003054FF0000340F200023D
:10094000C2F2000240F20001C0F6000105F104000D
:10095000C5F380045D589D5003F10403834226D102
:1009600009E05C589C5003F104035C58D45003F137
:1009700004038342F5D14EF60853CEF2000340F251
:100980000002C2F200021A604FF0B501CBF26B1107
:1009900043F25C50C2F2000001604EF61453CEF2F6
:1009A00000031A6842F01001196030BC7047002C37
:1009B000D7D05C589C5003F104038342D1D1DAE7CD
:1009C00000000008040000088B01000810B4034672
:1009D00000283ED002F1100440F20000C2F20000F4
:1009E00040F82430002A0ADA12F10C0F35DB02F14C
:1009F0000C024EF61850CEF2000011542DE04EF2CB
:100A00000014CEF200040F299CBF0901C9B24EF2B6
:100A10000043CEF20003D1541146002AB8BF02F1C0
:100A20001F014FEA611004EB80014FF01F03C8F271
:100A300000031340002B05DA03F1FF3262F01F03BD
:100A400003F1010358B24FF0010202FA00F30B6008
:100A500003E0002AC8DB024CD5E710BC704700BF9A
:100A600080E100E01EF0040F0CBFEFF30880EFF30D
:100A7000098020E9F00F00F001B800BF10B502684E
:100A800043F21053C2F200031A6041685960826851
:100A90009A60C168D96002691A61416959618269C5
:100AA0009A61C169D961026A1A62416A5962826AAD
:100AB0009A62C16AD962026B1A63416B5963826B95
:100AC0009A63C16BD96300F1400018644EF6285058
:100AD000CEF2000002685A641BF02AF8002800F0E9
:100AE000FB814BF69440C0F603001BF027F84EF64E
:100AF0002C54CEF200042368002B05DA4BF6A440F8
:100B0000C0F603001BF01AF84EF62C51CEF200018D
:100B1000086810F0020F05D04BF6B440C0F6030091
:100B20001BF00CF84EF62852CEF200025478002C3E
:100B300072D04BF6CC40C0F603001AF0FFFF4EF621
:100B40002853CEF20003597811F0010F05D04BF66F
:100B5000DC40C0F603001AF0F1FF4EF62850CEF24A
:100B60000000427802F00204E3B22BB14BF6FC40E5
:100B7000C0F603001AF0E2FF4EF62851CEF2000153
:100B8000487800F00402D4B22CB14BF62050C0F6E5
:100B900003001AF0D3FF4EF62853CEF20003597823
:100BA00001F00800C2B22AB14BF64450C0F603006F
:100BB0001AF0C4FF4EF62854CEF20004637803F016
:100BC0001001C8B228B14BF66450C0F603001AF009
:100BD000B5FF4EF62852CEF20002547804F02003FE
:100BE000D9B229B14BF68450C0F603001AF0A6FF23
:100BF0004EF62850CEF20000427802F08004E3B2B4
:100C000053B14EF63851CEF2000109684BF6A450AC
:100C1000C0F603001AF092FF4EF62850CEF2000004
:100C2000428894B2002C5ED04BF6C450C0F603004C
:100C30001AF084FF4EF62853CEF20003598811F0C3
:100C4000010F05D04BF6D450C0F603001AF076FF22
:100C50004EF62850CEF20000428802F00204A3B201
:100C60002BB14BF60060C0F603001AF067FF4EF69A
:100C70002851CEF20001488800F0040294B22CB151
:100C80004BF62460C0F603001AF058FF4EF62853C6
:100C9000CEF20003598801F0080082B22AB14BF667
:100CA0006460C0F603001AF049FF4EF62854CEF2F5
:100CB0000004638803F4807188B228B14BF6946015
:100CC000C0F603001AF03AFF4EF62852CEF20002A8
:100CD000548804F4007399B229B14BF6B060C0F6A1
:100CE00003001AF02BFF4EF62850CEF200000278D7
:100CF000002A63D04BF6C860C0F603001AF01EFF4E
:100D00004EF62854CEF20004237813F0010F05D0DC
:100D10004BF6D860C0F603001AF010FF4EF62851CB
:100D2000CEF20001087800F00202D4B22CB14BF6EA
:100D3000F860C0F603001AF001FF4EF62853CEF219
:100D40000003197801F00800C2B22AB14BF6107006
:100D5000C0F603001AF0F2FE4EF62854CEF200045C
:100D6000237803F01001C8B228B14BF63470C0F6F6
:100D700003001AF0E3FE4EF62852CEF20002147879
:100D800004F02003D9B229B14BF65870C0F6030025
:100D90001AF0D4FE4EF62850CEF20000027802F08F
:100DA0008004E3B253B14EF63451CEF2000109682B
:100DB0004BF67870C0F603001AF0C0FE43F21054F0
:100DC000C2F20004216A4BF6A470C0F603001AF0C8
:100DD000B5FE616A4BF6B870C0F603001AF0AEFEBD
:100DE000A16A4BF6CC70C0F603001AF0A7FEE16AC8
:100DF0004BF6E070C0F603001AF0A0FE21684BF637
:100E0000F470C0F603001AF099FE61684CF2080015
:100E1000C0F603001AF092FEA1684CF21C00C0F666
:100E200003001AF08BFEE1684CF23000C0F60300BC
:100E30001AF084FE21694CF24400C0F603001AF057
:100E40007DFE61694CF25800C0F603001AF076FE90
:100E5000A1694CF26C00C0F603001AF06FFEE16964
:100E60004CF28000C0F603001AF068FE216B4CF2D1
:100E70009400C0F603001AF061FE216C4CF2A80049
:100E8000C0F603001AF05AFE616B4CF2BC00C0F6CB
:100E900003001AF053FEA16B4CF2E000C0F6030011
:100EA0001AF04CFE43F25850C2F2000002684CF2B5
:100EB0000410C0F60300114612681AF03FFE40F617
:100EC0003C13C2F200031A684CF21C10C0F6030077
:100ED000114612681AF032FEFFF7B0FC10BD00BFD9
:100EE00000B507F0A1FA002808BF5DF804FBEFF396
:100EF0000981EFF3118221E9F40F5DF804EB1EF094
:100F0000100F08BF21ED108A41F804ED0B4C226848
:100F1000002A18BF516007F0F9FA2268516851F8A9
:100F200004EB1EF0100F08BFB1EC108AB1E8F40F0B
:100F300082F3118881F3098870470000583500203A
:100F400008B540F6E160C0F602004FF0FF016FF017
:100F50000102FFF73BFD08BDF8B507460C461E46EB
:100F60000799089D14F0030F00D0FEE722B1A4EB0F
:100F70008500A0F1480401E004F14800012D01D8EA
:100F8000A16205E02A4602F0D3F9A7EB8507A76224
:100F90004FF0000363604FF01130E0624FF02231F8
:100FA00021634FF0333262634FF04433A3604FF05C
:100FB0005530E0604FF0663121614FF07732626169
:100FC0004FF08833A3614FF09930E0614FF0AA31C0
:100FD00021624FF0BB3262624FF0CC33A363E66311
:100FE000069820644FF0807161646FF00202226005
:100FF00005F11200F8BD00BF62B64EF60453CEF202
:1010000000031A6842F08050186000BF4FEA0010D9
:101010004CF23413C0F603031A584CF6CC41C0F618
:10102000030151F82200704738B504460D46FFF71A
:10103000EDFF4CF23413C0F6030303EB04146168B4
:10104000012902D0022903D101E0856038BD456144
:1010500038BD00BF2DE9F84F40F20401C4F202018F
:101060000C684CF25422C0F60302136824EA03040D
:101070004CF22C25C0F60305286844EA00060E60F1
:1010800040F20447C4F202073968546821EA0401B7
:101090006B6841EA0300386040F60406C4F20206B9
:1010A0003768916827EA0107AC6847EA04033360B0
:1010B00040F60446C4F202063768D06827EA000703
:1010C000E96847EA0104346041F20406C4F202060A
:1010D0003368126923EA02032D6943EA0507376082
:1010E00041F20440C4F202000168016041F60404C8
:1010F000C4F202042668266041F60443C4F20203E7
:101100001A681A6042F20405C4F202052F682F60C3
:1011100040F20C01C4F202010C684CF20826C0F641
:101120000306306824EA00044CF2CC33C0F6030313
:101130001A6844EA02050D6040F20C47C4F2020747
:101140003968746821EA0401586841EA00023A608B
:1011500040F60C05C4F202052F68B16827EA0107C2
:101160009C6847EA0400286040F60C42C4F2020280
:101170001568F76825EA0705D96845EA010414608F
:1011800041F20C05C4F202052868366920EA06001F
:101190001B6940EA03022A6041F20C47C4F20207CD
:1011A0003968396041F60C04C4F2020425682560F0
:1011B00041F60C40C4F202000668066042F20C03DD
:1011C000C4F202031A681A604CF27827C0F60307CB
:1011D000396840F2140EC4F2020ECEF800107C689A
:1011E00040F21441C4F202010C60BD6840F6140CD8
:1011F000C4F2020CCCF80050FE6840F61440C4F271
:10120000020006603B6941F21402C4F2020213605C
:101210004FF0000341F21447C4F202073B6041F66D
:101220001404C4F20204236041F61445C4F202051A
:101230002B6042F21406C4F20206336040F2000052
:10124000C4F2020007684CF21434C0F603042268AA
:1012500027EA02074CF27816C0F60306356847EA1B
:10126000050040F20007C4F20207386040F2004B6C
:10127000C4F2020BDBF80020656822EA0502706800
:1012800042EA0007CBF8007040F6000AC4F2020AF6
:10129000DAF80020A56822EA0502B06842EA0007F1
:1012A000CAF8007040F60049C4F20209D9F80020DB
:1012B000E56822EA0502F06842EA0007C9F8007012
:1012C00041F20008C4F20208D8F80020246922EA9A
:1012D000040236693243C8F8002041F20047C4F2E4
:1012E00002073D683D6041F60006C4F20206306820
:1012F000306041F60045C4F202052A682A6042F2D5
:101300000004C4F20204206820604CF2CC22C0F633
:1013100003021068CEF80000506808609168CCF8AD
:101320000010D16840F61440C4F202000160126956
:1013300041F21401C4F202010A6041F21440C4F205
:101340000200036041F61402C4F20202136041F687
:101350001441C4F202010B6042F21400C4F2020014
:1013600003604FF0320008F03BFE40F20003C4F28D
:10137000020318684CF25412C0F60302116820EA06
:1013800001004CF2F023C0F603031968014340F258
:101390000000C4F202000160DBF80000516820EA9E
:1013A000010059680843CBF80000DAF800009168A2
:1013B00020EA010099680843CAF80000D9F8000043
:1013C000D16820EA0100D9680843C9F80000D8F8BC
:1013D0000010126921EA02011B6941EA0300C8F802
:1013E000000039683960326832602B682B602068F1
:1013F00020604FF0010004F0CFFBBDE8F88F00BF84
:1014000008B543F63002C4F2020213686FEA5320B3
:101410006FEA4021116043F62003C4F201031A6809
:1014200042F001001860FFF715FE08BD2DE9F0013C
:101430009DF814709DF81860079D4CF2B414C0F626
:10144000030454F820004FEA4104FF2F12D0D0F8D3
:101450000C804CF2AC1CC0F6030C1CF8077007FAA9
:1014600004FC4FF0030707FA04F728EA07074CEAE1
:101470000707C760FF2B10D0D0F804C04CF2C83764
:10148000C0F60307FF5C07FA01F74FF0010303FA08
:1014900001F32CEA03033B434360FF2E0FD0876820
:1014A0004CF2A013C0F603039E5D06FA04F64FF05B
:1014B000030303FA04F327EA030333438360B5F11C
:1014C000FF3F16D04FEAD10303F1080350F8236021
:1014D00001F007014FEA810105F00F0505FA01F55A
:1014E0004FF00F0707FA01F126EA0101294340F8FE
:1014F0002310FF2A10D001684CF2A413C0F6030396
:101500009B5C03FA04F34FF0030202FA04F421EAAD
:10151000040143EA01040460BDE8F001704700BF24
:101520002DE9F007079F089E099D4CF2B414C0F600
:10153000030454F820004FEA41044FEAD10801F0B7
:10154000070C4FEA8C0C6FB1D0F80C9029FA04FA12
:101550000AF003094CF2502AC0F6030A1AF809905F
:1015600087F8009053B1476827FA01F101F00101B3
:101570004CF29C17C0F60307795C197056B183686A
:1015800023FA04F303F003034CF2A811C0F603019D
:10159000CB5C337045B108F1080850F8281021FAE7
:1015A0000CFC0CF00F032B6052B1006820FA04F41D
:1015B00004F003044CF2B011C0F603010B5D13708C
:1015C000BDE8F007704700BF4CF26833C0F6030374
:1015D00053F820100A684CF2D813C0F6030353F8EE
:1015E00020100A404CF29833C0F6030353F8200051
:1015F000824214BF00200120704700BF4CF2B41398
:10160000C0F6030353F82000006970474CF2D8136A
:10161000C0F6030353F820307BB139B14CF23831B6
:10162000C0F6030151F82020136070474CF29C2251
:10163000C0F6030252F82000036070473A2800F217
:10164000938000EB80004CF2F033C0F6030353F8B4
:10165000202002F1FF300D2800F28680DFE800F044
:10166000071019222B343D464F58616A737C43F6AC
:101670004400C4F20200036861F300030360704792
:1016800043F64003C4F202031A6861F300021A60D1
:10169000704743F64003C4F20203186861F3410047
:1016A0001860704743F64000C4F20200026861F31C
:1016B00082020260704743F64000C4F202000368F1
:1016C00061F3C3030360704743F64003C4F20203AF
:1016D0001A6861F304121A60704743F64003C4F2BB
:1016E0000203186861F345101860704743F6440020
:1016F000C4F20200026861F341020260704743F6DF
:101700004400C4F20200036861F3104303607047B1
:1017100043F64403C4F202031A6861F351421A60AB
:10172000704743F64403C4F20203186861F3924021
:101730001860704743F64000C4F20200026861F38B
:1017400086120260704743F64000C4F2020003684C
:1017500061F3C7130360704743F64003C4F202030A
:101760001A6861F308221A60704700BF00EB80001E
:101770004CF2F033C0F6030353F820204CF610511E
:10178000C0F6030151F82200704700BF2DE9F84F61
:1017900004468A46914698469DF928709DF92C602A
:1017A0009DF930503A2800F2B680FFF7DFFF04EBD6
:1017B00084024CF2F033C0F6030303EB82035A6851
:1017C000022A94BF8369C369016A02F1FF3CBCF13C
:1017D000030F2ED8DFE80CF0021802186FF3010394
:1017E000BAF1000FC8BF6AF38203B9F1000FC8BF96
:1017F00069F3C303B8F1000FC8BF68F30613002FE5
:1018000017DD67F3C71314E06FF30923BAF1000F74
:10181000C8BF6AF38A23B9F1000FC8BF69F3CB23AD
:10182000B8F1000FC8BF68F30E33002FC8BF67F3CD
:10183000CF3302F1FF37032F44D8DFE807F002145B
:101840002638332C04D1002E06DD66F3820103E036
:10185000002EC8BF66F30001002DC8BF65F341012B
:101860006FF3C30130E0362C04D1002E06DD66F3A1
:10187000861103E0002EC8BF66F30411002DC8BF17
:1018800065F345116FF3C7111EE0382C04D1002E0B
:1018900006DD66F38A2103E0002EC8BF66F3082147
:1018A000002DC8BF65F349216FF3CB210EE0002E58
:1018B000C8BF66F30C31002DC8BF65F34D316FF31F
:1018C000CF3103E0022A01D8836100E0C3610162E5
:1018D00004EB84044CF2F030C0F6030050F82430DE
:1018E000012B02D0082B16D10BE04CF68C03C0F66E
:1018F00003031A6840F24401C4F201010A60BDE822
:10190000F88F4CF68C02C0F60302116840F2444096
:10191000C4F201000160BDE8F88F00BF38B504468D
:101920000D46FFF723FF04EB84014CF2F033C0F6C1
:10193000030303EB8104626802F1FF3103290AD833
:10194000DFE801F002040608456338BD856338BD51
:10195000C56338BD056438BD40F22823C2F20003D8
:1019600018684FF000020261016801F01003002BBB
:101970000CBF01204FF0FF3040F22C23C2F20003D5
:101980001A8810FA82F188B2188070472DE9F04F5A
:1019900089B0154640F22823C2F200034FF000023E
:1019A0001A604FEA01104CF69404C0F60304245860
:1019B000142900F2F480092C00F2F4804CF6FC1398
:1019C000C0F6030353F82430002B00F0EE804FEAFA
:1019D00005124CF69400C0F603008258944240F081
:1019E000E78004F1FF36072E4DD8DFE806F0340417
:1019F000101C284C4C4043F64007C4F202073868DC
:101A000040F001023A604FF0000605963EE043F6D2
:101A10004007C4F20207386840F002023A604FF013
:101A20000106059632E043F64007C4F20207386823
:101A300040F004023A604FF00106059626E043F6B6
:101A40004007C4F20207386840F008023A604FF0DD
:101A5000000605961AE043F64407C4F20207386808
:101A600040F001023A604FF0010605960EE043F6A1
:101A70004407C4F20207386840F002023A604FF0AF
:101A80000106059602E04FF00107059740F2282075
:101A90008246C2F2000ACAF800304CF69409C0F639
:101AA000030909EB011898F804B0D8F8081004915C
:101AB0000DF11F0300934FF0000601960296584661
:101AC00032460DF11E03FFF72BFD9DF81E309DF8E9
:101AD0001F2000924FF003070197D8F80C000290E6
:101AE000584604993A46FFF7A1FC09EB051595F80D
:101AF0000490D5F808800DF11F010091019602961F
:101B00004846414632460DF11E03FFF709FD9DF898
:101B10001F3000930197EA680292484641463A46D0
:101B20003346FFF783FCDAF800104CF62420C0F6A9
:101B3000030003680B604CF69002C0F603021068C5
:101B400088604CF6F813C0F603031A688A610E62C7
:101B50006FF07F40C862059B93B14CF6F412C0F65B
:101B600003021068C86041F65910C0F602004FF039
:101B70000F014CF6E413C0F603031A57FEF726FFD5
:101B800040F22821C2F2000108684FF00002826290
:101B9000036843F0010101604FF001000AE04FF0DB
:101BA000000007E04FF0000004E04FF0000001E00B
:101BB0004FF0000009B0BDE8F08F00BF40F22823CD
:101BC000C2F200031B689BB1A8B91A686FF3000248
:101BD0001A604FF00000586240F22C21C2F200015E
:101BE00008801A6842F0010018604FF00100704749
:101BF0004FF0000070474FF00000704710B483B002
:101C000040F22823C2F200031B6803B310BB40F26A
:101C10002C22C2F20002586A148840EA0440019063
:101C200000BF00BF00BF00BF00BF586A148840EA71
:101C300004400090019C00988442ECD1DDED017AD3
:101C4000B8EEE70A81ED000A4FF0010004E04FF022
:101C5000000001E04FF0000003B010BC704700BF6F
:101C600040F22823C2F200031B689BB1A8B91A688E
:101C70006FF300021A6059624FEA114140F22C20C2
:101C8000C2F2000001801A6842F0010119604FF0B1
:101C9000010070474FF0000070474FF000007047A0
:101CA00043F67403C4F20203186847F20402C4F254
:101CB0000002136840F22E22C2F200024FF000012F
:101CC000117013F0010F04D010464FF0040202709F
:101CD0003EE04FEA106212F0600F07D040F22E2172
:101CE000C2F200014FF020030B7031E002F004015A
:101CF000C9B239B140F22E20C2F200004FF04002CA
:101D0000027025E0C3F3400343EAD06010F0010FF6
:101D100007D040F22E21C2F200014FF080030B7079
:101D200016E002F01001CBB23BB140F22E20C2F21D
:101D300000004FF0010202700AE002F00202D0B28D
:101D400030B140F22E21C2F200014FF002030B70BD
:101D500043F67401C4F202010B6843F0807008601E
:101D600047F20001C4F200010A6842F008030B6068
:101D700043F25850C2F20000016840F23022C2F231
:101D800000021160704700BF40F22E23C2F2000330
:101D90001878704708B547F61021C1F6FF714FF06B
:101DA0000C0218F0E5F84FF00C0008BD00B583B048
:101DB00043F64003C4F202031A6842F080501860F0
:101DC00047F20001C4F200010B6843F480720A601C
:101DD0000DF107006946FEF7B3FA43F67001C4F24D
:101DE00002010A684CF64C23C0F6030319684A4006
:101DF0004CF64423C0F6030319680A421FD1F0B120
:101E000042F63C00C4F2000002684FEAC2534FEAB7
:101E1000D3510098814212D142F63C02C4F2000232
:101E20001368C3F3C0319DF80700814207D140F227
:101E30003423C2F200034FF001021A700BE04CF69B
:101E40003020C0F603004FF0070142F22D12C0F619
:101E5000020206F037F903B000BD00BF70B50646B8
:101E600040F23424C2F2000442F60C05C4F200052C
:101E700003E000F0C9FA06F031F92378002BF8D01E
:101E8000286810F0200FF4D042F60001C4F20001DF
:101E90000A6842F60403C4F200031B68C2F302108E
:101EA00000EB800102F00F0000EB41013160C2F352
:101EB000023000EB8001C2F3032000EB41017160AE
:101EC000C2F3015000EB8001C2F3034202EB410078
:101ED000B060C3F3072101F0E002E02A14BFC3F3AE
:101EE00042320022B261C3F3011000EB800203F022
:101EF0000F0101EB4200F060C3F300324FEA8201B0
:101F00008818C3F3032202EB400101F1FF30306176
:101F1000C3F3035202EB8201C3F3034303EB41001B
:101F200000F16400706170BD70B58AB0014601A80F
:101F30004FF0240218F01CF801A817F03FFE059C92
:101F400004F10104E4B2019A46F26763C6F26663E3
:101F500083FB02104FEAE271C1EBA0054FF00006CF
:101F600065F3061605EB8500A2EB400262F303065B
:101F7000029D83FB05104FEAE571C1EBA00262F3FD
:101F80000E3602EB8200A5EB400565F30B26039AA3
:101F900083FB02034FEAE271C1EBA30060F3155625
:101FA00000EB8005A2EB450262F31346079B13B1D9
:101FB00003F0070101E04FF007014FF0000561F366
:101FC0004F35049946F26762C6F2666282FB0130C1
:101FD0004FEAE173C3EBA00060F3051500EB80034B
:101FE000A1EB430161F303054CF6CD40CCF6CC40A8
:101FF000A0FB04034FEAD30161F30C3501EB810030
:10200000A4EB400464F30B25069982FB01304FEAF0
:10201000E173C3EBA00382FB03024FEAE370C0EB62
:10202000A20202EB8200A3EB400262F3175503EB1E
:102030008303A1EB430161F3134540F23420C2F264
:102040000000027852B940F23424C2F2000400F0D9
:10205000DBF906F043F82378002BF8D042F6240190
:10206000C4F200014FF0CA0008604FF053020A604A
:1020700042F60C03C4F20003196841F080001860B6
:102080001A46136813F0400FFBD042F60001C4F269
:1020900000010E6042F60400C4F20000056042F642
:1020A0000C03C4F200031A686FF3C7121A6042F6F9
:1020B0002401C4F200014FF0FF0008600AB070BDB7
:1020C00070B506460D46B1F5007F2ED242F60C03E0
:1020D000C4F20003186810F4803F09D042F60C04E3
:1020E000C4F2000405F0FAFF216811F4803FF9D131
:1020F00042F62403C4F200034FF0CA021A604FF004
:10210000530018604FF0000242F61801C4F20001BB
:102110000A6065F3080266F3CF3242F63C00C4F26F
:10212000000002604FF0FF021A6070BD30B583B04E
:102130000DF107006946FEF703F905464CF6482302
:10214000C0F603031A6843F67000C4F2020002608E
:102150004CF64C21C0F603010B680360026812F0D4
:10216000020F09D143F67004C4F2020405F0B6FF71
:10217000206810F0020FF9D042F62401C4F20001E9
:102180004FF0CA030B604FF053020A6042F60C0096
:10219000C4F20000016841F080030360026812F09D
:1021A000400F09D142F60C04C4F2000405F096FF7A
:1021B000206810F0400FF9D04CF62821C0F603013A
:1021C0000A6842F61003C4F200031A601A604CF663
:1021D0002C20C0F60300016842F60802C4F2000297
:1021E000116042F60C03C4F2000318686FF3C710C5
:1021F000186042F62401C4F200014FF0FF020A60A9
:102200002DB19DF807000099FFF75AFF04E04FF049
:1022100000000146FFF754FF40F23423C2F20003EE
:102220004FF00100187003B030BD00BF0000000087
:1022300010B542F20803CEF204031A6842F010000F
:10224000186042F2E920C0F602004FF00F014FF093
:102250003602FEF7BBFB43F64001C4F202010C68F4
:1022600044F010030B6041F20004C4F200044CF689
:102270005022C0F60302106820604CF6D441C0F62C
:102280000301886915F0BEFE15A3D3E9002316F0FB
:1022900025F94FF000024FF00003C3F6F07315F07C
:1022A000D7FF15F043FF41F22C03C4F2000318805E
:1022B00041F22800C4F200004FF0000202804CF608
:1022C0005421C0F60301086841F20C03C4F2000374
:1022D0001860228842F00101218010BDAFF3008018
:1022E0002D431CEBE2362A3F684620F007018D465D
:1022F00001B541F21003C4F200034FF000021A606E
:1023000006F0B6FBBDE801408546704770B504464F
:10231000B0F5CC7F2FD940F23233984216D940F233
:102320006560844215D940F6CB418C4214D941F600
:102330009712944213D943F22F36B44212D946F27F
:102340005F639C4298BF06250ED90FE04FF0010550
:102350000AE04FF0020507E04FF0030504E04FF0FC
:10236000040501E04FF00505072D06D1FEF766FADA
:102370004FF0070501E04FF00005FEF7B5FA0646FD
:1023800004EB84044FEAC4004CF65821C0F6030164
:1023900051F83520B0FBF2F39CB2012C05D9B4F50D
:1023A000805F04D3FEF74AFA01E04FF0020443F2E3
:1023B0000000C4F2000045F2555101604CF658226D
:1023C000C0F6030202EBC5052B7943F20401C4F207
:1023D00000010B6043F20802C4F2000214604AF6E6
:1023E000AA2303603046FEF789FA70BD08B543F2B0
:1023F0000003C4F200034CF6CC421A604FF0C80050
:10240000FFF784FF08BD00BF43F20003C4F20003DE
:102410004AF6AA221A60704710B5044643F2100328
:10242000C4F20003186810F0010F74D04FF03200AE
:1024300007F0D6FD43F21001C4F200010A6812F061
:10244000010F68D04FF0320007F0CAFD43F21003CD
:10245000C4F20003186810F0010F5CD04FF0320096
:1024600007F0BEFD43F21001C4F200010A6812F049
:10247000010F50D04FF0320007F0B2FD43F21003CD
:10248000C4F20003186810F0010F44D04FF032007E
:1024900007F0A6FD43F21001C4F200010A6812F031
:1024A000010F38D04FF0320007F09AFD43F21003CD
:1024B000C4F20003186810F0010F2CD04FF0320066
:1024C00007F08EFD43F21001C4F200010A6812F019
:1024D000010F20D04FF0320007F082FD43F21003CD
:1024E000C4F20003186810F0010F14D04FF032004E
:1024F00007F076FD43F21001C4F200010A6812F001
:10250000010F08D04FF0320007F06AFD43F21003CC
:10251000C4F200031B682046FFF7F8FE10BD00BFA1
:1025200002469CF8043043B1DCF8000040B140F2B0
:10253000C021C2F2000141F82200DCF8000050B9CD
:1025400040F2C023C2F2000353F8220049F6404291
:10255000002808BF104670474FF0010303FA00F04F
:1025600010F4E26F0CBF00200120704770B50D46DB
:102570004CF6C823C0F6030353F82040002C45D086
:1025800000EB800040F23826C2F2000606EBC006DF
:1025900030464FF0000105F08DF9122D07D142F2BF
:1025A0000431C4F201010A6842F480030B60606BDD
:1025B00065F304006063E36C4FF0050007F010FD65
:1025C000A16841F08042A260236813F0020FFBD0A3
:1025D000E46C122D16D142F20430C4F201000168FD
:1025E0006FF39651016042F20002CEF204021368CA
:1025F0004FEA03504FEA105140F2194291420CBF8A
:10260000A4006400304605F063FA01E04FF0FF34A7
:10261000204670BDF8B504460F464CF6B423C0F60C
:10262000030303EB80056E88002E53D013F82000BF
:10263000012803D16878FFF799F801E04FF0000016
:102640005FB940F2B020C2F2000000EB84044FF00A
:10265000000121604FF000012BE0BE420BD840F298
:10266000B022C2F2000202EB84044FF07E532360DA
:102670004FF6FF711DE02A78012A0CBFC16A40F6AF
:10268000FF7140F2B023C2F2000303EB840406EEB4
:10269000907AB8EE667A00EE101AF8EE407AC7EE3D
:1026A000270AC4ED000A06F1FF3007FB0101B1FB68
:1026B000F6F12A78012A03D16878FFF72FF9F8BDDF
:1026C000022A07D1687840F6FF73994228BF19465D
:1026D000FEF7AAFCF8BD00BF38B52DED028B04460D
:1026E00008EE101A4CF6B425C0F6030505EB80057C
:1026F000F7EE007AB4EEE78AF1EE10FA09DC08464C
:1027000016F01AF900289FED260A18BFB0EE408A8D
:1027100001E0B7EE008A2B78012B1CD16878FFF717
:1027200025F8D0ED0B1A6D78B8EE612A62EE082A12
:1027300012EE900A15F034FD4FF000024FF0000346
:10274000C3F6E07315F086FD15F0F0FC014628464F
:10275000FFF7E4F818E0022B16D16D78DFED110ACF
:1027600028EE201A11EE100A15F01AFD4FF00002A3
:102770004FF00003C3F6E07315F06CFD15F0D6FCC6
:1027800001462846FEF750FC40F2B020C2F200009D
:1027900000EB840484ED008ABDEC028B38BD00BFE1
:1027A0000000000000F07F4510B54FF000044FF02E
:1027B00000002146FFF790FF4FF001002146FFF790
:1027C0008BFF4FF002002146FFF786FF4FF003001A
:1027D0002146FFF781FF40F20C03C4F202031A689E
:1027E0001A6040F20C40C4F202000168016040F639
:1027F0000C03C4F202031A684CF60430C0F603005E
:10280000816822EA01024CF69020C0F6030081683C
:102810000A431A6040F60C43C4F202031A681A60B5
:1028200041F20C00C4F202000168016041F20C4365
:10283000C4F202031A681A6041F60C00C4F20200E6
:102840000168016041F60C43C4F202031A681A6081
:1028500042F20C00C4F202000168016040F2000381
:10286000C4F202031A681A6040F20040C4F2020087
:102870000168016040F60003C4F202031A684CF6D6
:102880003430C0F60300816822EA01024CF6D420FD
:10289000C0F6030081680A431A6040F60043C4F2A0
:1028A00002031A681A6041F20000C4F202000168D3
:1028B000016041F20043C4F202031A681A6041F653
:1028C0000000C4F202000168016041F60043C4F256
:1028D00002031A681A6042F20000C4F202000168A2
:1028E000016010BD08B502280ED84CF63033C0F692
:1028F0000303195CFF290AD04CF65C32C0F60302D0
:10290000105CFFF733FE08BD4FF0FF3008BD4FF0FD
:10291000FF3008BD10B50446FFF7E4FF07EE900A4C
:10292000B8EE677A4CF63033C0F60303185D112811
:102930000BD147F62A21C1F6FF710A8801EE102A51
:10294000F8EEC11AC1EE870A03E09FED030AC7EE55
:10295000000A10EE900A10BD00F07F4540F2B0234F
:10296000C2F2000303EB80000068704738B50D46E3
:10297000044600B30E2801D9FDF760FF4CF6D4439E
:10298000C0F6030353F8240055B1B0FBF5F14FEA4C
:10299000114202F10103B0FBF3F0B0FBF5F502E0E8
:1029A0004FF000052A464CF61051C0F6030151F8CD
:1029B00024309A62DD6238BD10B582B000918DF886
:1029C0000420042840F0E2804FF00000FFF7C4FD2F
:1029D00048B1EC464FF00000FFF7A2FD01464FF072
:1029E0000000FFF7C3FF4FF00100FFF7B5FD48B14E
:1029F000EC464FF00100FFF793FD01464FF0010058
:102A0000FFF7B4FF4FF00200FFF7A6FD48B1EC4618
:102A10004FF00200FFF784FD01464FF00200FFF780
:102A2000A5FF4FF00300FFF797FD48B1EC464FF0CC
:102A30000300FFF775FD01464FF00300FFF796FF17
:102A40004FF00400FFF788FD48B1EC464FF004005A
:102A5000FFF766FD01464FF00400FFF787FF4FF0D8
:102A60000500FFF779FD48B1EC464FF00500FFF790
:102A700057FD01464FF00500FFF778FF4FF00600C5
:102A8000FFF76AFD48B1EC464FF00600FFF748FD3E
:102A900001464FF00600FFF769FF4FF00700FFF710
:102AA0005BFD48B1EC464FF00700FFF739FD0146EA
:102AB0004FF00700FFF75AFF4FF00800FFF74CFDFB
:102AC00048B1EC464FF00800FFF72AFD01464FF0F1
:102AD0000800FFF74BFF4FF00900FFF73DFD48B13D
:102AE000EC464FF00900FFF71BFD01464FF00900CF
:102AF000FFF73CFF4FF00A00FFF72EFD48B1EC4610
:102B00004FF00A00FFF70CFD01464FF00A00FFF7F7
:102B10002DFF4FF00B00FFF71FFD48B1EC464FF0C3
:102B20000B00FFF7FDFC01464FF00B00FFF71EFF07
:102B30004FF00C00FFF710FD48B1EC464FF00C00D1
:102B4000FFF7EEFC01464FF00C00FFF70FFF4FF0D0
:102B50000D00FFF701FD48B1EC464FF00D00FFF707
:102B6000DFFC01464FF00D00FFF700FF4FF00E00B5
:102B7000FFF7F2FC48B3EC464FF00E00FFF7D0FC35
:102B800001464FF00E00FFF7F1FE1EE04CF6B423B5
:102B9000C0F6030313F82010012916D14CF6B42215
:102BA000C0F6030202EB8000447804EB84034CF28D
:102BB000F031C0F6030151F82340EC462046FFF700
:102BC000AFFC01462046FFF7D1FE02B010BD00BFAA
:102BD00070B584B040F23825C2F200054CF60034DE
:102BE000C0F603042846214604F04CFE05F12800F7
:102BF000214604F047FE05F15000214604F042FE54
:102C000043F64403C4F202031A6842F48070186069
:102C1000196841F400761E604CF62C35C0F60305A9
:102C20002C6842F20433C4F201031C604CF6F82213
:102C3000C0F60302106842F20401C4F20101086008
:102C400042F20416C4F2010630604CF6C425C0F608
:102C500003052C6842F20C03C4F201031C6042F22B
:102C60000C12C4F2010214604CF65830C0F6030096
:102C7000016842F21006C4F20106316042F21015FA
:102C8000C4F2010529604CF66034C0F603042368E1
:102C900042F22C02C4F20102136042F22C10C4F280
:102CA000010003604CF6FC21C0F603010E6842F2FD
:102CB0000805C4F201052E6042F20814C4F20104B2
:102CC00026604FF016004FF00101FEF7B7FC4FF001
:102CD00008004FF00101FEF7B1FC4FF00C004FF07F
:102CE0000101FEF7ABFC4FF005004FF00101FEF7CC
:102CF000A5FC4FF0000400944FF0010601960294E9
:102D00004FF01600214632464FF00603FEF73EFD17
:102D10004CF2F035C0F6030595F8C401D5F8C8119A
:102D200000940194D5F8C03102934FF0030223467A
:102D3000FEF77CFB0094019602944FF008002146B8
:102D400032464FF00603FEF721FD95F8AC00D5F8AA
:102D5000B01000940194D5F8A82002924FF003021D
:102D60002346FEF763FB0094019602944FF00C009B
:102D7000214632464FF00603FEF708FD95F8FC00A9
:102D8000D5F8001100940194D5F8F83002934FF073
:102D900003022346FEF74AFB0094019602944FF08B
:102DA0000500214632464FF00603FEF7EFFC95F88A
:102DB0007000696F00940194ED6E02954FF003026C
:102DC0002346FEF733FB4FF0040021462246FFF76F
:102DD000F3FD4FF0000520462946FFF77DFC304605
:102DE0002946FFF779FC4FF002002946FFF774FCF3
:102DF0004FF003002946FFF76FFC3046FFF7ACFBAE
:102E000050B14CF61050C0F6030041684CF6283221
:102E1000C0F6030213680B604FF00200FFF79CFB43
:102E200050B14CF61050C0F6030081684CF62832C1
:102E3000C0F6030213680B604FF00300FFF78CFB32
:102E400050B14CF61050C0F60300C1684CF6283261
:102E5000C0F6030213680B604FF00400FFF77CFB21
:102E600050B14CF61050C0F6030001694CF6283200
:102E7000C0F6030213680B604FF00500FFF76CFB10
:102E800050B14CF61050C0F6030041694CF62832A0
:102E9000C0F6030213680B604FF00600FFF75CFBFF
:102EA00050B14CF61050C0F6030081694CF6283240
:102EB000C0F6030213680B604FF00700FFF74CFBEE
:102EC00050B14CF61050C0F60300C1694CF62832E0
:102ED000C0F6030213680B604FF00800FFF73CFBDD
:102EE00050B14CF61050C0F60300016A4CF628327F
:102EF000C0F6030213680B604FF00900FFF72CFBCC
:102F000050B14CF61050C0F60300416A4CF628321E
:102F1000C0F6030213680B604FF00A00FFF71CFBBA
:102F200050B14CF61050C0F60300816A4CF62832BE
:102F3000C0F6030213680B604FF00B00FFF70CFBA9
:102F400050B14CF61050C0F60300C16A4CF628325E
:102F5000C0F6030213680B604FF00C00FFF7FCFA99
:102F600050B14CF61050C0F60300016B4CF62832FD
:102F7000C0F6030213680B604FF00D00FFF7ECFA88
:102F800050B14CF61050C0F60300416B4CF628329D
:102F9000C0F6030213680B604FF00E00FFF7DCFA77
:102FA00050B14CF61050C0F60300816B4CF628323D
:102FB000C0F6030213680B60FFF7F6FB04B070BDA8
:102FC00010B504464FF000004FF01101FFF7CEFAA4
:102FD00047F62A23C1F6FF73198807EE901AB8EE58
:102FE000670A06EE900AB8EE667AC0EE070AC4EDEC
:102FF000000A4FF0010010BD10B504464FF000006C
:103000004FF01201FFF7B2FA07EE900AB8EE677AB6
:103010009FED0B0AC7EE000A10EE900A15F0C0F8FB
:1030200005A3D3E9002315F059FA15F0D5F820606F
:103030004FF0010010BD00BF6666666666660A4016
:1030400000F07F45AFF3008010B504464FF000005C
:103050004FF01001FFF78AFA07EE900AB8EE677A90
:103060009FED1B0AC7EE000A10EE900A15F098F8C3
:1030700011A3D3E9002315F031FA15F0ADF815F0DE
:103080008FF80FA3D3E9002315F0E2F80EA3D3E9DC
:10309000002315F0D9FA4FF000024FF00003C4F2FC
:1030A000390315F0D7F815F097F820604FF00100BC
:1030B00010BD00BFAFF300806666666666660A40B4
:1030C00052B81E85EB51E83F7B14AE47E17A643F6E
:1030D00000F07F45AFF3008030B472B64CF6703329
:1030E000C0F603031A684EF63470CEF20000026098
:1030F0004CF67C31C0F603010A684EF68853CEF2D6
:1031000000031A604CF67830C0F60300016842F202
:103110000802CEF2040211604CF68033C0F60303BD
:10312000186842F20C01CEF20401086043F6000375
:10313000C4F202031A6842F48030186019460B6822
:1031400013F4003FFBD043F64000C4F202000268D3
:1031500042F08051016047F20003C4F20003186896
:1031600040F480421A604CF66831C0F603010868EA
:1031700043F60803C4F2020318604CF67432C0F63A
:103180000302116843F60040C4F2020001604CF6ED
:103190006433C0F603031A6843F60401C4F2020163
:1031A0000A6043F60000C4F20200036843F0807234
:1031B00002600146086810F0007FFBD043F6080368
:1031C000C4F202031A684FF0020161F301021A60AF
:1031D0001846036803F00C02082AFAD143F64401AA
:1031E000C4F20201086840F480430B6043F63000EB
:1031F000C4F20200026842F48011016047F2000349
:10320000C4F200031A6842F48071196047F20403A3
:10321000C4F200031A6842F400711960036843F4B1
:103220008022026043F61440C4F2020001684BF6AB
:103230000043C0F603031B684CF66C32C0F6030271
:1032400010686FEA000259400A4206D04BF600406F
:10325000C0F603004178CC2904D12A4B2A4999426F
:1032600021D344E043F60841C4F2020142F63B2078
:10327000C0F61900086046F67F60C4F65D4008603D
:10328000134043F61442C4F202021360136843F081
:103290000201116043F60C40C4F20200026812F40D
:1032A000803FFBD1D9E7194C194D281B20F00305AD
:1032B0004FF0000340F20002C1F200024EF6CC6172
:1032C000C0F6030105F10404C5F380005D589D506C
:1032D00003F10403A3420CD109E05858985003F1BC
:1032E00004035858985003F10403A342F5D130BCAD
:1032F00070470028F1D05858985003F10403A342B6
:10330000EBD1F4E7582B0408CCEE0308D0EE030809
:103310005B2B040843F63003C4F202031A6842F43C
:1033200000101860196841F480021A60704700BFED
:103330002DE9F0011546002A66D040F64C13C2F282
:10334000000353E8002F02F1010243E80024012C9E
:10335000F7D04CF68C32C0F60302146846F20846E9
:10336000C4F2020634604CF68837C0F603073A68A8
:1033700046F22843C4F202031A604FF6FF7846F281
:10338000304CC4F2020C46F23447C4F2020746F253
:103390002C46C4F202061C46454534BF2B46434624
:1033A000CCF8001038603360226842F001022260DD
:1033B000ED1A4FEA8303C918C018226812F0010FF2
:1033C000FBD1002DE8D140F64C13C2F2000353E8C4
:1033D000002FA2F1010243E80024012CF7D053E8AA
:1033E000002FB2F1004F0DD14FF0000243E800244E
:1033F000012CF4D04EF60450CEF20000016841F0EA
:1034000080510160BFF32F8FBDE8F001704700BF0E
:1034100070B41646002A37D046F21045C4F20205B1
:103420002C6814F0010FFBD14CF68432C0F6030275
:10343000146846F20842C4F20202146046F21842CE
:10344000C4F20202116046F21C41C4F2020108609B
:1034500046F21440C4F2020006604CF69032C0F608
:103460000302116846F21040C4F2020001600268D3
:1034700042F0010101603BB146F21040C4F202008B
:10348000036813F0010FFBD170BC704743F6104383
:10349000C4F20203186800280DDA43F60441C4F2AE
:1034A000020140F22312C4F267520A6048F6AB13DD
:1034B000CCF6EF530B6043F61040C4F202000168F3
:1034C00001F00042002A14BF02200020704700BF14
:1034D00043F61043C4F202031868002807DB43F6E2
:1034E0001041C4F202010A6842F000430B607047C9
:1034F00000F17840B0F5801F2CBF002001207047FC
:103500002DE9F04F83B006460D46FFF7F1FF002886
:1035100056D02846FFF7ECFF002854D0AE4255D8CD
:10352000FDF7E2F90190FFF7B1FF0446002841D111
:1035300006F178434FEA93304CF69432C0F603021A
:1035400012F8008041F28830FEF766FF4FF0020962
:1035500043F6104BC4F2020B43F60C47C4F20207C9
:103560004CF6D83AC0F6030AFEF74EFF494668F318
:10357000C60169F3092141F48033CBF80030386883
:1035800010F4803FFBD15AF82820B61808F1010842
:103590005FFA88F8B542E7D24FF06400FEF73CFFCF
:1035A0004CF60C41C0F60301086843F61043C4F220
:1035B00002031860FFF78CFF0198FDF79FF907E001
:1035C0004FF0020404E04FF0020401E04FF0020467
:1035D000204603B0BDE8F08F2DE9F04106460C46C9
:1035E00015460846FFF784FF002861D005F1FF303B
:1035F0002018FFF77DFF00285DD040F64C13C2F283
:10360000000353E8002F02F1010243E800210129E1
:10361000F7D0FFF73BFF074630BB4CF6D431C0F67E
:1036200003010A6843F61040C4F2020002608DB143
:1036300006F1FF3843F60C46C4F20206336813F471
:10364000803FFBD118F8011F04F8011BFEF7DCFED8
:10365000013DF3D14CF60844C0F60304226843F65A
:103660001040C4F202000260FFF732FF40F64C1334
:10367000C2F2000353E8002FA2F1010243E8002444
:10368000012CF7D053E8002FB2F1004F0DD14FF0CD
:10369000000243E80024012CF4D04EF60450CEF290
:1036A0000000016841F080510160BFF32F8F04E0FA
:1036B0004FF0020701E04FF002073846BDE8F08105
:1036C00040F20433C2F2000318684CF62042C0F600
:1036D0000302116801604FF0000303604CF62442BE
:1036E000C0F60302116841604CF61043C0F60303B4
:1036F0001A68C2614FF00D0101624CF62843C0F612
:1037000003031A680260704740F2FC23C2F2000310
:103710001868704770B48568C668446806FB054041
:103720004118196040F2FC20C2F20000006881429A
:103730000CD2521890420CD340F20030C2F200007A
:103740000268891819604FF0010004E04FF0000092
:1037500001E04FF0000070BC704700BF2DE9F04160
:103760000546FEF751FE4FF01E044FF0000840F2F0
:103770000436C2F200064FF00107052D26D8DFE817
:1037800005F0030A0F14191E3268936983F00200D2
:10379000C0F340011BE03068416901F0010116E00F
:1037A00032685369C3F3400111E030684169C1F3E5
:1037B000C0110CE032685369C3F3801107E033682D
:1037C000986980F0010101F0010100E0414689B9EA
:1037D00033685A6912F4807F10D1586910F4806FF1
:1037E00010D1384606F0FCFB013CC6D14FF000007A
:1037F000BDE8F0814FF00100BDE8F0814FF000001E
:10380000BDE8F0814FF00000BDE8F0812DE9F04106
:1038100084B014461D46072900F2AD80072A00F245
:10382000AD8001EB81024CF62C43C0F6030303EBA1
:103830008202137C002B40F0A48004EB84024CF63F
:103840002C43C0F6030303EB8202137C012B40F0F0
:103850009B804CF62C43C0F6030301EB810653F822
:10386000262004EB840653F826309A4240F08F80DD
:1038700040F20837C2F200073870022A15D0032A36
:1038800025D0012A34D143F64000C4F20200066874
:1038900046F40012026040F20433C2F2000345F223
:1038A0000047C4F200071F6022E043F64000C4F264
:1038B0000200066846F48002026040F20433C2F25D
:1038C000000345F60007C4F200071F6010E043F64E
:1038D0004000C4F20200066846F40002026040F2B2
:1038E0000433C2F2000345F60047C4F200071F602C
:1038F0004CF62C48C0F6030801EB810108EB81026D
:10390000107991684FF0000700974FF0010601967B
:10391000D36802934FF003023B46FDF787FD04EBAB
:10392000840408EB84042079A16800970196E2687A
:1039300002924FF003023346FDF778FDFFF7C0FE19
:1039400045B340F20030C2F200000A99016040F233
:10395000FC22C2F200020B9B136040F20C30C2F258
:1039600000004CF61441C0F603012A463B4608F01D
:1039700095F8304610E04FF000000DE04FF00000E9
:103980000AE04FF0000007E04FF0000004E04FF0C5
:10399000000001E04FF0010004B0BDE8F08100BF7D
:1039A00038B5044640F20433C2F200031D68A8692A
:1039B00010F0020F63D0FFF783FEA96911F0020F28
:1039C0005DD03BE040F20435C2F200052B684FF0B9
:1039D000A0021A614FF00200FFF7C0FE286881695B
:1039E00011F0010F08D0456915F4806F00F038829E
:1039F000036843F4007202604FF0050004F0A0FB7E
:103A00004FF0000516E040F20430C2F200000168F9
:103A10004FEA14230B614FF00300FFF79FFE38B10C
:103A200040F20432C2F200021068E4B2046101E024
:103A30004FF00005281C18BF012038BD4FF00000D2
:103A400038BD4FF0000038BD4FF0000038BD4FF0DA
:103A5000000038BD4FF0000038BD4FF0000038BD09
:103A60004FF0000038BD4FF0000038BD4FF00000AF
:103A700038BD4FF0000038BD4FF0000038BD40F2B7
:103A80000432C2F2000213684FF000005861196856
:103A900060F3492119601A6842F4807018604FF091
:103AA0000100FFF75BFE0028CBD040F20435C2F2E4
:103AB00000052B684FF0A00119614FF00200FFF7DD
:103AC0004DFE2868826912F0010F08D0436913F493
:103AD000806F00F0C881016841F4007202604FF00D
:103AE000050004F02DFB40F20430C2F20000036830
:103AF0004FF0000159611A6861F349221A60186891
:103B000040F4807119604FF00100FFF727FE002894
:103B10009AD040F20435C2F200052B684FF0A002A3
:103B20001A614FF00200FFF719FE2868816911F051
:103B3000010F08D0436913F4806F00F09781026889
:103B400042F4007101604FF0050004F0F9FA40F210
:103B50000430C2F2000003684FF0000159611A6896
:103B600061F349221A60186840F4807119604FF0BF
:103B70000100FFF7F3FD00283FF469AF40F2043580
:103B8000C2F200052B684FF0A0021A614FF002004C
:103B9000FFF7E4FD2868816911F0010F08D043693F
:103BA00013F4806F00F06581026842F400710160D7
:103BB0004FF0050004F0C4FA40F20430C2F20000F5
:103BC00003684FF0000159611A6861F349221A60D5
:103BD000186840F4807119604FF00100FFF7BEFDD6
:103BE00000283FF437AF40F20435C2F200052B68DD
:103BF0004FF0A0021A614FF00200FFF7AFFD2868F6
:103C0000816911F0010F08D0436913F4806F00F04F
:103C10003381026842F4007101604FF0050004F046
:103C20008FFA40F20430C2F2000003684FF0000146
:103C300059611A6861F349221A60186840F480716A
:103C400019604FF00100FFF789FD00283FF405AF30
:103C500040F20435C2F200052B684FF0A0021A6151
:103C60004FF00200FFF77AFD2868816911F0010F1B
:103C700008D0436913F4806F00F00181026842F4B8
:103C8000007101604FF0050004F05AFA40F2043070
:103C9000C2F2000003684FF0000159611A6861F335
:103CA00049221A60186840F4807119604FF00100D1
:103CB000FFF754FD00283FF4D3AE40F20435C2F2C2
:103CC00000052B684FF0A0021A614FF00200FFF7C9
:103CD00045FD2868816911F0010F08D0436913F48C
:103CE000806F00F0CF80026842F4007101604FF0F5
:103CF000050004F025FA40F20430C2F20000036827
:103D00004FF0000159611A6861F349221A6018687E
:103D100040F4807119604FF00100FFF71FFD00288B
:103D20003FF4A1AE40F20435C2F200052B684FF01B
:103D3000A0021A614FF00200FFF710FD28688169A8
:103D400011F0010F08D0436913F4806F00F09D80DB
:103D5000026842F4007101604FF0050004F0F0F9D0
:103D600040F20430C2F2000003684FF000015961D4
:103D70001A6861F349221A60186840F4807119606A
:103D80004FF00100FFF7EAFC00283FF46FAE40F26D
:103D90000435C2F200052B684FF0A0021A614FF003
:103DA0000200FFF7DBFC2868816911F0010F07D0E2
:103DB000436913F4806F6BD0026842F400710160B4
:103DC0004FF0050004F0BCF940F20430C2F20000EC
:103DD00003684FF0000159611A6861F349221A60C3
:103DE000186840F4807119604FF00100FFF7B6FCCD
:103DF00000283FF43EAE40F20435C2F200052B68C5
:103E00004FF0A0021A614FF00200FFF7A7FC2868EC
:103E1000816911F0010F07D0436913F4806F3AD024
:103E2000026842F4007101604FF0050004F088F967
:103E300040F20430C2F2000003684FF00001596103
:103E40001A6861F349221A60186840F48071196099
:103E50004FF00100FFF782FC00287FF4B3AD0BE6C2
:103E60004FF0010519E04FF00A0516E04FF0090583
:103E700013E04FF0080510E04FF007050DE04FF09C
:103E800006050AE04FF0050507E04FF0040504E0E1
:103E90004FF0030501E04FF0020540F20830C2F296
:103EA0000000017801F1FF33DAB2012A3FF6B8AD24
:103EB000A9E500BFF8B50D461446002A6FD080B2C0
:103EC000FFF76EFD002865D04FF00300FFF746FCBA
:103ED00000285FD040F20433C2F200031868026881
:103EE00042F4807101604FF00100FFF737FC0028B9
:103EF00050D040F20433C2F20003186814F1FF31CD
:103F000018BF0121026861F38A2202604FF0A10309
:103F100003614FF00200FFF721FC00283AD040F285
:103F20000430C2F2000001688A6912F0010F31D03A
:103F30004B6913F4806F2DD14FF0040640F2043723
:103F4000C2F200073046FFF709FC18B304F1FF3452
:103F5000012C27D1FCF7C8FC39680A696FEA020313
:103F600005F8013B0A686FF38A220A60FCF7C6FC79
:103F7000E8E72B681B6902E04FF004060E4D30465F
:103F8000FFF7ECFB0028F4D10B4B1868016841F4F3
:103F900000720260D4F1010038BF0020F8BD4FF07C
:103FA0000100F8BD386801696FEA010205F8012BCC
:103FB000002CC7D1E0E700BF0403002030B583B078
:103FC00015461C461A4601ABFFF7A4FB48B1019801
:103FD00029462246FFF76EFF00280CBF182000205C
:103FE00001E04FF01F0003B030BD00BF2DE9F84FD6
:103FF00093460D4600295DD004464FF0030840F279
:104000000439C2F2000901E0002E40D01FFA8BF003
:10401000FFF7C6FC00283DD00BF0070715F0010F95
:104020004CD14046FFF79AFB002836D0072F1AD80C
:10403000DDB13CB1D9F8000014F8011B6FEA0103AF
:10404000036104E0D9F800604FF0FF02326107F12C
:104050000107BA4605F1FF3635464046FFF77EFBBD
:10406000002845D119E02E4600E02E46D9F8000080
:10407000026842F4007101600BF1080B2BF0070B92
:104080004FF00500FFF76AFB0028BDD107E04FF0B5
:10409000010004E04FF0000001E04FF0000040F2AA
:1040A0000433C2F2000319680A6842F400730B601B
:1040B000BDE8F88F4FF00100BDE8F88F4046FFF7EC
:1040C0004DFB0028E9D0072FCDD82CB9D9F8003006
:1040D0004FF0FF021A6106E0D9F8000014F8011B46
:1040E0006FEA0103036107F1010705F1FF3598E766
:1040F000072FB8D82CB9D9F800504FF0FF022A6129
:1041000006E0D9F8000014F8011B6FEA010303610F
:1041100007F1010706F1FF3583E700BF30B583B033
:1041200015461C461A4601ABFFF7F4FA48B128467B
:104130002146019AFFF75AFF00280CBF18200020E3
:1041400001E04FF01F0003B030BD00BF08B543F2DF
:104150005C50C2F2000043F65C02C2F20002131A85
:104160004FF0FF314FEAA302FCF778FB43F65C0007
:10417000C2F2000044F25C01C2F200010A1A4FEAE6
:10418000A2024FF0FF31A2F12002FCF767FB02F020
:1041900087FB40F21C30C2F2000044F20001C4F27E
:1041A00002014FF480524FF0030313F005FFFCF7B8
:1041B00023FF4FF0000008BDBFF36F8F704700BFB3
:1041C0004CF64C53C0F60303185C00EB40014CF670
:1041D0007862C0F6030252F821305B68704700BF76
:1041E00038B54CF64C53C0F603031B5C03EBC30419
:1041F00040F23432C2F2000202EB840282F8211053
:1042000014693CB140F23435C2F200051346D2695C
:104210009B69A04738BD00BFF8B506460F464CF66F
:104220004C53C0F603031D5C05EBC50040F234346B
:10423000C2F2000404EB8004D4F810C0BCF1000FFB
:1042400007D0E2698A4204D030464FF00001A369EA
:10425000E047E76163695BB105EBC50040F23432CA
:10426000C2F2000202EB800230463946926998475A
:1042700094F8201079B127696FB105EBC50540F2BC
:104280003433C2F2000303EB8505304694F8211065
:10429000E269AB69B847F8BD4CF64C53C0F603036E
:1042A000185C00EB40014CF67862C0F6030252F84D
:1042B0002130D86840F08001D9607047F8B50446D5
:1042C00000EB40024CF67863C0F6030353F822601B
:1042D00035686FEA0500306005F0010215F0020F45
:1042E0001CBF42F00202D2B215F0040F18BF42F018
:1042F000080215F0080F18BF42F0040215F4807F81
:1043000005D0316911F4804F18BF42F0100215F04A
:10431000200F00D1E2B104EBC40740F23433C2F203
:10432000000303EB870087688FB1716804EBC4005A
:1043300040F23433C2F2000303EB80034CF64460D6
:10434000C0F60300005DC9B29B69B84700E073681E
:10435000F26812F0800F1CD015F0800F19D0F168B0
:104360006FF3C711F16004EBC40040F23433C2F2C2
:10437000000353F8203063B140F23432C2F200023D
:1043800002EB80024CF64460C0F60300005D9169C8
:10439000984715F0400F17D004EBC40140F23433B6
:1043A000C2F2000303EB810253686BB1084640F28E
:1043B0003431C2F2000101EB80024CF64460C0F6D9
:1043C0000300005D91699847F8BD00BF684620F082
:1043D00007018D4601B54FF00600FFF76FFFBDE8FE
:1043E00001408546704700BF684620F007018D46B2
:1043F00001B54FF00500FFF761FFBDE801408546BC
:10440000704700BF684620F007018D4601B54FF0A8
:104410000400FFF753FFBDE801408546704700BF29
:10442000684620F007018D4601B54FF00300FFF705
:1044300045FFBDE801408546704700BF684620F053
:1044400007018D4601B54FF00200FFF737FFBDE8C9
:1044500001408546704700BF684620F007018D4641
:1044600001B54FF00100FFF729FFBDE80140854687
:10447000704700BF10B582B08DF807104CF64C5352
:10448000C0F60303185C00EB40024CF67861C0F6FE
:10449000030151F82240236813F0800FFBD002A9DA
:1044A00011F8012D626000EBC00040F23434C2F21A
:1044B000000404EB8004608C4FF0010205F0A8FDBD
:1044C000608404F1200402B010BD00BF70B582B05A
:1044D0008DF807104CF64C53C0F60303185C00EB44
:1044E00040014CF67862C0F6030252F8214025687C
:1044F00015F0800F1DBF9DF807506560012600264E
:1045000000EBC00340F23430C2F2000000EB830540
:10451000688C0DF107014FF0010205F079FD688408
:1045200005F12005E16841F08002E260304602B00A
:1045300070BD00BF2DE9F84F81468B4690461E4660
:104540009DF828A04CF64C53C0F603031D5C05EB08
:1045500045024CF67860C0F6030050F822409DF802
:104560002C70012F14BF00270127082E06D0072E1C
:1045700002D1B8F1000F01D1FCF760F90AF1FF3167
:10458000CBB2012B01D9FCF759F94CF62862C0F6E1
:10459000030252F82500B0FBFBF1A1604FF00002CE
:1045A00067F38612BAF1010F04D0002F0CBF02236B
:1045B000002301E04FF0000363F30D3267F38E3206
:1045C00022614FF06C00B8F1020F14BF00230123E9
:1045D00063F3492018F1000818BF4FF0010868F391
:1045E0008A20082E18BF4FF0000868F30C3040F402
:1045F0000051E1604846FFF7E3FDBDE8F88F00BFDA
:10460000F0B585B00D461E464CF64C53C0F603037C
:10461000195C01EB41044CF67867C0F6030757F8C4
:1046200024704CF65863C0F60303185C00EB40019D
:104630004CF65054C0F6030404EBC1040AB1FCF775
:10464000FDF875B9207B21699DF82C2000924FF070
:1046500001030193626902924FF003023346FCF7B3
:10466000E5FE207861689DF8283000934FF0010244
:104670000192A36802934FF003023346FCF7D6FE83
:104680004CF64C60C0F603000168012D14BF0025F4
:10469000012565F3C301796105B0F0BD2DE9F8434B
:1046A00005464CF64C53C0F60303185C00EBC00201
:1046B00040F23434C2F2000404EB82044CF6786118
:1046C000C0F6030100EB40064FEA860301EB030846
:1046D00051F80390FCF708F9064694F82000B8B1A9
:1046E0004FF00007C9F80C703846394698F9042095
:1046F000FCF76CF928463946FFF772FDE3681BB1F9
:104700002846E169A26998474FF0000284F820200A
:104710003046FCF7F3F8BDE8F88300BF2DE9F04F11
:1047200085B005468B46924699464CF64C53C0F6EA
:1047300003031E5C40F23438C2F2000806EBC607E1
:104740004FEA870708EB070406EB46004CF6786152
:10475000C0F6030101EB8006FCF7C6F8039043F6B0
:104760004003C4F2020318684CF65061C0F603011E
:104770000A6820EA020E4CF65C62C0F6030210687A
:104780004EEA0000186043F64403C4F202031868BE
:10479000496820EA01005268104318604CF66461D1
:1047A000C0F6030105EB8503C818C95C427883781D
:1047B00090F803C0CDF800C0007901902846FFF7BB
:1047C0001FFF9DF8382000929DF83C10019128466B
:1047D000594652464B46FFF7ADFE109B48F807304E
:1047E0001298A060119A62601399E160149BA36112
:1047F000B0684FF00F0196F90420FCF7E7F84FF08E
:10480000010084F820000398FCF778F805B0BDE8B3
:10481000F08F00BF4CF64C53C0F60303185C00EB5E
:10482000C00340F23430C2F2000000EB8303196190
:104830005A6170474CF65863C0F60303185C00EBEE
:1048400040014CF69852C0F6030202EB011070478B
:10485000FA2884BF0530C0B2032812D84CF64C5356
:10486000C0F60303185C00EBC00140F23432C2F220
:10487000000202EB81034FF6FF7058844FF00100F5
:1048800070474FF000007047FA2884BF0530C0B26F
:1048900003280ED84CF64C53C0F60303185C00EB0B
:1048A000C00140F23432C2F2000202EB8103588CA4
:1048B00070474FF000007047082806D9102807D924
:1048C00020288CBF4020202070474FF00800704700
:1048D0004FF01000704700BF022809D0032804D011
:1048E000012814BF0020012070474FF003007047DB
:1048F0004FF00200704700BF40F60013C5F20003FE
:10490000186840F60802C5F200021168C1F34103BD
:10491000022B12BF6FF30200032363F3020040F483
:1049200000406FF3995040F60012C5F2000210608B
:1049300040F60401C5F200010B6843F48070086082
:10494000704700BF4CF66873C0F603031A6840F660
:104950001030C5F200000260704700BF10B440F68E
:104960005073C2F200031A5CE0B14FF0000340F64E
:104970000841C2F200014FF04C0404FB0212D1685E
:1049800021F0030202F1040262F312034FF001016D
:1049900061F3DC434CF6E862C0F6030202EB401020
:1049A00081690B6010BC704770B440F22003C5F2FF
:1049B00000031868C0F34342022A01D0062A29D115
:1049C00000F00F014CF66C75C0F6030555F8216038
:1049D000C0F30A1505F1030398081BD041F200014A
:1049E000C5F2000100F1FF3404F001040A68334607
:1049F00072604FF0010282420ED10AE00C6803F1AE
:104A0000040343F8044F0C685C6002F10202824226
:104A1000F4D1356070BC7047002CEFD00C6803F106
:104A200004035C6002F101028242E7D1F1E700BFBA
:104A300070B44CF6CC63C0F6030353F820603268C0
:104A4000002A3CD04CF6E861C0F6030101EB4011AE
:104A500002F103024FEA9202CB691B689A420CD919
:104A600040F63402C5F2000211684FF0010303FA68
:104A700000F008431060184623E006F10403C2B1B9
:104A800002F1FF3000F00105086953F8044B04609F
:104A9000501E18D10DE00C691A4652F8045B2560CF
:104AA00000F1FF300C695B68236002F104030138F8
:104AB000F1D14FF0000131604FF0010001E04FF003
:104AC000000070BC7047002DE5D00A6953F8044B14
:104AD00014600138DFD1ECE708B54FF0010303FAA9
:104AE00000F040F23242C2F200021388184210D0A5
:104AF00023EA000340F23240C2F200000380CA6B96
:104B000052B1086A4FF0000104F0C0FC4FF0000001
:104B100008BD4FF0000008BD4FF0010008BD00BF08
:104B200070B540F21403C5F200031C684CF6E06057
:104B3000C0F6030001680C4200F0BB8140F64C72E5
:104B4000C2F200021378012B40F2B38140F2180048
:104B5000C5F2000001684CF68472C0F603021368C7
:104B6000194200F0A68140F61800C5F20000016865
:104B700011F0010F56D040F60815C5F200052A685D
:104B800040F60830C5F2000003682A60036040F672
:104B90005071C2F20001087840F60841C2F20001EB
:104BA0004FF04C0505FB001503F00100E96A0143D5
:104BB000E962C3F3C000296B0143296303F00803D2
:104BC000D8B258BBD2B212F0010F0ED01DE0EA6A83
:104BD00022B105F1100000F087FF2BE02B6B002BBA
:104BE000F7D1686B0028F4D124E012F0900FEED0DA
:104BF00040F63403C5F20003186820F00101196083
:104C00004FF00000FFF714FFE1E76E6B4FF000007C
:104C10002946FFF761FF30436863D8E74FF0000192
:104C2000E963CFE740F61802C5F20002136813F4F7
:104C3000803FA0D140F61801C5F200010A6802F0D9
:104C4000020398B2002856D040F62815C5F2000598
:104C50002A6840F62830C5F2000003682A60036025
:104C600040F65071C2F20001487840F60841C2F2A5
:104C700000014FF04C0505FB001503F00100E96A47
:104C80000143E962C3F3C000296B0143296303F0C8
:104C90000803D8B258BBD2B212F0010F0ED01DE0FB
:104CA000EA6A22B105F1100000F01EFF2FE02B6B25
:104CB000002BF7D1686B0028F4D128E012F0900F98
:104CC000EED040F63403C5F20003186820F002016C
:104CD00019604FF00100FFF7ABFEE1E76E6B4FF09C
:104CE00001002946FFF7F8FE30436863D8E74FF02C
:104CF0000001E963CFE740F61801C5F200010A6838
:104D00004FEA124303F0020081B200299CD140F621
:104D10001801C5F200010A6802F0040398B20028E5
:104D200056D040F64815C5F200052A6840F64830CE
:104D3000C5F2000003682A60036040F65071C2F2B9
:104D40000001887840F60841C2F200014FF04C059E
:104D500005FB001503F00100E96A0143E962C3F3B2
:104D6000C000296B0143296303F00803D8B258BB84
:104D7000D2B212F0010F0ED01DE0EA6A22B105F1A5
:104D8000100000F0B1FE2FE02B6B002BF7D1686B09
:104D90000028F4D128E012F0900FEED040F6340352
:104DA000C5F20003186820F0040119604FF00200FA
:104DB000FFF73EFEE1E76E6B4FF002002946FFF77A
:104DC0008BFE30436863D8E74FF00001E963CFE71B
:104DD00040F61801C5F200010A684FEA124303F0D9
:104DE000040081B200299CD140F61801C5F20001EF
:104DF0000A6802F0080398B258B940F61801C5F2E3
:104E000000010A684FEA124303F0080081B200294A
:104E10004FD040F66815C5F200052A6840F66830A4
:104E2000C5F2000003682A60036040F65071C2F2C8
:104E30000001C87840F60841C2F200014FF04C056D
:104E400005FB001503F00100E96A0143E962C3F3C1
:104E5000C000296B0143296303F00803D8B210B1E5
:104E60004FF00001E963D2B212F0010F08D06E6B6F
:104E70004FF003002946FFF72FFE304368630EE032
:104E800012F0900F0BD040F63403C5F200031868FF
:104E900020F0080119604FF00300FFF7C9FDEA6A2E
:104EA0001AB92B6B0BB9686B18B105F1100000F043
:104EB0001BFE14F0100F01D0FFF776FD14F4805F95
:104EC0000DD040F61D71C2F200014FF001020A70D0
:104ED00040F61473C2F20003186802F09BFF14F44A
:104EE000005F01D0FFF708FD14F4006F14D040F606
:104EF0006860C2F200004FF00101017040F640739B
:104F0000C2F200034FF000021A7040F61470C2F2B1
:104F10000000006802F07EFF002C14DA40F66861A1
:104F2000C2F200014FF000030B7040F64070C2F275
:104F300000004FF00102027040F61471C2F200014D
:104F4000086802F067FF40F21403C5F200031C601A
:104F500070BD00BF684620F007018D4689B500AFDF
:104F6000FFF7DEFDBD46BDE889408546704700BFBE
:104F70002DE9F04140F60846C2F200064FF04C031E
:104F800003FB0066304650F8205F4CF6E868C0F638
:104F900003084FEA451708EB07044FF000014FF0F4
:104FA0001C0215F009F835624FF00100B06258F8A4
:104FB00007204FF00003136061690B60A0684FF099
:104FC000FF02026061680B60A0690360E1680A602B
:104FD0004CF66C72C0F6030252F8250003604CF6E2
:104FE000CC61C0F6030151F825201360BDE8F081C3
:104FF00000B583B04FF00003019340F21001C5F2F9
:1050000000010A68B0F1FF3F08BF102060F3891269
:1050100042F0200040F21003C5F200031860194668
:1050200040F63F52C0F20302019800F101000190E6
:105030000B6813F0200F02D001989042F4D94FF082
:10504000030004F0CDFF03B000BD00BF2DE9F8431D
:105050004FF04C0303FB00F040F60841C2F20001A0
:105060004418256A4FF0010606FA05F64CF6E86288
:10507000C0F6030202EB45174058002867D0A3682A
:10508000FBB1D7F80080D8F8001011F4004F18D108
:10509000D8F80020914663F30A09007AFFF71CFC58
:1050A00060F3934949F4004965F3995949F08050F8
:1050B000C0F3404363F39A60C8F800002846FFF746
:1050C00097FFE168F1B17A68106810F4004F19D1C8
:1050D0002846FFF743FCD7F80480D8F80070E3684F
:1050E00063F30A072168087AFFF7F6FB60F393473A
:1050F00047F4004242F01047C7F3404060F39A671C
:10510000C8F800704CF66C73C0F6030353F8251012
:105110004FF000020A60A06858B140F61C03C5F2C7
:105120000003196846EA010290B2196860F30F01A2
:105130001960E3685BB140F61C00C5F2000002682C
:1051400046EA1246B6B2016866F31F410160BDE847
:10515000F88300BF70B582B04FF00002019240F2B8
:105160001003C5F20003196841F0010018600192B4
:105170001A6812F0010F19D0019940F63F53C0F29E
:105180000303994212D840F21000C5F2000040F625
:105190003F52C0F20302019901F10101019103683C
:1051A00013F0010F02D001999142F4D94FF003009E
:1051B00004F016FF4FF00000019040F21002C5F21B
:1051C00000021368002B1DDB019940F63F50C0F22E
:1051D0000300814216D84FF0030640F21005C5F2D5
:1051E000000540F63F54C0F20304304604F0F8FED8
:1051F000019A02F1010201922B68002B02DB019956
:10520000A142F2D902B070BD00B583B04FF00003E7
:10521000019340F21000C5F20000026842F0100154
:10522000016040F63F52C0F20302019B03F101030B
:105230000193016811F0100F02D0019B9342F4D941
:105240004FF0030004F0CCFE03B000BD50B14CF6AB
:105250007C71C0F603010A6840F21803C5F200032E
:105260001A6070474CF68073C0F603031A6840F268
:105270001800C5F200000260704700BF38B54FF05B
:10528000000440F60063C5F200031C6040F6000213
:10529000C5F20002106840F0030164F3820164F378
:1052A0000A11116040F22405C5F200052B684FF089
:1052B000400262F30F032B60204662F31F40214639
:1052C00062F31F4162F30F0140F22805C5F20005A9
:1052D00029604FF0800363F30F0040F20412C5F21F
:1052E000000210604FF0C00161F30F0040F208159A
:1052F000C5F2000528604FF4807363F30F0040F29D
:105300000C12C5F2000210604FF0FF30FFF770FE84
:10531000FFF77AFF40F61000C5F20000046040F687
:105320001401C5F200010C604FF0FF3540F6180380
:10533000C5F200031D6040F61C02C5F200021460B5
:105340002046FFF715FE4FF00100FFF711FE4FF06A
:105350000200FFF70DFE4FF00300FFF709FE4FF0CC
:105360000400FFF705FE4FF00500FFF701FE4FF0C8
:105370000600FFF7FDFD4FF00700FFF7F9FD40F2D3
:105380001800C5F20000046040F21401C5F20001EB
:105390000D604FF00100FFF759FF38BD40F2324376
:1053A000C2F2000319884FF0010202FA00F008402F
:1053B00000280CBF02200320704700BF40F60013F6
:1053C000C5F200031B68C3F3076202F08000C1B29C
:1053D00009B143F0804343F4001040F60012C5F2D7
:1053E00000021060704700BF2DE9F84305461646DD
:1053F0004CF6E868C0F6030808EB40184CF6CC639E
:10540000C0F6030353F820704FF0010909FA00F9C0
:105410000C46A9B9386840B940F23243C2F20003E1
:10542000188819EA000F5AD10AE040F23241C2F25C
:1054300000010A8819EA020F02D02846FFF7D8FDBA
:1054400006F1030107F1040388081CD000F1FF32C4
:1054500002F0010CA4F1040151F8042F43F8042BCD
:1054600001383ED10FE001F1040249681C4644F8BE
:10547000041B00F1FF3002F1040152685A6004F18C
:1054800004030138EFD13E6040F23243C2F2000320
:10549000198849EA0109A3F8009065B940F610108F
:1054A000C5F2000002684FF0010161F3D44266F3D7
:1054B0000602026009E0D8F8140002684FF0010308
:1054C00063F3DC4266F312020260D8F80030186819
:1054D00040F004421A6016B12846FFF7A9FABDE869
:1054E000F883BCF1000FBED051F8042F43F8042B11
:1054F0000138B8D1C7E700BF70B504464CF66C73ED
:10550000C0F6030353F82060334653F8045BAA4205
:1055100038BF1546084619462A4614F029FD4FF0B3
:10552000000030602046FFF719FA4CF6E861C0F63B
:10553000030101EB441463681A6842F004401860E8
:10554000284670BDF8B5054640F60843C2F2000390
:105550001868002871D040F60841C2F20001CA6CF8
:10556000002A71D040F60844C2F20004D4F89860D2
:10557000002E6DD040F60847C2F20007D7F8E4309D
:10558000002B69D040F60840C2F20000D0F830117C
:10559000002965D040F60842C2F20002D2F87C41F0
:1055A000002C61D040F60846C2F20006D6F8C87159
:1055B000002F5DD040F60843C2F20003D3F8140276
:1055C000002859D040F60841C2F20001D1F860220B
:1055D000002A55D0464E4FF00807FBF72FF92C7ADA
:1055E000002C53D040F23042C2F200021088014633
:1055F00010F0020F55D04FF0010404F1010441FAFC
:1056000004F212F0010FF8D14FF0010101FA04F198
:10561000084340F23043C2F20003188044B968895D
:10562000FFF74AF9B060A889FFF746F9F06042E059
:105630006A89B260A989F1603DE040F60846C2F28D
:1056400000064FF000071EE02A4E4FF001071AE057
:10565000294E4FF0020716E0284E4FF0030712E0E4
:10566000274E4FF004070EE0264E4FF005070AE0E4
:10567000254E4FF0060706E0244E4FF0070702E0E4
:105680001B4E4FF00807072FA9D9A6E740F2304379
:10569000C2F20003188840F0010119804FF00004A5
:1056A000BDE740F0020440F23043C2F200031C8028
:1056B0004FF00104BCE740F65070C2F200000755FD
:1056C000374647F8205B38464FF000014FF01C0288
:1056D00014F072FC34626B68B36306F110004FF093
:1056E00006012A683B4600F0DFF92046F8BD00BFFE
:1056F000680E0020540C0020A00C0020EC0C0020B0
:10570000380D0020840D0020D00D00201C0E00203C
:10571000022907D140F60003C5F200031A6860F3BE
:105720000A121A60704700BF10B54FF0000440F62F
:105730003403C5F200031C6040F60400C5F200000B
:10574000026842F0010101602046FFF711FC4FF0B2
:105750000100FFF70DFC4FF00200FFF709FC4FF0CE
:105760000300FFF705FC4FF00400FFF701FC4FF0CA
:105770000500FFF7FDFB4FF00600FFF7F9FB4FF0C8
:105780000700FFF7F5FB4FF0FF30FFF731FC40F269
:105790003243C2F200031C8040F61800C5F200003C
:1057A0004FF0FF3202604CF68871C0F603010868C2
:1057B00040F61C03C5F2000318604CF6E462C0F624
:1057C0000302116840F61400C5F2000001604CF6B7
:1057D000DC63C0F603031A6840F61001C5F200014D
:1057E0000A6020464FF00201FFF792FFFFF7AAF888
:1057F0002046FFF72BFC4FF00100FFF727FC4FF08E
:105800000200FFF723FC4FF00300FFF71FFC4FF0EF
:105810000400FFF71BFC4FF00500FFF717FC4FF0EB
:105820000600FFF713FC4FF00700FFF70FFC10BD59
:1058300008B5FFF779FF08BD704700BFF0B585B028
:10584000054641F28830FCF7E7FD002D62D043F6B3
:105850003401C4F202010C6844F080060E604FF07F
:10586000000400944FF0030601964FF00A070297D8
:1058700020464FF00B0132462346FBF7D7FD00943C
:105880000196029720464FF00C0132462346FBF763
:10589000CDFD40F20C06C5F20006336843F040022D
:1058A0003260FFF757FC40F23800C5F200004FF4B9
:1058B0000411016044F6206004F092FBFCF7A4FDA3
:1058C000336843F0400064F3082064F349204FF04C
:1058D000050262F38D2064F35D7040F08041316019
:1058E00044F6206004F07CFBFCF78EFDFFF7C6FC5D
:1058F00040F20803C5F2000340F28110186044F63C
:105900005570C0F602004FF00F014FF04302FBF755
:105910005DF813E04FF000004FF00F014FF043022D
:10592000FBF754F84FF0000340F23802C5F20002D2
:10593000136040F21800C5F2000003602846FFF72C
:105940007BFF4FF06400FCF767FD05B0F0BD00BFC2
:105950002DE9F04182B04CF68C77C0F6030745F68E
:105960003126C0F6020640F28C15C2F200054FF057
:105970000408CDF8008038464FF0800132462B46AF
:1059800002F094FB40F26444C2F200042060CDF8BF
:10599000008038464FF08101324605EB080302F0E3
:1059A00085FB6060CDF8008038464FF082013246BA
:1059B00005F1080302F07AFBA060CDF800803846BC
:1059C0004FF08301324605F10C0302F06FFBE060FB
:1059D000CDF8008038464FF08401324605F11003BF
:1059E00002F064FB2061CDF8008038464FF085015D
:1059F000324605F1140302F059FB6061CDF80080D6
:105A000038464FF08601324605F1180302F04EFB8E
:105A1000A061CDF8008038464FF08701324605F18D
:105A20001C0302F043FBE06102B0BDE8F08100BF5F
:105A300080B505464FF0000640F23C49C2F200092D
:105A400040F28448C2F2000840F23847C2F2000730
:105A50001FE0FAF749FF2C68616829604FF00002E7
:105A60006260237B062B0ED1216849F82610092E8F
:105A70009CBF0136F6B2012E03D93A8802F1010229
:105A80003A8088F80060FAF739FF23680BB1A06804
:105A900098472B6803F1FF3010F1030FD9D902F0BA
:105AA00087F94FF00006F4E70260B3F1FF3F18BF3B
:105AB0008360FF290ED143F25853C2F200031A68E3
:105AC00022B192F829304FEA530101E04FF007016B
:105AD0000173704701F07F010173704710B14FF0FF
:105AE00000020260704700BF38B50446FAF7FCFEBA
:105AF000054640F28643C2F200031A8802F1010211
:105B00001A80002C35D06368EBB940F28840C2F2AD
:105B10000000028802F101020280207B40F28C1317
:105B2000C2F2000353F82010616043F82040247B48
:105B300040F26442C2F2000252F8240002F06AF914
:105B40004FF0010422E040F23440C2F2000002882B
:105B500002F101020280247B062C15D140F23A4169
:105B6000C2F200010B8803F101030B804FF0000427
:105B70000CE040F23640C2F20000018801F1010160
:105B800001804FF0000401E04FF000042846FAF7CE
:105B9000B5FE204638BD00BF10B5044640F2946003
:105BA000C2F200004FF000014FF0240214F004FA9A
:105BB000D4B140F2D440C2F200004FF000014FF0E7
:105BC000480214F0F9F940F26450C2F200004FF0BC
:105BD00000014FF0240214F0EFF940F25C53C2F2DE
:105BE00000034FF002021A7010BD00BF38B54CF62A
:105BF000F473C0F6030353F8205040F22051C2F270
:105C0000000151F820404DF23802C0F60302105C4A
:105C1000FBF7F4FC2840A04214BF0020012038BD4F
:105C20004DF23803C0F603031A5C40F26451C2F22D
:105C3000000151F822204CF6F473C0F6030353F828
:105C4000200002420CBF00200120704770B440F6D3
:105C50004C13C2F2000353E8002F02F1010243E8A3
:105C600000210129F7D04DF23802C0F60302155C7D
:105C700040F29461C2F2000151F825404CF6F476EE
:105C8000C0F6030656F8202024EA020041F8250059
:105C900053E8005FA5F1010543E80056012EF7D057
:105CA00053E8005FB5F1004F0DD14FF0000543E818
:105CB0000056012EF4D04EF60450CEF200000168DA
:105CC00041F080510160BFF32F8F14420CBF0020C0
:105CD000012070BC704700BF4DF24803C0F60303BB
:105CE000185C704708B54FF0000040F25851C2F2FE
:105CF0000001FAF7A7FD003018BF012008BD00BF62
:105D000010B50446FBF77AFC40F2AC13C2F2000374
:105D100053F82410484010BD10B504464FF0010060
:105D2000FFF73AFF4CF6BC73C0F6030353F8342078
:105D300040F26051C2F200010A6003EBC4046068E3
:105D400040F28C53C2F20003186010BD00B585B05C
:105D50004FF00000FFF7E0FF4FF00003009340F228
:105D60009052C2F2000201924FF0400002904DF2B8
:105D70002C00C0F603004FF0020145F62162C0F688
:105D8000020202F07FF840F29063C2F20003186052
:105D900005B000BD2DE9F001804600283CD04FF051
:105DA00000034FEA8302086850F823404D6855F815
:105DB000236086EA0407886850F8235084EA050CBB
:105DC0004CEA07076FEA070CC86850F8235026EA28
:105DD000050707EA0C0705EA0C0C66EA0C063540D5
:105DE00040F82350CD6855F82300384345F8230088
:105DF0000D6955F82300384345F823004D690DB16E
:105E000045F82370486885588868855048688450EC
:105E100003F101034345C4D1BDE8F001704700BF61
:105E20002DE9F84340F26058C2F2000840F288566B
:105E3000C2F2000640F28C44C2F200044FF00005AA
:105E400040F28C57C2F20007D8F8000000EB800047
:105E500002F076F93368002B40F00B822046294689
:105E60004FF0240214F0A8F803E24FF009004CF6BA
:105E7000DC71C0F60301FFF78DFF40F25C53C2F204
:105E80000003197859B101F1FF3040F25C52C2F2BF
:105E90000002107040F29463C2F200031D6040F2F1
:105EA0005851C2F200010868E8B940F25852C2F2F3
:105EB0000002156040F21C53C2F20003197849B980
:105EC00040F25851C2F20001086860B1284606F05D
:105ED000A7FC08E040F25850C2F20000026842F00D
:105EE00000630360ECE740F25C52C2F200021378F8
:105EF0005BB103F1FF3140F25C50C2F2000001706F
:105F000040F29462C2F20002556040F25853C2F26D
:105F10000003196841BB4CF69870C0F60300426854
:105F200040F2B043C2F2000359680A4040F25850B0
:105F3000C2F20000026040F21C52C2F2000213786A
:105F40004BB940F25853C2F20003196861B12846B8
:105F500006F066FC08E040F25851C2F20001086801
:105F600040F000620A60ECE740F25C50C2F20000D0
:105F700002785AB102F1FF3340F25C51C2F20001E3
:105F80000B7040F29460C2F20000856040F25852FB
:105F9000C2F200021368EBB940F25851C2F200019C
:105FA0000D6040F21C50C2F2000002784AB940F283
:105FB0005852C2F20002136863B1284606F030FC62
:105FC00008E040F25853C2F20003196841F0006043
:105FD0001860ECE740F25C51C2F20001087858B159
:105FE00000F1FF3340F25C52C2F20002137040F243
:105FF0009461C2F20001CD6040F25850C2F200003C
:106000000368EBB940F25852C2F20002156040F248
:106010001C51C2F20001087848B940F25850C2F24F
:106020000000036863B1284606F0FAFB08E040F27E
:106030005853C2F200031A6842F000611960ECE79D
:1060400040F25C52C2F20002117859B101F1FF3006
:1060500040F25C53C2F20003187040F29462C2F244
:106060000002156140F25851C2F20001086840BBBD
:106070004CF69873C0F603031A6940F2B041C2F2BD
:1060800000010869024040F25853C2F200031A604E
:1060900040F21C52C2F20002117849B940F2585144
:1060A000C2F20001086860B1284606F0B9FB08E0BA
:1060B00040F25850C2F20000036843F000620260F0
:1060C000ECE740F25C53C2F200031A785AB102F1D5
:1060D000FF3140F25C50C2F20000017040F2946364
:1060E000C2F200035D6140F25852C2F20002116830
:1060F000E9B940F25850C2F20000056040F21C536A
:10610000C2F200031A784AB940F25852C2F20002B1
:10611000116861B1284606F083FB08E040F258514F
:10612000C2F20001086840F000630B60ECE740F247
:106130005C50C2F2000003785BB103F1FF3140F222
:106140005C52C2F20002117040F29460C2F2000090
:10615000856140F25853C2F200031968E9B940F270
:106160005852C2F20002156040F21C50C2F2000008
:1061700003784BB940F25853C2F20003196861B179
:10618000284606F04DFB08E040F25851C2F20001EB
:106190000A6842F000600860ECE740F25C52C2F22C
:1061A0000002107858B100F1FF3340F25C51C2F2A6
:1061B00000010B7040F29462C2F20002D56140F21D
:1061C0005850C2F200000368EBB940F25851C2F2D5
:1061D00000010D6040F21C52C2F20002107848B972
:1061E00040F25850C2F20000036863B1284606F03E
:1061F00017FB08E040F25853C2F20003196841F05F
:1062000000621A60ECE740F25C51C2F200010A78C9
:106210005AB102F1FF3040F25C53C2F20003187031
:1062200040F29461C2F200010D6240F25852C2F293
:1062300000021068D8B940F25853C2F200031D6042
:1062400040F21C51C2F200010A783AB140F25850B3
:10625000C2F20000036843F00061016040F258524E
:10626000C2F20002106810B1284606F0D9FA356073
:10627000EAE5D4F800902846FFF742FD40EA09011C
:106280002160D4F804904FF00100FFF739FD40EA97
:1062900009026260D4F808904FF00200FFF730FD69
:1062A00040EA0900A060D4F80C904FF00300FFF71B
:1062B00027FD40EA0903E360D4F810904FF0040092
:1062C000FFF71EFD40EA09012161D4F814904FF058
:1062D0000500FFF715FD40EA09026261D4F8189045
:1062E0004FF00600FFF70CFD40EA0900A061D4F86A
:1062F0001C904FF00700FFF703FD40EA0903E3613C
:10630000D4F820904FF00800FFF7FAFC40EA0901AA
:106310002162306800F1010030603A689042FFF479
:1063200093ADA2E500B585B04FF00003009340F2B5
:10633000FC62C2F2000201924FF0400002904DF266
:106340005810C0F603004FF0060146F26532C0F661
:10635000020201F097FD40F2B863C2F20003186038
:1063600005B000BD2DE9F04F85B040F66C031E4628
:10637000C2F2000640F624000746C2F2000740F2CF
:10638000D861C2F20001019101F012FD3268002AC9
:10639000FAD061E1E359002B53D02846FFF7B0FC57
:1063A00001996258605090434BD0E35910EA0302C0
:1063B00047D0039991F800E04DF26019C0F6030947
:1063C0004FEA451840F2BC61C2F200014FF6FF7C73
:1063D0004DF2580AC0F6030A40F6000BC2F2000B59
:1063E00000957046C2F10003134022EA030218B977
:1063F00054F80B502B4221D15FEA136E04D01AF8E7
:106400000E3003F118030EE01D0C04D01AF805300D
:1064100003F1100307E05FEA132E1ABF1AF80E30DB
:1064200008331AF80330434419F8035031F815E0E3
:10643000E6451CBF0EF1010E21F815E0002AD1D16E
:10644000009D05F1010504F10404092DA2D1029C6F
:10645000621E029240F0F7800399087800F1010073
:10646000C3B20B700B2B03D14FF000040C7002E091
:10647000002B40F0E58040F64802C2F200021168AD
:1064800091B16FEA01003B6803403B6040F60005B4
:10649000C2F200052C682040286040F64801C2F294
:1064A00000014FF000020A6040F64800C2F200000E
:1064B000436893B16FEA03057C682C407C6040F62A
:1064C0000002C2F2000251680D40556040F64800DB
:1064D000C2F200004FF00003436040F64805C2F2EC
:1064E0000005AC6894B16FEA0400BA680240BA6073
:1064F00040F60003C2F2000399680840986040F635
:106500004805C2F200054FF00004AC6040F64800B8
:10651000C2F20000C26892B16FEA0203F968194042
:10652000F96040F60005C2F20005EC682340EB601C
:1065300040F64800C2F200004FF00002C26040F690
:106540004803C2F20003196991B16FEA01053C6981
:106550002C403C6140F60000C2F200000269154088
:10656000056140F64803C2F200034FF000011961D3
:1065700040F64805C2F200056C6994B16FEA040068
:106580007A6902407A6140F60003C2F20003596959
:106590000840586140F64805C2F200054FF000047B
:1065A0006C6140F64800C2F20000826992B16FEA65
:1065B0000203B9691940B96140F60005C2F200054D
:1065C000AC692340AB6140F64800C2F200004FF0D6
:1065D0000002826140F64803C2F20003D96991B11A
:1065E0006FEA0105FC692C40FC6140F60000C2F234
:1065F0000000C2691540C56140F64803C2F20003BD
:106600004FF00001D96140F64805C2F200052C6A3E
:1066100094B16FEA04003A6A02403A6240F600031D
:10662000C2F20003196A0840186240F64805C2F237
:1066300000054FF000042C624FF4FA70029002E063
:106640004FF4FA7502954FF0010001F079FD3268C0
:10665000002A3FF499AE07E04FF4FA75029540F234
:10666000FC74C2F2000403944FF00004254691E646
:1066700010B54FF0000440F66C03C2F200031C603A
:1066800040F60000C2F2000021464FF00902FAF77E
:10669000E5F840F62400C2F2000021464FF009025E
:1066A000FAF7DCF840F64800C2F2000021464FF04D
:1066B0000902FAF7D3F840F2D860C2F2000021468E
:1066C0004FF00902FAF7CAF840F2BC60C2F20000CB
:1066D00021464FF01A0213F06FFC40F2FC70C2F238
:1066E0000000047010BD00BF70B54DF23803C0F655
:1066F00003031B5C4CF6F472C0F6030252F8202030
:1067000040F66C00C2F20000046840F62405C2F2B4
:10671000000555F82300104206D104F1010640F6A9
:106720006C05C2F200052E6049B140F60001C2F2CC
:10673000000151F82350154341F8235009E040F679
:106740000001C2F2000151F8235025EA020541F888
:106750002350104340F62401C2F2000141F8230007
:1067600040F64801C2F2000151F8230020EA02027B
:1067700041F8232034B940F2B863C2F2000318682C
:1067800001F048FB70BD00BF30B44DF23803C0F6D5
:1067900003031B5C4CF6F472C0F6030252F820208F
:1067A00040F62400C2F2000050F82300104229D025
:1067B00040F66C04C2F20004256805F1010525606D
:1067C00071B140F64801C2F2000151F82340144370
:1067D00041F8234040F2FC71C2F20001097889B906
:1067E0006FEA020240F60001C2F2000151F82340B4
:1067F000144041F82340024040F62400C2F2000059
:1068000040F8232030BC704730B4034640F64C12A9
:10681000C2F2000252E8000F00F1010042E8000459
:10682000012CF7D040F2BC60C2F2000030F8132017
:1068300039B140F2BC61C2F200014FF0000421F80E
:10684000134040F64C13C2F2000353E8004FA4F18A
:10685000010443E80045012DF7D053E8004FB4F19F
:10686000004F0DD14FF0000443E80045012DF4D056
:106870004EF60450CEF20000016841F080510160F4
:10688000BFF32F8F104630BC704700BF40F2FC733F
:10689000C2F200031878D0F1010038BF0020704721
:1068A0002DE9F84FDFF834814B4FC8EB07004FEA72
:1068B000D00707F101074FF0000540F2982AC0F613
:1068C000000A40F28039C0F6000931E044464FF03A
:1068D00000066FEA060B0BEB070101F0010B58F8FD
:1068E000043CAB4229D135E054F8043CAB4205D11D
:1068F00054F8080C8047FBF787FD0BE0FF2B09D904
:10690000FF2D07D154F8040C4FF0070154F8082C60
:1069100001F0D8FB06F1010604F1080454F8041C48
:10692000A94240D14CE005F10105B5F5807F02D0C8
:10693000CA45CBD3F7E7BDE8F88FFF2B0FD9FF2D62
:106940000DD158F8040C4FF0070158F8082C01F04D
:10695000B9FB04E058F8082C9047FBF755FD06F109
:10696000010604F10804BE42DDD0BBF1000FBBD02C
:1069700054F8040CA8420AD0FF280DD9FF2D0BD1E2
:106980004FF0070154F8082C01F09CFB04E054F888
:10699000081C8847FBF738FD06F1010604F10804DE
:1069A000BE42A1D1BFE7FF290FD9FF2D0DD154F869
:1069B000040C4FF0070154F8082C01F083FB04E0AD
:1069C00054F8082C9047FBF71FFD06F1010604F16F
:1069D0000804BE4288D1A6E787030008A002000889
:1069E000027840F6E103C2F200031B789A4206D314
:1069F0004FF000020270087800F1010008700A7878
:106A000040F6E203C2F200031878824224BF00205D
:106A10000870704738B140F61840C4F202004FF0D9
:106A200002010180704740F61A43C4F202034FF09E
:106A300002021A80704700BF08B540F61843C4F23E
:106A400002034FF008021A8000EA0201CBB23BB108
:106A500040F61843C4F202034FF08001198006E0AB
:106A600040F61A41C4F202014FF080020A8000F0A1
:106A70000402D3B23BB140F61841C4F202014FF018
:106A800040030B8006E040F61A41C4F202014FF0C9
:106A900040020A8010F0010F19BF40F61841C4F2FD
:106AA000020140F61A41C4F202014FF010020A80BE
:106AB00000F00200C1B239B140F61840C4F2020041
:106AC0004FF02001018006E040F61A43C4F20203B1
:106AD0004FF020021A804FF0010003F081FA40F6D7
:106AE0001A43C4F202034FF008021A8008BD00BF27
:106AF00010B50C46FFF78EFF40F61843C4F20203B0
:106B00004FF008021A8014F0800F19BF40F61843A6
:106B1000C4F2020340F61A43C4F202034FF08000AD
:106B2000188004F04001CBB23BB140F61841C4F2EA
:106B300002014FF040030B8006E040F61A40C4F219
:106B400002004FF04002028004F01000C2B23AB1DD
:106B500040F61840C4F202004FF01002028006E036
:106B600040F61A41C4F202014FF010030B8004F00A
:106B70002001CBB23BB140F61841C4F202014FF004
:106B800020030B8006E040F61A40C4F202004FF0EA
:106B9000200202804FF0010003F022FA40F61A4072
:106BA000C4F202004FF0080202802046FFF744FFC3
:106BB0004FF0320003F014FA10BD00BF08B50329EE
:106BC00014D8DFE801F0020B05084FF0800107E060
:106BD0004FF0940104E04FF0D40101E04FF0C00108
:106BE0000A184FF00000D1B2FFF782FF08BD00BFC6
:106BF00008B540F6F603C2F20003187830B940F643
:106C0000EC01C2F20001086801F004F940F6F60355
:106C1000C2F200034FF002021A7008BD10B5A0F1D5
:106C20000803052B3DD8DFE803F01F3C2C3C03850F
:106C300040F67C00C2F200004FF020014FF05402F9
:106C400013F0BAF940F6D400C2F200004FF0FF3161
:106C50004FF00C0213F0B0F940F6F000C2F2000061
:106C6000026802F1010202604FF0000140F6760373
:106C7000C2F20003197040F67700C2F20000017002
:106C800056E040F67601C2F200014FF000030B70AF
:106C900040F67700C2F20000027802F101020270B1
:106CA0003CE040F67602C2F20002127840F677012C
:106CB000C2F200010B7840F6E101C2F2000109784E
:106CC00001FB032340F67C01C2F20001C95C814252
:106CD0001DD040F67C04C2F20004E0544FEA531089
:106CE00040F6D401C2F2000103F01F034FF001048B
:106CF00004FA03F351F820401C4341F8204040F6C9
:106D0000F000C2F20000016801F10101016002F12E
:106D1000010240F67603C2F200031A7040F67600D4
:106D2000C2F2000040F67701C2F20001FFF758FE00
:106D3000FFF75EFF4FF0000010BD00BF70B4039D71
:106D4000049C064628B140F6E300C2F20000007839
:106D5000307029B140F6F400C2F2000000780870EB
:106D60002AB140F6E001C2F20001087810702BB1A0
:106D700040F6F502C2F20002117819702DB140F60A
:106D80007603C2F20003187828702CB140F677021F
:106D9000C2F200021178217070BC704706281DD81D
:106DA000002808BF022040F6E303C2F20003187077
:106DB0004DF28423C0F6030313F8101040F6E102ED
:106DC000C2F20002117003EB4000417840F6E2038A
:106DD000C2F2000319704FF0010070474FF000003D
:106DE000704700BF10B540F6F403C2F200034FF045
:106DF00001021A704FF00200FFF7D0FF4FF00004BD
:106E000040F67800C2F20000046040F6E801C2F2E9
:106E100000010C604DF28020C0F603004FF08701A6
:106E200047F28932C0F6020201F04CF940F6EC0359
:106E3000C2F2000318604FF00C002146FFF7EEFE8F
:106E400010BD00BF034628B140F6E100C2F20000C9
:106E50000078187029B140F6E203C2F200031878F6
:106E600008702AB140F6F001C2F200010B6813600D
:106E700040F67C00C2F20000704700BF2DE9F041EF
:106E800040F67C07C2F200073F1853284DD8002A6D
:106E90004BD03B4607F1010702F1FF3257FA82F768
:106EA0004FF0000640F6D404C2F200044FF0010592
:106EB0006FEA030C0CEB070202EA050C13F8018BD6
:106EC00001F1FF3111F8012F904530D13EE013F868
:106ED00001CB01F1010049788C450ED003F8011C6B
:106EE0004FEA521102F01F0605FA06FC54F8216021
:106EF0004CEA060644F821602E4602F10102D2B2A5
:106F0000542A07D013F801CB00F1010140788445E1
:106F100043D151E04EB140F6F003C2F200031968CC
:106F200001F101011960FFF763FEBDE8F08103F88C
:106F3000012C4FEA501600F01F0805FA08F854F823
:106F4000262048EA020244F826202E4600F10100DD
:106F5000C2B2542ADED0BB42DCD0BCF1000FB6D0A6
:106F600013F801CB11F8010F84450ED003F8010C82
:106F70004FEA521002F01F0605FA06FC54F8206092
:106F80004CEA060644F820602E4602F10102D2B215
:106F9000542ABFD0BB429AD1BCE703F8010C4FEA98
:106FA000521002F01F0605FA06FC54F820604CEA65
:106FB000060644F820602E4602F10102D2B2542A9D
:106FC000A8D0BB4283D1A5E740F6D003C2F20003AC
:106FD0004FF000021A7070474FF05400704700BF26
:106FE00038B540F6D003C2F20003187868B14FF00C
:106FF000050540F6D004C2F20004FBF705FA284666
:1070000001F09EF821780029F7D140F6D003C2F2B2
:1070100000034FF001021A7038BD00BF38B54FF0C1
:10702000000240F6E803C2F200031868B0F1FF3F27
:1070300000F0CE8010B140F001010847FFF7D0FF0B
:1070400040F6F600C2F200004FF0010202704FF06D
:10705000000340F67001C2F200010B6040F67500BB
:10706000C2F20000037089E040F67403C2F200032C
:107070004FF000021A704FF001026BE040F670050D
:10708000C2F200052B684FF0010103F01F0401FA62
:1070900004F44FEA531340F6D405C2F2000555F844
:1070A00023301C4245D0AAB140F67501C2F200015E
:1070B0000978FFF783FD40F6E800C2F20000494B73
:1070C00003604FF0010038BD40F6E804C2F200044E
:1070D000444A226040F67004C2F2000421684FF076
:1070E000010040F67C02C2F20002515CFFF700FD95
:1070F00020684FEA501240F6D403C2F2000300F0B9
:107100001F044FF0010000FA04F153F8224024EA72
:10711000010443F8224040F6E803C2F20003324A79
:107120001A6038BD40F6E803C2F200032E4818602A
:1071300000E00A4640F67403C2F20003197801F138
:107140000101197040F67000C2F20000036803F1FB
:107150000103036040F67401C2F20001087840F6B2
:10716000E103C2F200031978814287D840F6750026
:10717000C2F20000027802F10102027040F67503CB
:10718000C2F20003197840F6E200C2F20000027871
:107190009142FFF469AF40F6F603C2F2000319789A
:1071A00001297FF44DAF40F6F600C2F200004FF027
:1071B0000002027040F67603C2F20003187840F62F
:1071C0007701C2F200010978FFF7F8FCFFF7FCFE37
:1071D00040F6E801C2F200014FF000020A604FF0F1
:1071E000030038BDC87002082471020808B50030D9
:1071F00018BF012040F6F403C2F2000318700031FA
:1072000018BF012140F6E000C2F200000170003218
:1072100018BF012240F6F503C2F200031A70FFF70F
:10722000DFFE40F6E401C2F20001087800B340F648
:10723000F402C2F200021378002B14BF04200020D5
:1072400040F6E001C2F200010A78002A14BF0223CE
:10725000002340F6F501C2F200010A78002A14BFAB
:107260000921082101434FF000001943FFF740FCBA
:10727000FFF7AAFE08BD00BF10B540F60043C4F2F8
:1072800002031A684FF0010464F387121A60186849
:1072900064F383001860196864F3092119601A689F
:1072A00064F38B221A60186864F30D301860196853
:1072B00064F38F3119604FF00000FFF7ABFB4FF024
:1072C0000300FFF7B9FB41F2040002F089FE4FF022
:1072D0000300FFF7B1FB4FF0640002F081FE4FF0B6
:1072E0000300FFF7A9FB4FF0320002F079FE4FF0E8
:1072F0000200FFF7A1FB4FF0320002F071FEFFF732
:107300006FFE4FF000004FF02801FFF7F1FB4FF048
:1073100000004FF00601FFF7EBFBFFF755FE40F6CC
:10732000E403C2F200031C7040F6F402C2F2000251
:10733000107840F6E001C2F20001097840F6F5034A
:10734000C2F200031A78FFF751FFFFF749FE4FF032
:1073500000002146FFF7CCFB40F2A46002F040FEA3
:10736000FFF732FEFFF73CFE40F67600C2F2000067
:10737000007840F67702C2F200021178FFF71EFC97
:10738000FFF722FE10BD00BF10B540F6F603C2F2B3
:1073900000034FF001021A704FF47A7000F0D0FE33
:1073A000FFF76AFF4FF0020402E0204600F0C8FE3B
:1073B000FFF734FE0128F8D000F0FAFCF8E700BF30
:1073C0002DE9F04180460C46174640F6E403C2F230
:1073D0000003187868B94FF0320640F6E405C2F2AF
:1073E0000005FBF711F8304600F0AAFE29780029C5
:1073F000F7D04FF4FA6002F0F3FDFFF7F1FD4FF024
:10740000000048F04001FFF773FB4FF0320002F03C
:10741000E7FD4FEAC702D3B203F1FF37FFB2FBB17A
:1074200007F10107E7194FF001066FEA0405781923
:1074300000EA0605304614F8011BFFF759FBBC4271
:1074400022D10DE0254615F8011B3046FFF750FB11
:10745000617805F101043046FFF74AFBBC42F1D1E7
:1074600040F67401C2F20001087840F67502C2F2DB
:1074700000021178FFF7A2FB4FF0320002F0B0FDDE
:10748000FFF7A2FDBDE8F081002DDBD0304614F8F7
:10749000011BFFF72DFBBC42D4D1E1E708B540F654
:1074A0007602C2F20002107040F67703C2F20003C7
:1074B000197010461946FFF793FA40F6E000C2F241
:1074C0000000017879B1FFF78BFD40F67602C2F239
:1074D0000002107840F67703C2F200031978FFF734
:1074E0006DFBFFF771FD08BD10B5044640F6F800CE
:1074F000C2F2000001F0C2F92CB140F62710C2F22E
:107500000000017804E040F62613C2F20003197867
:1075100040F62412C2F20002117040F62513C2F2A6
:1075200000031C704FF00300FBF774F810BD00BFA0
:1075300010B582B040F62014C2F20004206800307A
:1075400018BF0120FFF7D0FF216879B14FF0000389
:107550000093019340F6F800C2F200004FF0FF02E2
:1075600047F2E943C0F6020301F02EFA02B010BD63
:1075700010B5082824DC082925DC002804DB40F6A7
:107580002614C2F200042070002904DB40F6271004
:10759000C2F200000170002A08DBC2EB02124FEABF
:1075A000820040F62011C2F20001086040F61C1271
:1075B000C2F200021370FFF7BBFF4FF0010010BDD5
:1075C0004FF0000010BD4FF0000010BD40F6241336
:1075D000C2F2000318787047034628B10868834256
:1075E00014BF0020012070474FF00000704700BF1B
:1075F00010B440F64C13C2F2000353E8002F02F11E
:10760000010243E800210129F7D00468C4B162688F
:10761000824202D19268626002E0436881689960A8
:107620002368834202D15B68236002E0826841687C
:107630005160A26802F1FF31A1604FF000040460C4
:1076400040F64C13C2F2000353E8002FA2F10102EE
:1076500043E80024012CF7D053E8002FB2F1004F8B
:107660000DD14FF0000243E80024012CF4D04EF677
:107670000450CEF20000016841F080510160BFF378
:107680002F8F10BC704700BF38B504460D464FF031
:1076900000014FF0100212F08FFCE56038BD00BF12
:1076A000F8B504460F46C6688D192946FFF794FFC2
:1076B00000283CD140F64C13C2F2000353E8002FDF
:1076C00002F1010243E800210129F7D04FF0000048
:1076D00068606168A96001B14D60226802B92560E7
:1076E0006560BC51A36803F10103A36040F64C132D
:1076F000C2F2000353E8002FA2F1010243E8002484
:10770000012CF7D053E8002FB2F1004F0DD14FF00C
:10771000000243E80024012CF4D04EF60450CEF2CF
:107720000000016841F080510160BFF32F8FF8BD68
:107730002DE9F04104468846C6688D199719C2B9EB
:1077400040F64C13C2F2000353E8002F02F101028D
:1077500043E800210129F7D002686A6005604FF014
:107760000000A860616809B9656020E06B689D60F1
:107770001DE03946FFF730FF00283FD02846FFF7CD
:1077800037FF40F64C13C2F2000353E8002F02F11A
:10779000010243E800210129F7D0B868A8606F60B2
:1077A000BD602168B9420EBF2560A9684D6048F8E8
:1077B0000640A26802F10102A26040F64C13C2F238
:1077C000000353E8002FA2F1010243E80024012C3A
:1077D000F7D053E8002FB2F1004F0DD14FF0000267
:1077E00043E80024012CF4D04EF60450CEF2000001
:1077F000016841F080510160BFF32F8FBDE8F08137
:10780000C368C918486808B1C01A70474FF0000033
:10781000704700BF036813B1C068181A70474FF073
:107820000000704708B5C368C918FFF7D5FE08BD4A
:1078300008B5C0680818FFF7DBFE08BD08B540F6BC
:107840002810C2F200004FF01C01FFF71DFF08BD19
:1078500070B5054600F108063046FFF7DBFF044629
:10786000686050B130462146FFF7E2FF4FF001005B
:10787000A861204600F0CEFA70BD4FF00003AB6166
:1078800070BD00BF38B504460D464FF000014FF003
:10789000280212F091FB204640F8085B4FF01C01D3
:1078A000FFF7F2FE40F62810C2F200002146FFF773
:1078B000F7FE38BD2DE9F0410746884643F258539C
:1078C000C2F200031868002800F0FE8040F64C1455
:1078D000C2F2000454E8002F02F1010244E8002142
:1078E0000129F7D0796831B143F25852C2F200024F
:1078F000136899422ED143F25850C2F20000046836
:107900007C60B96901F10101B96140F64C13C2F222
:10791000000353E8002FA2F1010243E80024012CE8
:10792000F7D053E8002FB2F1004F0DD14FF0000215
:1079300043E80024012CF4D04EF60450CEF20000AF
:10794000016841F080510160BFF32F8F4FF00100BB
:10795000BDE8F081B8F1FF3F24D140F64C13C2F2EC
:10796000000353E8002FA2F1010243E80024012C98
:10797000F7D053E8002FB2F1004F0DD14FF00002C5
:1079800043E80024012CF4D04EF60450CEF200005F
:10799000016841F080510160BFF32F8F4FF000006C
:1079A000BDE8F08107F108052846FFF733FF0246DE
:1079B000F0B143F25856C2F20006306892F82940FE
:1079C00090F829108C4208D912E0336892F8290007
:1079D00093F82940A04204D90AE043F25856C2F273
:1079E000000628461146FFF70BFF02460028ECD19F
:1079F000284643F25851C2F200010968FFF798FE89
:107A000040F64C16C2F2000656E8002FA2F1010221
:107A100046E80024012CF7D056E8002FB2F1004FC1
:107A20000DD14FF0000246E80024012CF4D04EF6B0
:107A30000450CEF20000016841F080510160BFF3B4
:107A40002F8FB8F1000F04D008EB880000F078FB0E
:107A500001E000F0ADF940F64C14C2F2000454E825
:107A6000003F03F1010344E80032012AF7D043F25A
:107A70005856C2F2000628463168FFF7D9FE54E88E
:107A8000003FA3F1010344E80032012AF7D054E893
:107A9000003FB3F1004F0DD14FF0000344E8003236
:107AA000012AF4D04EF60450CEF20000016841F0F5
:107AB00080510160BFF32F8F78683268904214BF05
:107AC00000200120BDE8F0814FF00100BDE8F08109
:107AD00010B5044643F25853C2F200031868002858
:107AE00060D06268904201D0F8F7A8FE40F64C13CF
:107AF000C2F2000353E8002F02F1010243E8002123
:107B00000129F7D0A16901F1FF30A06118B340F657
:107B10004C13C2F2000353E8002FA2F1010243E824
:107B20000024012CF7D053E8002FB2F1004F0DD103
:107B30004FF0000243E80024012CF4D04EF604502C
:107B4000CEF20000016841F080510160BFF32F8F39
:107B50004FF0000010BD2046FFF77AFE40F64C13B0
:107B6000C2F2000353E8002FA2F1010243E800240F
:107B7000012CF7D053E8002FB2F1004F0DD14FF098
:107B8000000243E80024012CF4D04EF60450CEF25B
:107B90000000016841F080510160BFF32F8F4FF06A
:107BA000010010BD4FF0010010BD00BFF8B5054643
:107BB00040F64C13C2F2000353E8002F02F1010219
:107BC00043E800210129F7D040F62810C2F2000056
:107BD000FFF720FE0446E0B140F62817C2F2000786
:107BE0006068A84203D12046FFF732FE0AE004F1A4
:107BF000080630462946FFF715FE18B130462946DB
:107C0000FFF716FE38462146FFF7FAFD0446002826
:107C1000E6D140F64C13C2F2000353E8002FA2F164
:107C2000010243E80024012CF7D053E8002FB2F101
:107C3000004F0DD14FF0000243E80024012CF4D096
:107C40004EF60450CEF20000016841F08051016010
:107C5000BFF32F8FF8BD00BF02282BD111F0030F07
:107C60001FD148F21F52C5F2EB12A2FB01204FEACE
:107C700050134FF0640202FB131083B2A3B948F211
:107C80001F52C5F2EB12A2FB01204FEAD0134FF4B2
:107C9000C87202FB131188B2D0F1010338BF002370
:107CA00004E04FF0000301E04FF0010303F11C0377
:107CB000D8B2704700F1FF3042F29343C9F2492332
:107CC00083FB00210B184FEAE072C2EBA301C1EB6A
:107CD000C103C21A4FF00101C8F20001114000298E
:107CE00005DA01F1FF3060F0010101F10101C1F19C
:107CF0001F03D8B2704700BF08B54DF29023C0F6FD
:107D00000303195C012906D011B102290BD105E04A
:107D1000FCF790FD08BD02F023F908BDF8F78EFDD1
:107D20004FF0000008BD4FF0000008BD4EF60453B0
:107D3000CEF200031A6842F080501860704700BF0E
:107D40004FF0010280F8282040F64813C2F20003E9
:107D500090F8291002FA01F2188802431A8070473D
:107D600010B440F64413C2F200031A68C2B1904244
:107D700013D104E088420FD102F1140203E040F66F
:107D80004412C2F2000243691BB19C698169611807
:107D900099614369136003E00A4651690029E9D1FA
:107DA0004FF0000282614FF0FF31416110BC70471B
:107DB00010B5F8F799FD044643F25853C2F2000398
:107DC000186890F82820032A1BD0F8F78DFD43F29D
:107DD0005853C2F2000319684FF0000281F82820BE
:107DE00091F82920096940F63823C2F2000343F8CC
:107DF0002210F8F783FD2046F8F780FDFFF796FF85
:107E000010BD4FF0020180F828102046F8F776FDEB
:107E100010BD00BF38B5044690B3036883B3F8F7CC
:107E200063FD054694F8280010BB2046FFF788FF45
:107E300043F25851C2F200010B6843B194F8292073
:107E400093F8290020F00101531A002B15DA40F6AF
:107E50004C12C2F20002106838B140F0004140F606
:107E60004C13C2F20003196007E0FFF75FFF04E064
:107E7000022804BF032084F828002846F8F73EFDB6
:107E800038BD00BF2DE9F04F85B006460F4693463A
:107E900098460F9DDDF84090F8F726FD824640F6A3
:107EA0009013C2F200031968504881420FD240F289
:107EB0000002C2F2020252F82C4C54B14C4B1C4648
:107EC0008B4207D953F82C090028F8D102E0474C1F
:107ED00000E0464CA14206D1A1F12C0140F69012DF
:107EE000C2F20002116020464FF000014FF02C0258
:107EF00012F062F84FF0FF3161611EB94DF2942625
:107F0000C0F603062660B8F1000F08D00E9B042BC4
:107F100008D9184600F103004FEA900604E04FF03C
:107F2000000601E04FF000060DBB44F25C09C2F20E
:107F3000000940F63815C2F20005296848F2A13060
:107F4000C0F602000090CDF80480029648464FF03B
:107F500000025B46F9F700F82A68A260E0604FEA89
:107F6000800153182B60C1EB0900606020E02846B7
:107F70004FF0FF314A46F8F771FC4AF2ED52CDF668
:107F8000CE622A60E56005EB8905656048F2A131A3
:107F9000C0F602010091CDF80480029628462946D9
:107FA0004FF001025B46F8F7D7FFA5EB8003636053
:107FB0006FEA0702C2F3C01101EB470707F0FF07A2
:107FC00084F8297040F65013C2F2000353F82700DA
:107FD000206143F827405046F8F790FC2046FFF711
:107FE00019FF204605B0BDE8F08F00BFD4FF012087
:107FF000A8FF012030B585B04FF0000143F258537F
:10800000C2F200031960284C40F20005C2F20205DA
:108010002A1B20464FEAA202F8F720FC40F638104F
:10802000C2F200000460A5F12C0540F69011C2F2E6
:1080300000010D6043F65C03C2F200034FF0B5048B
:10804000CBF26B141C6003F14C004FF0FF3243F88D
:10805000042F43F8042F43F8042F8342F9D14FF043
:108060000004009440F69411C2F2000101914FF017
:10807000280302934DF2A020C0F603004FF0070141
:1080800048F22112C0F602022346FFF7FBFE40F63B
:108090003422C2F20002106040F65010C2F200001A
:1080A000C46305B030BD00BF6040002010B584B08F
:1080B000069C00944FF0000401940294FFF7E2FE46
:1080C00004B010BD00B585B04FF0000300930193DC
:1080D0000293FFF7D7FE05B000BD00BF38B543F2ED
:1080E0005853C2F200031868C0B1F8F7FDFB05460B
:1080F00043F25854C2F200042068FFF721FE2168C1
:1081000091F82920086940F63823C2F2000343F8A9
:1081100022002846F8F7F2FBFFF708FE38BD00BF43
:1081200038B543F25855C2F2000540F65014C2F279
:1081300000042B6822681A61FFF7D0FFF9E700BF3F
:1081400038B543F25853C2F200031968002900F011
:10815000918020B9FFF7C2FF4FF001029AE0B0F121
:10816000FF3F04D1FFF724FE4FF0000292E040F6FB
:108170004C14C2F2000454E8002F02F1010244E85A
:1081800000210129F7D040F64412C2F2000215681E
:10819000002D7AD0AB6998426FD3C01A05F1140153
:1081A0006D691DB1AB698342F7D96AE043F2585556
:1081B000C2F200052B689861086858611846F8F704
:1081C00041FB40F64C14C2F2000454E8003FA3F116
:1081D000010344E80032012AF7D054E8003FB3F12C
:1081E000004F0DD14FF0000344E80032012AF4D0D3
:1081F0004EF60450CEF20000016841F0805101605B
:10820000BFF32F8FFFF7D4FD54E8003F03F10103C4
:1082100044E80032012AF7D028684169B1F1FF3FF4
:1082200004D0FFF79DFD4FF0000201E04FF0010286
:1082300040F64C13C2F2000353E8004FA4F10104CE
:1082400043E80045012DF7D053E8004FB4F1004F4B
:108250000DD14FF0000443E80045012DF4D04EF657
:108260000450CEF20000016841F080510160BFF37C
:108270002F8F0FE04FF001020CE040F64411C2F2E4
:108280000001AC69221AAA6190E740F64411C2F2DB
:1082900000018BE7104638BDF8B5044600287AD0B7
:1082A000F8F722FB064640F69013C2F20003196865
:1082B0003948814211D240F20002C2F2020252F861
:1082C0001C5CA54263D0354B1D468B4205D9A3F1FA
:1082D0002C03D86BA042F7D15AE094F8293040F62D
:1082E0005012C2F2000252F82300A04206D10169E6
:1082F00040F65012C2F2000242F823102046FFF767
:108300002FFD2046FFF752FC94F82900236940F620
:108310003821C2F2000141F8203043F25852C2F233
:1083200000021068A04229D0A06838B3E76800EBCB
:10833000870540F63817C2F200073B685A1B2946EA
:108340004FEAA2024FF00003FBF762F8E1683868D9
:10835000A0EB81033B6040F69012C2F2000211686C
:108360000D4B99420AD29A68954203D8E068A2EB75
:1083700080029A60A3F12C038B42F4D84FF00001E5
:10838000216084F828103046F8F7B8FAF8BD024D9D
:1083900021692961A1E7F8BDD4FF0120A8FF0120D0
:1083A00000BFF04772B643F25854C2F2000420688E
:1083B000FFF772FF4FF000032360F8F71DFE00BFC8
:1083C00040F64413C2F20003196849B1886950B1FC
:1083D00000F1FF328A61D2F1010038BF00207047FE
:1083E0004FF0000070474FF00000704770B540F646
:1083F0004413C2F200031C68A4B1A06990B940F60E
:108400004415C2F200054FF0FF3660692946F8F7BF
:1084100019FA66612046FFF7FDFC2C6814B1A169CA
:108420000029F2D070BD00BFF0B472B640F6481318
:10843000C2F200031C882CB940F63423C2F20003B8
:1084400018685FE04DF2A82CC0F6030C40F6382502
:10845000C2F2000540F65016C2F20006C4F1000355
:1084600023401A0A1ABF1CF8021008311CF8031026
:1084700011F0010F0AD141F0010055F8200038B188
:1084800090F82820012A38D81F4602E01F4600E055
:108490001F4655F82120B2B192F828307BB140F642
:1084A0004810C2F20000048010462BE090F82830FB
:1084B00033B140F64812C2F20002148022E01046A6
:1084C00000690028F2D156F82100824207D1BC434E
:1084D000C4D140F64811C2F200010C80ACE745F867
:1084E000210011F0010FD4D114EA4703D1D04FEA93
:1084F0004707BFB241F00101CBE740F64811C2F295
:1085000000010C8062B6F0BC704700BF70B543F24A
:108510005853C2F200031B6883420FD193F82820FE
:10852000012A9CBF022283F8282093F8291040F6E4
:108530003820C2F2000040F8213070BD40F63C12F5
:10854000C2F20002136043F25851C2F20001086007
:1085500090F8292040F63823C2F2000343F82200A5
:1085600090F8281001299CBF022180F82810826809
:10857000AAB9C1684AF2ED53CDF6CE6308689842B5
:1085800001D0F8F75BF943F25852C2F200021168C9
:108590004868CB6898427ED2F8F750F970BD40F633
:1085A0004013C2F200031B68984274D093B358681A
:1085B00044F25C04C2F20004251A4FEAA501D96016
:1085C00043F65C02C2F2000290420AD34FF0B503B8
:1085D000CBF26B1343F65C00C2F2000004689C42CD
:1085E00001D0F8F72BF940F64015C2F200052A68D1
:1085F00040F63814C2F2000420685168D2684FF087
:108600000003FAF705FF296823688B60C86803EB4D
:108610008002226043F25851C2F200010B6840F61A
:108620004010C2F200000360DA68002A33D05868B4
:1086300099684FF00103FAF7EBFE43F25856C2F285
:1086400000063568A868EC6800EB840440F638162C
:10865000C2F200063268131B21464FEAA3024FF014
:108660000003FAF7D5FEE9683068A0EB81023260BA
:1086700040F69013C2F200031968074B99420AD2E0
:108680009A68944203D8E868A2EB80029A60A3F14A
:108690002C038B42F4D870BDD4FF012000B585B007
:1086A00040F6D430C2F200004FF00001FEF7ECFFBC
:1086B00040F67C20C2F200004FF00001FEF7E4FF1C
:1086C0004FF00003009340F69422C2F200020192A0
:1086D0004FF0500002904DF2A830C0F6030019464A
:1086E00048F61922C0F60202FFF7CCFB40F67823C9
:1086F000C2F20003186005B000BD00BF08B5FFF767
:1087000089F8034648B1C06850B100F1FF31D96023
:10871000D1F1010038BF002008BD4FF0000008BDB6
:108720004FF0000008BD00BF70B505460E46144668
:1087300040F64C13C2F2000353E8002F02F101028D
:1087400043E800210129F7D0FFF764F8024600282A
:1087500039D0C06884422DD3241A28461146FFF729
:108760004FF8024600282ED0C068A042F4D921E07C
:1087700040F64C13C2F2000353E8002FA2F10102AD
:1087800043E80024012CF7D053E8002FB2F1004F4A
:108790000DD14FF0000243E80024012CF4D04EF636
:1087A0000450CEF20000016841F080510160BFF337
:1087B0002F8F70BDF460D1680B1BD3602846314603
:1087C000FEF7B6FFD4E7F46028463146FEF768FFAF
:1087D000CEE700BFF8B50646FFF71CF80446F8B12F
:1087E000C368EBB930462146FFF70AF80546F8F7AB
:1087F0007BF8074630462146FFF71AF83846F8F767
:108800007DF822691AB130462146FFF78DFF04F149
:108810001400FDF769F91DB12C46E8680028E1D085
:10882000F8BD00BF08B540F69023C2F200031A68F5
:1088300002F101021A6040F67C20C2F20000FFF74C
:108840005DFF28B140F67C20C2F20000FFF7C2FFB6
:1088500008BD00BF08B5014640F6D430C2F20000A2
:10886000FEF7E0FF20B140F6D430C2F2000008BDB0
:1088700040F67C20C2F2000008BD00BF70B504467F
:1088800040F64C13C2F2000353E8002F02F101023C
:1088900043E800210129F7D0FFF7DCFF0546214618
:1088A000FEF7C0FF002845D040F64C10C2F2000091
:1088B00050E8002F02F1010240E800210129F7D021
:1088C00028462146FEF79CFF18B1C168E2688B1864
:1088D000C360F8F709F8064628462146FEF7A8FFC8
:1088E0003046F8F70BF84FF0FF35E56040F64C13D3
:1088F000C2F2000353E8002FA2F1010243E8002571
:10890000012DF7D053E8002FB2F1004F0DD14FF0F9
:10891000000243E80025012DF4D04EF60450CEF2BB
:108920000000016841F080510160BFF32F8F4FF0CC
:10893000010501E04FF0000504F11400FDF7CEF849
:1089400040F64C13C2F2000353E8002FA2F10102DB
:1089500043E80024012CF7D053E8002FB2F1004F78
:108960000DD14FF0000243E80024012CF4D04EF664
:108970000450CEF20000016841F080510160BFF365
:108980002F8F284670BD00BF2DE9F04105460F46E8
:1089900014469846FFF772FF064694B19DF82030C2
:1089A000002B14BF20460020286105F11400414629
:1089B000069A079BFDF778F8384629462246FFF7C6
:1089C000B3FE3046BDE8F08170B584B00E46154662
:1089D0000093089C01949DF82430029340F67C217A
:1089E000C2F2000132462B46FFF7CEFF04B070BD45
:1089F00070B584B00E4615460093089C01949DF80E
:108A00002430029340F6D431C2F2000132462B46A4
:108A1000FFF7BAFF04B070BD00B583B04FF000039C
:108A200000934FF00100019040F6E430C2F20000E4
:108A300041F288314FF0FF0248F62503C0F60203E9
:108A4000FFF7D6FF40F6D434C2F20004FFF7CEFCA5
:108A50002046FFF7BFFEFFF7ABF9F7E740F68C23A0
:108A6000C2F2000318681A689042FBD1704700BF39
:108A700010B540F68C23C2F200031A6802F101021D
:108A80001A60FFF79DFC044640F6D430C2F20000A5
:108A9000FFF734FE204310F0FF0F06D040F6782099
:108AA000C2F200000068FFF7B5F910BD08B54DF23D
:108AB0004440C0F603004FF0060148F6E962C0F6F4
:108AC0000202FFF7FFFA40F61473C2F200031860C7
:108AD00008BD00BF38B504460D4640F60843C2F253
:108AE0000003586AA0420AD040F60841C2F20001D1
:108AF0004C620A681AB115B14948FCF7F5FF40F617
:108B00000843C2F20003186F84420AD040F60841BD
:108B1000C2F200010C67CA6C1AB115B14148FCF7EA
:108B2000E3FF40F60843C2F20003D3F8BC008442DE
:108B30000CD040F60841C2F20001C1F8BC40D1F8A7
:108B400098201AB115B13848FCF7CEFF40F608431B
:108B5000C2F20003D3F8080184420CD040F6084169
:108B6000C2F20001C1F80841D1F8E4201AB115B1F0
:108B70002E48FCF7B9FF40F60843C2F20003D3F8D1
:108B8000540184420CD040F60841C2F20001C1F801
:108B90005441D1F830211AB115B12548FCF7A4FF92
:108BA00040F60843C2F20003D3F8A00184420CD07F
:108BB00040F60841C2F20001C1F8A041D1F87C2181
:108BC0001AB115B11B48FCF78FFF40F60843C2F2FB
:108BD0000003D3F8EC0184420CD040F60841C2F205
:108BE0000001C1F8EC41D1F8C8211AB115B1124801
:108BF000FCF77AFF40F60843C2F20003D3F83802CC
:108C0000A0420CD040F60841C2F20001C1F838423F
:108C1000D1F814221AB115B10848FCF765FF38BD28
:108C2000180C0020640C0020B00C0020FC0C00206C
:108C3000480D0020940D0020E00D00202C0E002097
:108C40002DE9F04707460D4691460898DDF8288043
:108C50000C683E68D8F800108A19944202D80219AC
:108C6000964203D304192C60BDE8F087341B061B21
:108C7000B14234BF8A46B246099931B1D9F80000F1
:108C800008181919524611F073F9D8F80030CAEBD8
:108C90000302C8F800203E6806EB0A013960D9F8E3
:108CA000000000EB0A03C9F800302E68A4195444F0
:108CB0002C60BDE8F08700BF70B584B09CF81960E7
:108CC000157A947B4FF007038CF810304FF00502B3
:108CD0008CF8112006F00F0260F3C7128CF81220F6
:108CE0004FF0000065F301008CF813004FF0000214
:108CF00061F30A02ACF814208CF81640DCF80C1072
:108D00000093DCF804300193CDF808C001F10400B1
:108D10000CF108020CF11003FFF792FF04B070BDD4
:108D20002DE9F04F8FB00746059114464FF0000330
:108D30000793136012896068131A8B4238BF05933A
:108D40000599002900F0AA8040F61875C2F20005C6
:108D50002D6815B34FEAC5054FF000024FF0FF0133
:108D6000134640F62070C2F20000A5F10806C6F3D3
:108D7000C00E1658F6798E4240F0958096E016584F
:108D8000F6798E421CBF0133314602F10802865843
:108D9000F6798E4240F09F80A0E04FF0000303EB95
:108DA00043024FEAC20000F1100008904FF48071B6
:108DB000ADF824104FF00402ADF826208DF82830CD
:108DC0000DF129004FF000014FF0070211F0F4F807
:108DD00004F1040B04944FF010030093019705A8CD
:108DE00002905846214607AA08ABFFF729FF0599CC
:108DF000002951D04FF001028DF821200DF13200F1
:108E00004FF000014FF0060211F0D6F840F618734B
:108E1000C2F20003186800283ED04FF0FF014FF067
:108E2000000440F62079C2F200094DF2B438C0F6D1
:108E3000030840F6187AC2F2000A59F83450ED7966
:108E40008D4223D08DF820404FEA05160DF1220007
:108E500008EB06014FF0080211F08AF806F108014C
:108E60000DF12A0041444FF0080211F081F84FF053
:108E700018020092019705AB02935846049907AA7D
:108E800008ABFFF7DDFE059830B1294604F1010477
:108E9000DAF80020A242D0D8079801E04FF0FF3066
:108EA0000FB0BDE8F08F03F10103314602F1080273
:108EB000AA423FF474AFBEF1000F3FF460AF165802
:108EC000F6798E421CBF0133314602F10802AA42F4
:108ED0007FF455AF63E703F10103314602F1080265
:108EE000AA427FF44CAF5AE72DE9F0414FF0010060
:108EF000FCF7A4FC4DF23440C0F60300FCF722FB63
:108F000040F64C73C2F200034FF001021A7040F6B3
:108F1000D060C2F20000016841B940F6D064C2F2EC
:108F20000004FEF745FF2568002DFAD040F61D77B6
:108F3000C2F2000740F64C74C2F2000440F66866C4
:108F4000C2F2000640F64075C2F2000540F6CC6859
:108F5000C2F200083B783BB14FF000023A704FF08C
:108F600002002070FCF764FC317859B14FF0000327
:108F70003370227862F07F0020704FF001000146CC
:108F8000FFF7A8FD297851B14FF000002870237831
:108F900003F07F0222704FF00101FFF79BFD98F86C
:108FA000000010B9FEF704FFD4E740F64C71C2F29E
:108FB00000014FF002030B704FF00000FCF73EFC85
:108FC000BDE8F08108B540F6D063C2F20003186036
:108FD00040F61470C2F200000068FEF71BFF08BDE7
:108FE00070B505460E4640F66473C2F20003186879
:108FF000032801D9F7F722FC40F66472C2F200029E
:10900000116840F6AC64C2F2000444F8316004EB2D
:10901000C104656001F10101116070BD70B50546C4
:109020000C461646032801D9F7F708FC40F62073D2
:10903000C2F2000353F8350008B1F7F7FFFB40F622
:109040002071C2F2000141F8354001EBC5056E60A8
:1090500040F61873C2F200031A6802F101021A60A6
:10906000206930B1FCF76EFA04F10404206900288D
:10907000F8D170BD08B540F60843C2F20003196884
:1090800081425AD040F60842C2F20002D36C8342B9
:1090900034D040F60841C2F20001D1F89820824253
:1090A0002FD040F60843C2F20003D3F8E410814207
:1090B0002AD040F60842C2F20002D2F83031834290
:1090C00025D040F60841C2F20001D1F87C2182424D
:1090D00020D040F60843C2F20003D3F8C811814201
:1090E0001BD040F60842C2F20002D2F8143283428A
:1090F00016D0F7F7A3FB4FF0080013E04FF0010084
:1091000010E04FF002000DE04FF003000AE04FF0D6
:10911000040007E04FF0050004E04FF0060001E016
:109120004FF0070040F60841C2F200014FF04C0238
:1091300002FB001090F8200008BD4FF00000F1E79E
:109140002DE9F04F8FB0089007910A924FF000037D
:1091500009931360546813891B1B8B4238BF079314
:109160000799002900F04A81082C69D840F6187444
:10917000C2F20004D4F800E040F66475C2F20005C3
:109180002E680EEBCE0707EBC60404F109044FF07E
:10919000000140F62077C2F20007CB598BB1DD68A1
:1091A000641903F110051B695BB15E890EB104F10E
:1091B00007049B890BB104F1070455F8043F002B09
:1091C000F3D101F108012029E7D140F6D061C2F2C4
:1091D00000010D682F7E6E7EEB8A03F10103C3F35D
:1091E00047054FF000010C914FF009038DF82C302A
:1091F0004FF002018DF82D10ADF82E408DF830E0C3
:109200004FF001018DF831104FF0000167F3451167
:1092100066F3861161F07F018DF833108DF83450BC
:109220000093019007A8029002F10400114609AAD8
:109230000BABFFF705FD079A002A00F0DD80E0E0A8
:109240004FF009001060DCE05BF83640002C00F0C5
:10925000CE80059D286800284BD07A68B2420CD099
:109260004FF0000310F0010F3ED1DFE007EBC30227
:109270005268B24240F0E38001E04FF0000357F83B
:109280003300D2B290F8048090F805C090F806E060
:10929000C579016819B143F01000C3B201E04FF085
:1092A00000034FF008008DF82C004FF00B018DF8F3
:1092B0002D108DF82E208DF82F808DF830C08DF870
:1092C00031E08DF832508DF833300A990090089AC9
:1092D000019207AB029301F1040009AA0BABFFF75F
:1092E000AFFC079828B987E003F101052B468542BA
:1092F000BCD104F1100523697BB129464FF000026F
:10930000588908B102F101029B890BB102F10102F7
:1093100051F8043F002BF3D101E04FF000025FFA57
:1093200086FCD2B294F804E06079A17923681BB17D
:1093300046F02003DBB201E04FF000038DF82CA0D3
:109340004FF004088DF82D808DF82EC04FF0000CE2
:109350008DF82FC08DF830208DF831E08DF8320077
:109360008DF833108DF834300A99CDF800A0089AA2
:10937000019207A8029001EB080009AA0BABFFF7C6
:109380005FFC0799002937D0A3686BB10A99E2689E
:1093900000920898019007AA029201EB080009AA1E
:1093A000FFF74EFC079B3BB3246904B34FF0010861
:1093B0004FF000092046FFF75DFE8DF8350061890A
:1093C00039B10DF11C0C40462246FFF775FC079998
:1093D00091B1A18939B10DF11C0C48462246FFF725
:1093E0006BFC079840B155F8044F002CE2D106F110
:1093F0000106042E7FF428AF099814E04FF0FF30E7
:1094000011E04FF0000640F6207BC2F2000B40F660
:109410006474C2F2000405944FF0090A40F6AC6788
:10942000C2F2000710E70FB0BDE8F08F03F10103AF
:1094300007EBC3014A68B2427FF456AF1FE705F15C
:10944000010307EBC3014A68B2427FF44DAF16E750
:1094500008B540F65073C2F200031A5C40F60841AA
:10946000C2F200014FF04C0000FB0210436AD3F13E
:10947000010238BF002242634FF00001C163016462
:10948000416400F11000FCF72FFB08BD2DE9F84FF7
:1094900081468A4640F65073C2F200031A5C40F6D9
:1094A0000840C2F200004FF04C0404FB020404F137
:1094B00048064FF001084FF0000740F6D46BC2F2A7
:1094C000000B354640463146F7F7BCF930B14FF056
:1094D00002003146F7F7B6F9BDE8F88FBAF1000F90
:1094E00005D148464146FBF759FF032827D0256C94
:1094F00075B15846A168E26BA8470546B0F1FF3F39
:1095000014D06064484659462A46FBF76DFF0EE0CA
:10951000616CA5688D4228BF0D464846E16B2A461E
:10952000FBF762FFE36B5A19E26300E03D46606CB3
:10953000A16888423CBFE7632764451B65643846E1
:109540003146F7F77FF90228BBD0BDE8F88F00BF9E
:10955000F8B505460E46174640F65073C2F20003B2
:109560001A5C40F60840C2F200004FF04C0404FBC5
:1095700002044FF00000FBF769FEE76326644FF03A
:109580000001616428464FF00101FFF77FFF4FF0B3
:109590000100FBF75BFEF8BDF8B505460F46164621
:1095A00040F65073C2F200031A5C40F60840C2F263
:1095B00000004FF04C0404FB0204A168B1420DD23C
:1095C00043F65C03C2F200039F4207D344F25C02FD
:1095D000C2F20002974201D2F7F730F94FF00000D3
:1095E000FBF734FEE7634FF0000020646664284612
:1095F0004FF00101FFF74AFF4FF00100FBF726FE95
:10960000F8BD00BF08B5FBF777FF08BD70B586B0A1
:1096100005460C46164602A8F8F7BCFB01462EB1DB
:1096200002A82A46234600F0A5FD07E04FF00103FB
:10963000009302A82A46234600F04EFE06B070BDF5
:1096400070B58AB00378212B00F0938004D86BB1F9
:10965000012B40F0D88186E0A12B00F0A781C02B20
:1096600000F0B481802B40F0CE8195E0417805294F
:1096700003D0092940F0CA8146E0408840F64C7288
:10968000C2F200021378022B02D0032B33D118E070
:1096900000F1FF318AB27E2A30D8C0B240F6607342
:1096A000C2F2000318704FF00201FCF731F840F6E7
:1096B0004C70C2F200004FF0030101704FF0010046
:1096C000C3E170B940F66072C2F20002107040F659
:1096D0004C70C2F200004FF0020303704FF0010023
:1096E000B3E17F280DD840F66071C2F20001087026
:1096F0004FF00100A9E14FF00200A6E14FF0020097
:10970000A3E14FF00200A0E1827840F64C73C2F270
:1097100000031978022923D972B940F64C73C2F2BA
:1097200000034FF0030119704FF001000146FFF7ED
:10973000D1F94FF0010088E1012A18BF022040F062
:10974000848140F64C70C2F200004FF004020270B7
:109750004FF000000146FFF7BDF94FF0010074E142
:109760004FF0020071E140780B280CBF012002206D
:109770006BE18388032B00F24C8140F62074C2F227
:10978000000404EBC3035B68002B00F0458198479D
:10979000002808BF022058E142781AB1062A40F09A
:1097A0003E8121E0C18802291BD14FF00000ADF8B5
:1097B000040040F6D062C2F2000212680346517EF5
:1097C00061F30003ADF80430127E62F341030AA98D
:1097D00021F8243D4FF00202FFF7DEFE4FF00300B8
:1097E00033E14FF0020030E18278C1888CB2C37857
:1097F000022B2ED0032B3DD0012B40F0D48040F61D
:109800006C65C2F2000528464DF25841C0F60301CE
:109810004FF0120210F0ACFB40F6D060C2F2000034
:1098200001688A892A81CB896B81088AA8818A7C10
:109830002A71CB7C6B71097DA9714FF0000029461C
:10984000122C34BF22461222FFF7A6FE4FF003006F
:10985000FBE040F66872C2F2000211814FF0000096
:10986000506049F24111C0F60201FFF771FE4FF05E
:109870000300EAE0D2B940F66C64C2F2000404F1DD
:1098800002004DF25441C0F603014FF0020210F005
:109890006FFB4FF0040222704FF0030565704FF02C
:1098A00000002146FFF778FE2846CEE0012A06D1C7
:1098B00040F6D063C2F20003196809682FE0022A5B
:1098C00006D140F6D062C2F200021068416826E07C
:1098D000032A06D140F6D063C2F2000319688968F2
:1098E0001DE002F00F0022F00F03102B08D15A4B9D
:1098F000196888420EDA594A52F8300001680EE0C1
:10990000202B07D1032805D8554951F8300008B15C
:10991000016804E0EE2A04D04FF0020095E009B996
:109920003EE05049B1F1FF3F40F0888001A84FF080
:1099300020014FF00102FFF769FE0AAD2A184FF02F
:10994000000002F8240C01A978E000F10206428030
:1099500003F10102134611F8015F5DB100F104004B
:10996000758002F1010311F8012F002A6FD101E087
:109970004FF0000340F66C61C2F200014FF00305A6
:109980004D7003F101034FEA4303DAB20A704FF05E
:109990000000A24228BF2246FFF7FEFD284654E001
:1099A0004FF0020051E04FF002004EE08388032B9D
:1099B00038D840F62074C2F2000404EBC3035B689D
:1099C0009BB39847002808BF02203EE04378212B34
:1099D0002ED1C18840F66873C2F2000319814FF09E
:1099E00000025A608088042825D1104648F621518B
:1099F000C0F6020140F66872C2F20002FFF7A8FD4D
:109A00004FF0030021E04FF002001EE04FF0020093
:109A10001BE04FF0020018E04FF0020015E04FF09D
:109A2000020012E04FF002000FE04FF002000CE0E5
:109A30004FF0020009E04FF0020006E00A78002A29
:109A400096D009484FF000037FE70AB070BD1E2B87
:109A50007FF47BAF8EE700BF640F0020AC0E0020C8
:109A6000200F002048D403086C0E002010B50446D7
:109A7000436993B14FF00000606140F64C71C2F24F
:109A800000010A78032A08D140F66073C2F200038D
:109A900018784FF00301FBF73BFE206958B34FF0F5
:109AA00000002061E06040F61C71C2F20001087005
:109AB00040F64471C2F200014FF00802FFF7A2FD28
:109AC000082853D140F64472C2F20002137813F012
:109AD000800F06D140F64470C2F20000C188002910
:109AE00044D140F64470C2F200004FF000010A4633
:109AF000FFF7A6FD2DE0E168002937D04FF0000008
:109B0000E06040F61C72C2F20002137840F66C610D
:109B1000C2F20001C3F14002FFF774FD034628B30F
:109B200040F61C70C2F2000001785A18D2B20270DE
:109B300040F64473C2F20003D888904216D140F632
:109B40004470C2F2000040F66C61C2F20001FFF7FF
:109B500077FD012804D0022808D1FBF72FFC10BDA7
:109B60004FF0000001460246FFF716FD10BD00BF92
:109B700008B540F67473C2F200031B693BB14FF0A5
:109B8000000140F67472C2F200025269984740F632
:109B90007470C2F200004FF00001017041608160FA
:109BA000C1600161416108BD40F67470C2F20000FD
:109BB00081614DF28C41C0F603018A5C4277837764
:109BC000037F6FF3070303774FF000014162704793
:109BD00030B583B040F67474C2F200042070089D62
:109BE0006560099DA5600A9DE5600B9D25610C9D42
:109BF00065619DF8184000949DF81C400194FFF7A2
:109C0000D3FF03B030BD00BF40F67473C2F200034F
:109C10005B6AB3F1FF3F09D140F67471C2F20001F3
:109C20004FF000034B624FF0010070473F2B0BD801
:109C300040F67472C2F20002106AC15403F10103CB
:109C400053624FF0010070474FF00000704700BFB3
:109C5000704700BF70B540F67474C2F2000404F19E
:109C600018004DF2E041C0F603014FF0070210F07A
:109C70007FF94FF000004DF2E841C0F60301FFF715
:109C8000AFF949F6C966C0F602064FF000004DF282
:109C90009041C0F603013246FFF7C0F94DF2F0459E
:109CA000C0F603054FF0010029463246FFF7B6F92A
:109CB0002869FFF7DFF984F8280040F6A070C2F2A7
:109CC00000004FF0070149F6D942C0F602024FF0FA
:109CD0000003FBF7E9FE70BD38B541F25403C2F250
:109CE00000034FF001021A7040F67474C2F20004CF
:109CF00094F828004FF000010A46FFF74DFC606819
:109D000068B140F67474C2F200044FF0FF3565622A
:109D10006368207861699847616A0029F7D040F646
:109D20007470C2F200004FF000024262836833B1E7
:109D300040F67471C2F2000108784969984738BD4D
:109D40002DE9F04F83B0804643680BB9806828B195
:109D50004FF00001C8F80810FFF7BEFFD8F80C203C
:109D6000002A45D04FF00003C8F80C30D8F80000A6
:109D700041F21401C2F200014FF04002FFF742FC31
:109D8000814640F67470C2F20000C16800292FD0ED
:109D9000B9F1000F2CD040F67474C2F2000441F205
:109DA0001406C2F200064FF0000509F1FF3B0BF06C
:109DB000010B2078715D2A466369E768B84705F1B1
:109DC000010AD14570D113E0207816F80A102A460E
:109DD0006369E768B8470AF1010A207816F80A10A3
:109DE0002A466369E768B8470AF1010AD145EBD111
:109DF000D8F81420002A54D04FF0000441F2540344
:109E0000C2F200031C70C8F8144040F6F070C2F2B1
:109E10000000FEF733FD40F67470C2F200004462A9
:109E20004168002936D040F67475C2F2000540F64C
:109E3000B074C2F200042C622C46656A6268207815
:109E400061699047636A9D42F7D11DB3D8F800005D
:109E500040F6B071C2F200012A46FFF79DFB4FF0B9
:109E600000000090019040F6F070C2F200004FF048
:109E70004B014FF0FF0249F6D943C0F60203FEF74B
:109E8000B7FD0EE040F67472C2F20002107851691C
:109E9000984706E040F67471C2F200018B68002B0F
:109EA000F0D103B0BDE8F08FBBF1000F8CD020786B
:109EB00016F80A102A466369E768B8470AF1010AEA
:109EC000D14581D194E700BF10B544780378212BA8
:109ED00002D0A12B1BD10EE0202C04D0222C14BFC9
:109EE0000020012010BD072A14D10D4810F040F8C1
:109EF0004FF0010010BD212C0FD14FF00000084998
:109F00004FF00702FFF748FB4FF0030010BD4FF082
:109F1000000010BD4FF0020010BD4FF0000010BD5A
:109F20008C0F002008B541F25403C2F200031878E8
:109F300070B940F67471C2F200014A6A72B940F613
:109F40007473C2F2000393F82800FFF781FA08BD8A
:109F500040F6A070C2F20000FBF7C6FD08BD00BFCE
:109F60004DF21C50C0F60300704700BF70B4037878
:109F700001298CBF4478002402298CBF85780025F4
:109F8000DCF8000048B34FEA93064DF24C50C0F69F
:109F90000300365C16704FEA031343EA141303F010
:109FA0003F031B5C5370012907D94FEA840444EA3C
:109FB000951303F03F04205C01E04FF03D009070EA
:109FC000022907D905F03F054DF24C53C0F60303B3
:109FD000E95C01E04FF03D01D17070BC704700BFFB
:109FE00082B04FF015010CE00191019B03F1FF32AB
:109FF000019233B100BF019B03F1FF320192002BAC
:10A00000F8D100F1FF30B0F1FF3FEDD102B0704761
:10A0100070B4C4B24FEA10204DF2E056C0F6030609
:10A020004DF2E065C0F6030511F8013B1AB94BB9D2
:10A0300044EA00200BE06340F45C4440E85C013AF1
:10A04000F2D1F5E76340F45C4440E85CECE770BCB7
:10A05000704700BF10B444F6FB43C0F2861311F8FA
:10A06000014B02B9ACB380EA04404FEA400010F063
:10A07000807F18BF58404FEA400010F0807F18BF23
:10A0800058404FEA400010F0807F18BF58404FEA18
:10A09000400010F0807F18BF58404FEA400010F099
:10A0A000807F18BF58404FEA400010F0807F18BFF3
:10A0B00058404FEA400010F0807F18BF58404FEAE8
:10A0C000400010F0807F18BF5840002AC7D0013AE6
:10A0D000C5D120F07F4010BC704700BF82B0019016
:10A0E0009DF806304FF0000063F307009DF805204F
:10A0F00062F30F209DF8042062F317409DF80720BB
:10A1000012F0800F14BF63F07F0103F07F0161F351
:10A1100007004FEA4201CAB262F31F6013F0800FDA
:10A1200018BF42F0010262F31F6002B0704700BF27
:10A1300084B0C0F307438DF80C30C0F307228DF8CC
:10A140000D20C3B24FEA10604FEA500210F0010F29
:10A1500014BF63F07F0103F07F018DF80E1013F040
:10A16000800F18BF62F07F028DF80F20039804B0B3
:10A17000704700BF2DE9F04F83B005460F461446E7
:10A180001E46019201F1FF3313F1050F44D8032E4F
:10A1900043D9A6F10400C0F380080DF1040C284651
:10A1A000FFF7E4FE05F10305A7F1030104F1040440
:10A1B000A6F10406A7F1040717F1050F67D92CE0F3
:10A1C0000DF1040C284639462246FFF7CFFE05F173
:10A1D000030B5D46A7F1030104F1040A5446A6F1FE
:10A1E00004094E46A7F1040717F1050F15D80F46CD
:10A1F0000DF1040C58465246FFF7B8FE0BF103056B
:10A20000A7F103010AF10404A9F10406A7F1040867
:10A2100018F1050F59D900E0FFE799B396B30DF196
:10A22000040C28466A46FFF7A1FE022E11D0032E29
:10A2300002D0012E26D11AE0019929B19DF8002003
:10A2400022704FF0010301E04FF0000304F101041C
:10A2500001E04FF00003019830B102A9CA1812F8CA
:10A26000080C207003F1010304F1010401E04FF038
:10A270000003019921B102AAD31813F8080C207029
:10A2800004F101040199601A03B0BDE8F08F0F4694
:10A29000032EC2D9B8F1000F92D00DF1040C28465C
:10A2A0002246FFF763FE05F10305A7F1030104F160
:10A2B0000404A6F10406A7F1040717F1050FACD8B2
:10A2C0000F46032E3FF67CAFA7E7A7F10307032E47
:10A2D0003FF676AFA1E700BFF0B49DF81040ECB1B7
:10A2E0004FEA41079F421CD2DD1B1DD056194FF08B
:10A2F00030046FEA0203F31803F0010302F8014B84
:10A30000B24240F0928007E0134603F8014B5470CC
:10A3100003F10102B242F7D13B4607E04FF00005DE
:10A3200004E04FF0000501E04FF0000500293CD0AB
:10A3300003F1FF34002B3AD000F101034118284605
:10A34000521B04F1FF3515F0020F10D032E0A4F1DA
:10A35000020603F101031F46012C29D03446B446FE
:10A3600013F8016C4FEA1616092E42D944E01E4636
:10A3700013F8015C4FEA1515092D8CBF37353035C0
:10A38000155414B900F1010012E013F8016C06F045
:10A390000F05092D8CBF373530351618757000F153
:10A3A000020528468B42D2D102E0284600E028462A
:10A3B000F0BC70471E4613F8015C4FEA1515092DD5
:10A3C00094BF303537351554002CDBD013F8016CB1
:10A3D00006F00F05092D94BF303537351618757006
:10A3E00000F102008B42E3D003F10103A4F1020467
:10A3F000BDE706F1300601E006F137065655BCF11F
:10A40000000FBFD013F8016C06F00F06092E94BFA1
:10A41000303637361018467005F102008F42C7D02B
:10A4200003F10103A4F10204A1E7002B3FF46CAF98
:10A4300002F8014BB2427FF467AF6DE7DCF81430ED
:10A4400093F8452083F84420DCF8141091F8463046
:10A4500081F84530DCF8141091F8472081F8462047
:10A46000DCF8143083F84700704700BFDCF8143084
:10A4700093F8470093F8462083F84720DCF814103F
:10A4800091F8453081F84630DCF8141091F84420FA
:10A4900081F84520704700BF43F21822C2F2000243
:10A4A000136840F20001C0F60101C85CC918497880
:10A4B00003F10203136041EA00207047DCF8043026
:10A4C000DCF8082002EBD300CCF8080003F0070109
:10A4D0004FF0010303FA01F2CCF80420704700BFEB
:10A4E0002DE9F04F83B004468A4693461E46CDF8C8
:10A4F00004C04FF00007B846B9463DE02546304657
:10A50000D047034600283DD0B9F1000F0CD12028D8
:10A5100029D0092829D00A2829D00D2829D0022D90
:10A520004FF0010988BF0225A3F13002D1B20929F9
:10A5300010D9A3F14100C1B2052903D8A3F1370313
:10A54000D9B207E0A3F16102D0B205281AD8A3F16D
:10A550005703D9B24FEA0717FCB241EA040708F1E2
:10A5600001082C4606E02C4604E02C4602E02C466E
:10A5700000E02C463046D847FF2CBFD004F1FF3511
:10A58000002CBCD1DDF804C03846FFF757FF019B13
:10A590005A69D8F1010838BF4FF0000882F850809E
:10A5A00003B0BDE8F08F00BF43F2E403C2F2000342
:10A5B0001B684B634BB19A68824209D0DB684B63DE
:10A5C0001BB19A688242F9D102E04FF01E00704739
:10A5D0004FF00000704700BF884204D8884234BF63
:10A5E0000220002070474FF001007047D0F804317E
:10A5F000D0F80021934214BFC05C0020704700BF18
:10A60000D0F80431FF2B14BF01330023C0F804310C
:10A61000704700BF10B4DCF81420D16C0B46044620
:10A6200058B14FEA016343EA116301F47F4043EA02
:10A63000002301F47F0143EA1123DCF8040030B168
:10A6400099B24FEA134060F30F0361F31F435CB903
:10A650004FEA036141EA136103F47F4041EA0021BC
:10A6600003F47F0341EA1323D36410BC704700BF97
:10A67000DCF80030FA2B05D841F26002C2F2000289
:10A68000D05C70474FF00000704700BFDCF800302E
:10A6900003F10103CCF80030DCF8140090F85120ED
:10A6A00002F1010280F85120704700BF70B40446E7
:10A6B0000846A1B199188C4211D22518AA420ED28F
:10A6C00094423ABFC4EB0206F6B20026A94205D274
:10A6D0000019821AD31AF118C8B200E0304670BCD3
:10A6E000704700BFF0B583B043F2BC03C2F2000371
:10A6F0004FF00C021A7043F26400C2F200000468CA
:10A700003CB3154643F2BC07C2F200074FF0000607
:10A7100021680B6873B10DF107000DF10601984730
:10A720009DF807009DF8061032463B78FFF7BEFF04
:10A730004519EDB26468002CEAD143F2BC02C2F2C2
:10A7400000021078A84204D243F2BC01C2F2000118
:10A750000D7043F2BC03C2F200034FF00A025A70BC
:10A7600043F2D404C2F2000424683CB3154643F219
:10A77000BC07C2F200074FF000062068036873B1FF
:10A780000DF107000DF1060198479DF807009DF8AF
:10A79000061032467B78FFF789FF4519EDB26468F1
:10A7A000002CEAD143F2BC01C2F200014A78AA426D
:10A7B00004D243F2BC00C2F20000457043F2BC0375
:10A7C000C2F200034FF00201997043F2B404C2F2E6
:10A7D000000424683CB30D4643F2BC07C2F20007F4
:10A7E0004FF000062268136873B10DF107000DF1F8
:10A7F000060198479DF807009DF806103246BB7881
:10A80000FFF754FF4519EDB26468002CEAD143F21A
:10A81000BC00C2F200008178A94204D243F2BC021B
:10A82000C2F20002957043F2BC03C2F200034FF083
:10A830000100D87043F21C24C2F2000424683CB327
:10A84000054643F2BC07C2F200074FF0000621683C
:10A850000A6872B10DF107000DF1060190479DF8ED
:10A8600007009DF806103246FB78FFF71FFF4519D9
:10A87000EDB26468002CEAD143F2BC03C2F20003DB
:10A88000D878A84204D243F2BC01C2F20001CD70D4
:10A8900003B0F0BD43F21023C2F20003196840F286
:10A8A0000000C0F60200401A704700BF034610B116
:10A8B00082688A4218D043F2B803C2F200031868D3
:10A8C00060B182688A4203D10BE083688B420AD070
:10A8D00040680028F9D14FF0000305E04FF0000375
:10A8E00002E0034600E003461846704710B540F208
:10A8F000A064C1F200044FF4117303FB0044D4F8C8
:10A900000811B1F1FF3F03D0D4F8042191420DD1D9
:10A9100023689A6A4FF0FF019047002834D0D4F89A
:10A92000080100F10100C4F8080110BD91422BD8C4
:10A930006318197943F2A802C2F2000213787BB9B6
:10A94000FD290FD923689A6A4FF0FE019047D8B1CC
:10A9500043F2A800C2F200004FF00101017010BDE7
:10A960006FEA01012268936AC9B2984760B1D4F8CE
:10A97000080100F10100C4F8080143F2A801C2F285
:10A9800000014FF000020A7010BD00BF70B506460E
:10A9900040F2A065C1F200054FF4117404FB00F40D
:10A9A0002B194FF00101C3F80C112A5993699847EC
:10A9B0002859016A3046884770BD00BF38B540F25B
:10A9C000A061C1F200014FF4117202FB00F28C1879
:10A9D000D4F80831D4F80451AB420DD08958E318AB
:10A9E0008A6A1979904738B1D4F80801FF2814BF52
:10A9F00001300020C4F8080138BD00BF38B540F26E
:10AA0000A064C1F200044FF4117202FB00F2A3181B
:10AA1000D3F80451D3F808118D4206D14FF000014C
:10AA2000C3F80C11A2589369984738BD10B440F28E
:10AA3000A063C1F200034FF4117202FB003000F575
:10AA40008870D0F80031FF2B14BF5A1C0022D0F8B8
:10AA50000441A2421CBFC154C0F8002110BC704781
:10AA6000F8B543F21024C2F2000424688568C76870
:10AA7000466807FB05604518611911D2CE180B48CE
:10AA8000864210D8012B04D1635D13704FF0000093
:10AA9000F8BD10461A460FF06BFA4FF00000F8BDF3
:10AAA0004FF01F00F8BD4FF01F00F8BD0100020875
:10AAB00010B543F26003C2F200031A8840F2A060AE
:10AAC000C1F200004FF4117404FB0204F5F70CFF0F
:10AAD0004FF0FF31C4F810124FF00003C4F81832E1
:10AAE00004F58874F5F70AFF10BD00BFF8B50646F7
:10AAF0004FF00203037044F20000C0F60000C28B66
:10AB00004FF6FF718A4221D03F4C404BA34222D2E4
:10AB100003F110033E4DEF1A4FEA17124FF6FF757F
:10AB200002F1010002F001071C46D98BA9424FD166
:10AB300015E01C46D98BA94211D002F1010203F1A4
:10AB400010031C46D98BA94257D108E044F20004F7
:10AB5000C0F6000403E044F20004C0F600044FF61F
:10AB6000FF7021464FF00D02FFF752FA4FF6FF73C8
:10AB7000984208BF0020E28982421BD0A4F1100550
:10AB800044F20000C0F6000085421AD34FF6FF7071
:10AB900029464FF00D02FFF73BFA4FF6FF7188424E
:10ABA00008BF002034F8024C84420AD12C464FF0F2
:10ABB000010201E04FF00002607BFF2806D13270F5
:10ABC00004E04FF0020333704FF000042046F8BD5C
:10ABD0004FF0000202F1010203F110038242BED0E5
:10ABE000002FA6D01C46D98BA942B8D002F1010291
:10ABF00003F1100382429CD1B1E702F1010203F19B
:10AC00001003824295D1AAE70080000800400008A6
:10AC10000F80000870B5C0B005460E4620F0FF0456
:10AC2000684621464FF04002F8F782FB00AB53FA2A
:10AC300085F031464FF010020FF09AF96846214630
:10AC40004FF48072F8F7C8FC40B070BD38B50546C7
:10AC500040F2A064C1F200044FF4117303FB0044FE
:10AC6000D4F81C02FDF718FB43F26000C2F20000AA
:10AC70000188A94206D143F26003C2F200034FF6F5
:10AC8000FF721A804FF00000C4F81C0238BD00BFEC
:10AC900010B54FF00000FAF77FFF43F26403C2F2F1
:10ACA00000031C6834B12068016901B188476468F9
:10ACB000002CF8D110BD00BF10B50446072827D8D6
:10ACC000032894BF4FF4FA73322303FB01F140F2DF
:10ACD000A063C1F2000303EBC000C0F8141969B10E
:10ACE000FDF7BCFE002808BF012040F2A063C1F2BE
:10ACF000000303EBC404C4F8100910BD40F2A061C6
:10AD0000C1F2000101EBC4044FF00002C4F81029A5
:10AD100010BD00BF38B50446072851D840F2A063E3
:10AD2000C1F2000303EBC000D0F8145935B340F270
:10AD3000A061C1F2000101EBC402D2F81039EBB1FD
:10AD4000FDF78CFE002808BF012040F2A061C1F28F
:10AD5000000101EBC402D2F81039C01A85420CD2AE
:10AD600040F2A065C1F2000505EBC4014FF00005FB
:10AD7000C1F81459C1F8105900E02D1A05F1040565
:10AD80004CF6CD42CCF6CC42A2FB05234FEA930011
:10AD9000032C0AD800F1630348F21F51C5F2EB11EE
:10ADA000A1FB03324FEA521038BD00F109014CF605
:10ADB000CD42CCF6CC42A2FB01304FEAD00038BDE8
:10ADC0004FF0000038BD00BF70B506466446DCF8A1
:10ADD00014305D6AFDF742FE6169CA6A0AB9C86249
:10ADE00008E0801A05EB850506FB05F6B04224BF96
:10ADF0000020C8626369D96AD1F1010038BF002020
:10AE000070BD00BF10B540F2A063C1F200034FF463
:10AE1000117404FB003303F58873D3F80841002C48
:10AE20005FD15AB14FF0FF31C3F8001143F2202334
:10AE3000C2F200034FF00000187010BDD3F80021DB
:10AE4000B2F1FF3F06D1FF294BD14FF00002C3F80A
:10AE5000002110BDFF291ED143F22021C2F20001C2
:10AE60004FF000040C70012A10D94FF00102C3F812
:10AE7000082140F2A063C1F200034FF4117101FBFD
:10AE80000030D0F81C02FCF7C5FF10BD4FF00000E9
:10AE9000C3F8000110BDFE2907D143F22023C2F2FE
:10AEA00000034FF00101197010BD43F22020C2F2DF
:10AEB0000000007848B16FEA0101C9B243F22020D6
:10AEC000C2F200004FF000040470FF2A05D8995424
:10AED00002F10102C3F8002110BD4FF0FF32C3F8A8
:10AEE000002110BD08B540F2A063C1F200034FF489
:10AEF000117202FB0030D0F80811D0F8043100F1D3
:10AF0000040099420AD94FF00002C0F8002143F230
:10AF1000E800C2F200004068FCF77CFF08BD00BFFB
:10AF2000F8B5654643F21423C2F200031A7802F022
:10AF30000804E7B227B1DCF8146096F8516007E026
:10AF400012F0110F06BFDCF8147097F8526000265B
:10AF500001EB800411F8203003F0070302F0200217
:10AF6000D7B23FB111F8202002F00807FAB20AB1B7
:10AF70004FEA430311F820704FEA9712012A08D0D4
:10AF8000022A10D111F82000C0F3011101FB06675D
:10AF90000BE06F6997F8517011F82020C2F301108F
:10AFA00000FB077701E04FF00007042B50D8DFE8E3
:10AFB00013F0C60140003B002200050043F21821B7
:10AFC000C2F200010B6840F20007C0F60107FA1850
:10AFD00092F802E0D0784FEA006040EA0E405278E2
:10AFE00040EA0220FF5C03F104030B603843FFF7E3
:10AFF0009FF868602CE043F21822C2F20002136846
:10B0000040F20000C0F60100C11891F801C0C05C18
:10B010004FEA004040EA0C208978084303F103031B
:10B0200013603F186F6013E0FFF736FAC2196A60C9
:10B030000EE043F21823C2F20003186840F2000148
:10B04000C0F601010A5CBF186F6000F101001860D2
:10B05000637803F0070343F21420C2F20000017882
:10B0600001F02002D7B237B1607800F00801CAB20F
:10B070000AB14FEA430367784FEA9710012807D0D7
:10B0800002280ED16178C1F3011202FB06670AE0C3
:10B090006F6997F851006178C1F3011202FB000754
:10B0A00001E04FF00007042B50D8DFE813F048010F
:10B0B00040003B002200050043F21821C2F20001CB
:10B0C0000B6840F20007C0F60107FA1892F802E098
:10B0D000D0784FEA006040EA0E40527840EA022001
:10B0E000FF5C03F104030B603843FFF721F8A8600D
:10B0F0002CE043F21822C2F20002136840F2000072
:10B10000C0F60100C11891F801C0C05C4FEA0040D0
:10B1100040EA0C208978084303F1030313603F18C9
:10B12000AF6013E0FFF7B8F9C219AA600EE043F26E
:10B130001823C2F20003186840F20001C0F60101B2
:10B140000A5CBF18AF6000F101001860A37803F03B
:10B15000070343F21420C2F20000017801F020023C
:10B16000D7B237B1A07800F00801CAB20AB14FEAED
:10B170004303A7784FEA9710012807D002280ED181
:10B18000A178C1F3011202FB06670AE06F6997F824
:10B190005100A178C1F3011202FB000701E04FF05A
:10B1A0000007042B50D8DFE813F0CA0040003B0032
:10B1B0002200050043F21821C2F200010B6840F2A0
:10B1C0000007C0F60107FA1892F802E0D0784FEABB
:10B1D000006040EA0E40527840EA0220FA5C03F137
:10B1E00004030B601043FEF7A3FFE8602CE043F27A
:10B1F0001822C2F20002136840F20000C0F60100FB
:10B20000C11891F801C0C05C4FEA004040EA0C2030
:10B210008978084303F1030313603F18EF6013E0DC
:10B22000FFF73AF9C219EA600EE043F21823C2F2BE
:10B230000003186840F20001C0F601010A5CBF1863
:10B24000EF6000F101001860E37803F0070343F2B8
:10B250001420C2F20000017801F02002D0B230B117
:10B26000E17801F00802D0B208B14FEA4303E17877
:10B270004FEA9112012A02D0022A0FD108E06E692A
:10B2800096F85100E278C2F3011101FB000607E0D5
:10B29000E078C0F3011101FB066601E04FF0000603
:10B2A000042B4CD8DFE803F04B031318300043F2B3
:10B2B0001823C2F20003186840F20001C0F6010131
:10B2C0000A5CB6182E6100F101001860F8BDFFF7A6
:10B2D000E3F882192A61F8BD43F21822C2F2000293
:10B2E000136840F20000C0F60100C1184C78C05C41
:10B2F0004FEA004040EA04208978084303F1030341
:10B30000136036182E61F8BD43F21821C2F2000115
:10B310000B6840F20004C0F60104E2189678D07879
:10B320004FEA006040EA0640527840EA0220E25CC0
:10B3300003F104030B601043FEF7FAFE2861F8BD29
:10B3400010B58AB0044601A8F6F788FD039B237068
:10B35000029860700199A170079A1AB102F1FF304A
:10B36000C3B201E04FF00603E3704FF0010101FAB0
:10B3700003F222710AB010BD70B582B00546124CBE
:10B3800004EB80066846FFF7DBFF9DF8002014F809
:10B3900025309A4212D19DF80100717888420DD172
:10B3A000B2789DF804301A4208D0F078D0F101004C
:10B3B00038BF00204FF00101F17002E04FF00000B3
:10B3C000F07002B070BD00BFF00F001008B5032888
:10B3D0001ED8DFE800F0020910174DF61C10C0F669
:10B3E000030010F0B5FB08BD4DF62010C0F60300B9
:10B3F00010F0AEFB08BD4DF63410C0F6030010F09F
:10B40000A7FB08BD4DF64C10C0F6030010F0A0FBE2
:10B4100008BD00BF2DE9F8430546884616461F467D
:10B4200043F26003C2F20003B3F8009043F25850B5
:10B43000C2F20000016843F2A402C2F200021368E3
:10B44000994201D0FFF734FB072D6ED81F2E6CD820
:10B4500040F2A064C1F200044FF4117000FB0944F3
:10B4600043F2E800C2F200004FF00001FCF722FABC
:10B47000217965F34711072D14BF00250125AA196D
:10B4800062F304012171CBB22DB184F805804344ED
:10B490004FF0020001E04FF0010006F1FF3E5FFABD
:10B4A0008EFE46B302463F1A0EF0010C3D5C04F1DD
:10B4B000040635545B1902F101020EF1FF31C9B2E5
:10B4C000FF2934D114E0BD5C04F10406B5545B19C6
:10B4D00002F1010201F1FF3101F0FF01BD5CB55441
:10B4E0005B1902F1010201F1FF31C9B2FF29EAD172
:10B4F00000F1010070442218137100F10100C4F83A
:10B5000004014FF0FF33C4F8083121680B6A43F29D
:10B510006000C2F2000000789847FCF749FC43F253
:10B52000E800C2F20000FCF7D3FABDE8F8834FFA56
:10B530008CF5002DC7D0BD5C04F10406B5545B1931
:10B5400002F1010201F1FF31C9B2FF29BBD1CFE7FE
:10B5500010B586B00DF10700FFF7C8FA044618B120
:10B560009DF8073023B90FE044F20004C0F6000450
:10B57000E2894FF6FF7082422BD048F20001C0F6FC
:10B5800000018C4209D32AE0304821464FF00D02D9
:10B590000EF098F8002848D0EAE74FF6FF7248F21C
:10B5A0000000C0F600006FEA0403C118C1F30011E7
:10B5B00004F11004E389934239D10AE004F1100345
:10B5C0001C46D989914204D003F11004E3899342C7
:10B5D00039D148F20002C0F60002944207D344F287
:10B5E0000004C0F6000420462146F7F789FF02A8B0
:10B5F00016494FF00D020EF0BBFC4FF0FF008DF826
:10B6000015004FF6FF7002A94FF00D02FEF700FD86
:10B610004FF6FF71884212BFADF816000021ADF859
:10B620001610204602A9FFF7F5FA06B010BD8442B5
:10B63000D5D20029C2D004F11004E1899142C8D0CA
:10B640008442BBD3CBE78442B8D3C8E7661000205E
:10B650002DE9F04F85B0884691461D46E2464FF0F1
:10B66000000426464FF0020B2DE007462846C0474F
:10B67000034670B324B9202822D0092802D11FE044
:10B68000012C05D12B2B0DD02D2B0DD05C4601E0CC
:10B69000022C01D12E2B09D0A3F13002D0B20928FF
:10B6A00017D805E05C4603E05C4601E04FF0030478
:10B6B0000E2E05D804A98A1902F8103C06F10106DD
:10B6C0002846C8473846FF28CFD000F1FF3700286A
:10B6D000CCD1012C12D98EB104ACA6194FF00004C4
:10B6E00006F8104C684621460EF046F8DAF81410B9
:10B6F000C864DAF8142082F8504005E0DAF8143013
:10B700004FF0010083F8500005B0BDE8F08F00BF96
:10B7100010B5044643F26800C2F20000FCF7D8F905
:10B72000F6F772FEFAF7DEFA08B1FBF701FF2046E2
:10B73000FCF706FD43F26800C2F200004FF0000182
:10B74000FCF7B8F810BD00BF10B586B040F200009D
:10B75000C0F601003449F7F7D3FE00284BD1334B34
:10B76000334A9A421DD240F20001C0F601010B6833
:10B77000B3F1FF3F42D102F104032E4AD01A20F068
:10B780000302991812F0040F3FD118468B420CD0D7
:10B7900003F104021B68B3F1FF3F3ED04FF00000FD
:10B7A00031E040F20000C0F6010040F20003C0F6B4
:10B7B0000203984225D10DF10700FFF797F90446DF
:10B7C000B0B19DF80710022912D002A821464FF00F
:10B7D00010020EF0CDFB9DF815006FF307008DF8F9
:10B7E0001500204602A9FFF715FA4FF001000AE004
:10B7F0004FF0010007E04FF0000004E04FF00000C0
:10B8000001E04FF0000006B010BD184603F104033C
:10B810000268B2F1FF3FB8D0C0E702F1040310683C
:10B82000B0F1FF3FB1D0B9E7FFFF01080000020807
:10B8300000000108030002082DE9F0070346002874
:10B840004ED040F20022C0F6000292F8469092F8E4
:10B85000470043F2BC04C2F2000494F8018092F85D
:10B8600048C0257843F2D802C2F200021468177A61
:10B87000567AD2F804A04FF000021A7083F80190B3
:10B880009870DA704FF0FB0018714FF0060983F8DA
:10B8900005909D7183F807804FF0040883F80880B5
:10B8A00083F8098083F80AC0DD721A734FEA142501
:10B8B0005D739C73DF731E745A744FF01D029A748B
:10B8C0004FF00202DA744FF0FE021A755A754FEA11
:10B8D0001A229A7583F817A018764FF01F00587631
:10B8E00029B143F2BC03C2F200031A680A60BDE842
:10B8F000F0077047034628B143F2D802C2F20002B3
:10B900001068186043F2D801C2F20001087A70474B
:10B9100070B505460E4614464FF000002946FEF766
:10B92000C5FF08B1F4F78AFF43F2B803C2F200037F
:10B930001A686260A56026601C6070BD08B539B1E8
:10B9400043F26403C2F200031A68426018601EE00A
:10B9500043F26403C2F200031B6883420FD15868AC
:10B9600043F26401C2F20001086010E042685A60CC
:10B9700041605A688242F9D013461BB907E033B1DF
:10B980004FF000015A688242F0D01346F5E7FEF707
:10B99000A9FE08BD08B539B143F2D403C2F20003D1
:10B9A0001A68426018601EE043F2D403C2F200033A
:10B9B0001B6883420FD1586843F2D401C2F20001E0
:10B9C000086010E042685A6041605A688242F9D0CB
:10B9D00013461BB907E033B14FF000015A688242A9
:10B9E000F0D01346F5E7FEF77DFE08BD08B539B186
:10B9F00043F2B403C2F200031A68426018601EE00A
:10BA000043F2B403C2F200031B6883420FD15868AB
:10BA100043F2B401C2F20001086010E042685A60CB
:10BA200041605A688242F9D013461BB907E033B12E
:10BA30004FF000015A688242F0D01346F5E7FEF756
:10BA400051FE08BD08B539B143F21C23C2F2000310
:10BA50001A68426018601EE043F21C23C2F2000321
:10BA60001B6883420FD1586843F21C21C2F20001C7
:10BA7000086010E042685A6041605A688242F9D01A
:10BA800013461BB907E033B14FF000015A688242F8
:10BA9000F0D01346F5E7FEF725FE08BD01604360D0
:10BAA000826043F2E403C2F200031A68C2601860C5
:10BAB000704700BF70B582B006464FF000038DF8A6
:10BAC00007300D4601B10B7043F26400C2F2000072
:10BAD000046874B121684B6843B130460DF1070129
:10BAE0002A46984710B19DF8070013E06468002CBF
:10BAF000F0D10B2E05DC0C2E03D83046FAF790F867
:10BB000008E02DB14FF005022A704FF0000001E06F
:10BB10004FF0000002B070BD70B582B006464FF025
:10BB200000038DF807300D4601B10B7043F264003D
:10BB3000C2F20000046874B121688B6843B13046DA
:10BB40000DF107012A46984710B19DF807001BE048
:10BB50006468002CF0D10B2E0DDC0C2E0BD8304677
:10BB6000FAF774F88DF8070010B13046FAF7B4F818
:10BB70009DF8070008E02DB14FF005022A704FF044
:10BB8000000001E04FF0000002B070BD70B582B05F
:10BB900006464FF000038DF807300D4601B10B70DB
:10BBA00043F26400C2F20000046874B12168CB68FB
:10BBB00043B130460DF107012A46984710B19DF870
:10BBC000070013E06468002CF0D10B2E05DC0C2E6E
:10BBD00003D83046FAF70AF808E02DB14FF0050215
:10BBE0002A704FF0000001E04FF0000002B070BD7D
:10BBF00070B582B006464FF000038DF807300D4651
:10BC000001B10B7043F2D400C2F2000004685CB1D1
:10BC100021688B682BB130460DF107012A46984701
:10BC200058B96468002CF3D1092E0CDC0A2E0AD80E
:10BC30003046F5F7C9FC8DF807009DF80700003085
:10BC400018BF012008E02DB14FF006022A704FF016
:10BC5000000001E04FF0000002B070BDF0B583B00D
:10BC600005460E464FF000038DF8073043F2D4002E
:10BC7000C2F200000468E4B14FF000072168CA680E
:10BC80001AB1284631469047F0B923689B6833B112
:10BC900028460DF106010DF10702984700E03846ED
:10BCA0009DF8071099B9646814B10028E6D004E043
:10BCB00018B9092D0DDC0A2D0ED82846314607F09B
:10BCC000A9F84FF0000009E04FF0000006E0084638
:10BCD00004E04FF0060001E04FF0060003B0F0BDB5
:10BCE00070B582B005460E464FF000038DF8073060
:10BCF00012B11946FFF7B2FF43F2D400C2F20000BE
:10BD000004686CB121684B68284631460DF1070282
:10BD1000984710B19DF8070012E06468002CF1D13B
:10BD2000092D08DC0A2D09D828463146F5F76EFCA6
:10BD30004FF0000004E04FF0060001E04FF0060075
:10BD400002B070BD08B54FF0000001464FF001028F
:10BD5000FFF7C6FF08BD00BF70B582B005460E46AE
:10BD60004FF000038DF8073043F2B400C2F2000038
:10BD700004689CB121684B68284669460DF10702AA
:10BD8000984728B10EB1009830609DF8070014E084
:10BD900064681CB19DF80720002AEBD0012D07D85C
:10BDA0004EB12846F6F7B6FD30604FF0000004E0D3
:10BDB0004FF00F0001E04FF0000002B070BD00BF77
:10BDC00070B582B005460E464FF000038DF807307F
:10BDD00043F21C20C2F20000046884B121684B6861
:10BDE000284631460DF10702984710B19DF807002B
:10BDF00010E064681CB19DF80720002AEED03DB920
:10BE00004FF000003146F6F767FC4FF0000001E00C
:10BE10004FF00E0002B070BD70B582B005460E4600
:10BE20004FF000038DF8073043F21C20C2F20000EF
:10BE30000468A4B121688B685BB1284669460DF19E
:10BE40000702984728B10EB1009830609DF80700AE
:10BE500014E064681CB19DF80720002AEAD045B9B7
:10BE600056B14FF00000F6F779FD30604FF000005A
:10BE700004E04FF0060001E04FF0000002B070BD9A
:10BE80002DE9F04F2DED048B8BB083469246914205
:10BE900064D289464FF000089FED379A9FED328BB0
:10BEA000DFED369A32A7D7E900674FF000044FF074
:10BEB0000005C3F6E0758DED019ABBF1020F05D1C7
:10BEC0005FFA89F001A9FFF7A7FF04E05FFA89F0A4
:10BED00001A9FFF741FF08EB48030AAAD01800F8B0
:10BEE000209C01980CF05CF953EC182B0CF0D0FC62
:10BEF00008B1CDED019A01980CF052F932463B465B
:10BF00000CF0ECFA22462B460CF0A4F90CF00EF9DA
:10BF100081B208EB48030AAAD31803F81E1C4FEAA3
:10BF2000112003F81F0C08F10108B8F10A0F06D020
:10BF30000AF1FF3149450DD1B8F1000F0AD008EBE5
:10BF400048024FF007005946D2B202ABFFF762FA3F
:10BF50004FF0000809F10109CA45ACD80BB0BDEC9F
:10BF6000048BBDE8F08F00BF9831CB64FE0F7040AA
:10BF70000000000000E06F4000000000F37F8043FD
:10BF80002DE9F04F9FB040F6C410FCF7D9F84FF000
:10BF900002004FF0000143F2BC03C2F20003DA7862
:10BFA000FFF76EFF4FF0010002904FF0000BDA46F2
:10BFB000D94607464CF6CD41CCF6CC4103914FF023
:10BFC0007D00FCF7BDF88DF83790C8464E464C46CC
:10BFD00013E045F0800504F10804E4B216A9725C90
:10BFE000AA4202D016ABF554B84606F101069DF8F8
:10BFF0003750002D50D1202E4ED020460DF1370164
:10C00000FFF758FD051C18BF012504F10102D0B24D
:10C010000DF13701FFF74EFD10B145F00205EDB20D
:10C0200004F10203D8B20DF13701FFF743FD08B167
:10C0300045F0040504F10300C0B20DF13701FFF72C
:10C0400039FD08B145F0080504F10401C8B20DF14D
:10C050003701FFF72FFD08B145F0100504F1050287
:10C06000D0B20DF13701FFF725FD08B145F02005ED
:10C0700004F10603D8B20DF13701FFF71BFD08B13B
:10C0800045F0400504F10700C0B20DF13701FFF79C
:10C0900011FD00289DD19EE7B8F1000F02D1BAF141
:10C0A000000F0CD14FF002004946F2B216ABFFF779
:10C0B000B1F94FF03200FCF743F8019701E0CDF8F9
:10C0C00004908DF83790C8464E464C4613E045F034
:10C0D000800504F10804E4B20EA8315CA94202D044
:10C0E0000EAAB554B84606F101069DF83750002D4A
:10C0F00050D1202E4ED020460DF13701FFF778FDAC
:10C10000051C18BF012504F10100C0B20DF1370173
:10C11000FFF76EFD10B145F00201CDB204F102024D
:10C12000D0B20DF13701FFF763FD08B145F004050A
:10C1300004F10303D8B20DF13701FFF759FD08B13F
:10C1400045F0080504F10400C0B20DF13701FFF716
:10C150004FFD08B145F0100504F10501C8B20DF11D
:10C160003701FFF745FD08B145F0200504F106024F
:10C17000D0B20DF13701FFF73BFD08B145F04005A6
:10C1800004F10703D8B20DF13701FFF731FD0028A4
:10C190009DD19EE7B8F1000F02D1BAF1010F0AD18B
:10C1A00048464946F2B20EABFFF734F94FF0320081
:10C1B000FBF7C6FF019743F2BC03C2F200039A7873
:10C1C000B2B1039EA6FB0A044FEA141000EB8001F3
:10C1D000BAEB810F0CD138464946FFF751FE4FF0BC
:10C1E0003200FBF7ADFFBBF1000F40F0B88003E079
:10C1F000BBF1000F40F09C8005A849464FF020029B
:10C200000DF0DAFE43F2BC06C2F20006B478ACB31D
:10C210004D466FEA0900011901F0010209F0070318
:10C2200007FA03F69DF8140046EA00018DF8141091
:10C2300005F10105A542C0F2B3801FE01EAB03EB80
:10C24000D50605F0070007FA00F216F8641C42EA6A
:10C25000010306F8643C05F101051EA800EBD502B8
:10C2600005F0070107FA01F312F8646C43EA0600CF
:10C2700002F8640C05F10105A542DFDB4FF0070071
:10C280004FF011014FF01E0205ABFFF7C3F84FF05E
:10C290003200FBF755FF05A849464FF020020DF08C
:10C2A0008BFE43F2BC04C2F20004E578A5B34B4612
:10C2B0006FEA0902511901F0010609F0070007FAB7
:10C2C00000F49DF8142044EA02018DF8141003F1E3
:10C2D00001039D4250DC1FE01EAC04EBD30203F0CF
:10C2E000070007FA00F612F8641C46EA010402F897
:10C2F000644C03F101031EAA02EBD30403F0070010
:10C3000007FA00F614F8641C46EA010204F8642CEB
:10C3100003F101039D42DFDC4FF007004FF01201F3
:10C320004FF01E0205ABFFF775F84FF0060B16E055
:10C33000019AA2B9BBF1020F11D1029D7DB943F25E
:10C34000BC03C2F20003DA784AB14FF0020049465A
:10C35000FFF796FD4FF03200FBF7F2FE0297BAF1BD
:10C36000000F06D10BF1FF3BCDF808904FF0280AE3
:10C3700025E60AF1FF3A22E6002EADD01EAE06EB0E
:10C38000D30403F0070007FA00F214F8641C42EA31
:10C39000010604F8646C03F101039D429CDCBBE7D9
:10C3A000002A3FF44BAF1EAA02EBD50305F00706A7
:10C3B00007FA06F013F8641C40EA010203F8642C43
:10C3C00005F10105A542FFF639AF57E72DE9F04F1A
:10C3D0002DED028B87B008EE100A0C4617469946E1
:10C3E000129E1399B5EEC08AF1EE10FA54BF0025E3
:10C3F0000125A84604F1FF33D8B2082807D8092A36
:10C4000005D8A24601F1FF32944205D808E001F1B7
:10C41000FF339C4240F2CD8001F1FF34E4B2C8E02A
:10C4200018EE100A0CF0ACFA48B930464FF03F0154
:10C4300022460DF0C1FD4FF000013155C4E018EE69
:10C44000100A0CF0A1FF06EE900AF2EE047AF4EE68
:10C45000E76AF1EE10FA0DDB4FF00100B0EE677AFB
:10C4600000F1010067EE877AF4EEE76AF1EE10FA68
:10C47000F6DA03E04FF00100F2EE047A21464319A8
:10C48000A34200F39680C0EB040EC5EB0E0202F14E
:10C49000FF3E4DF6040AC0F6030ADFED9C4AF6EEB5
:10C4A000003AB2EE044AC0EB040CC5EB0C0303F0F7
:10C4B000010BBEF1000F00F38F808AE0BEF1000F88
:10C4C00004DDBE45B4BF72463A4601E04FF00002BB
:10C4D0005AF8223003EE103AB8EE430A20EE027A00
:10C4E000B4EEE47AF1EE10FA48BF37EE237ABDEEEF
:10C4F000C73A13EE10CABCFBF3FB06EE10BAB8EE57
:10C50000C65AB4EEE75AF1EE10FA0DDB00F1010C59
:10C5100087EE006A67EE847A0EF1FF3E6046BEF158
:10C52000000200F3C380BEE013EE105AB5FBF3F433
:10C5300003FB14542CB916EE107A002F08BF4FF0ED
:10C540000008B9F1000F07D0C8EB0103181A002A40
:10C5500018BF0138831A01E04FF0000301F1010117
:10C56000B8F1000F04D04DF67017C0F6030703E0D2
:10C570004BF6D847C0F6030722B14DF67410C0F64B
:10C58000030003E04BF6D840C0F603004DF68815D3
:10C59000C0F60305009501978DED026A03900492A1
:10C5A000059430464DF67812C0F603020DF0CEF831
:10C5B0000AE03046002D0CBF2B212D2122460DF024
:10C5C000FBFC4FF00000305507B0BDEC028BBDE81E
:10C5D000F08F4FF0000203E0BE45B4BF72463A460A
:10C5E0005AF8223000EE103AB8EE405A65EE260AAC
:10C5F000F4EEE40AF1EE10FA48BF70EEA30ABDEEC5
:10C60000E03A13EE10CABCFBF3FC06EE10CAF8EEDB
:10C61000C65AF4EEE75AF1EE10FA85DB00F101009C
:10C6200080EE852A67EE847A0EF1FF3E4219914230
:10C63000BFDBBBF1000F3FF441AFBEF1000F02DCE6
:10C640004FF0000203E0BE45B4BF72463A465AF8C6
:10C65000223001EE103AF8EE411A21EE822AB4EEB1
:10C66000E42AF1EE10FA48BF32EE232ABDEEC23AB8
:10C6700013EE10BABBFBF3FB06EE10BAF8EEC62AB7
:10C68000F4EEE72AF1EE10FAFFF64EAF00F10100EA
:10C6900082EE212A67EE847A0EF1FF3E4319994219
:10C6A000BFF60CAF85E74FF0000202E0BA42A8BF28
:10C6B0003A465AF8223006EE903AF8EE660A20EE34
:10C6C000861AB4EEE41AF1EE10FA48BF31EE231ADE
:10C6D000BDEEC13A13EE10BABBFBF3FB06EE10BA87
:10C6E000F8EEC65AF4EEE75AF1EE10FAFFF61CAF78
:10C6F0000CF1010081EE202A67EE847A0EF1FF3EF4
:10C7000042199142BFF6DAAE53E700BF0000004B7A
:10C71000F8B505460F46F4F7E7F8064640F2A06282
:10C72000C1F200024FF4117303FB05F01418115805
:10C7300011B18A682846904784F820724FF00005AE
:10C74000C4F81052C4F81452C4F80451C4F8085183
:10C750003046F4F7D3F804F5097029464FF0080283
:10C76000F4F77CF8F8BD00BF70B588B0054640F21C
:10C77000A064C1F200044FF4117303FB004494F869
:10C78000200200284AD043F26001C2F200010A8868
:10C790004FF6FF76B24204D0D0B24FF00401FFF75B
:10C7A000B7FF28464FF00001FFF7B2FF43F26006E3
:10C7B000C2F2000635804DF69410C0F603004FF02B
:10C7C000070142F21122C0F60302FBF77BFCC4F81A
:10C7D0001C02246830784FF0010300934FF00002F0
:10C7E00001924AF6ED01C0F6020102914AF6E563B4
:10C7F000C0F6020303934AF60561C0F602010491F4
:10C800004AF64D43C0F602030593069264684FF45E
:10C8100016514FF00803A047FEF74AF908B070BD63
:10C82000704700BF08B5B0F1FF3F04D040B90246E1
:10C83000F6F7C2F808BD4FF000000246F6F7BCF864
:10C8400008BD00BF38B506F0D9FA43F2C003C2F202
:10C8500000034FF001021A704FF000042546E0B2C9
:10C8600029462A46FFF73CFA40B904F10104E0B238
:10C8700029462A46FFF734FA002867D04FF0FF30E8
:10C880004FF00001FFF7CEFF4FF000004FF0000126
:10C89000FFF796FA43F21C21C2F200010C6834B192
:10C8A0002368DA6802B190476468002CF8D143F23B
:10C8B000B800C2F2000004683CB121680B680BB1FB
:10C8C000A06898476468002CF7D1F9F7D1FEFEF70D
:10C8D000DFF940F2A062C1F2000292F820020428BF
:10C8E00006D028B14FF000004FF00401FFF710FF11
:10C8F00040F2A061C1F2000191F86434042B06D02B
:10C900002BB14FF001004FF00401FFF701FF40F29F
:10C91000A062C1F2000292F8A806042806D028B14D
:10C920004FF002004FF00401FFF7F2FE40F2A06169
:10C93000C1F2000191F8EC38042B06D02BB14FF076
:10C9400003004FF00401FFF7E3FE38BD04F10104DA
:10C95000B4F5807F83D191E738B5054643F2A4044E
:10C96000C2F200042068FBF797FC4FF0000323603D
:10C970008DB14DF6A410C0F603004FF007014CF640
:10C980009122C0F60202FBF79DFB43F2AC01C2F21A
:10C990000001086038BD43F2AC04C2F20004206814
:10C9A000FBF77AFC4FF000002060FAF70DFBFFF771
:10C9B00049FF0AF067FD43F26001C2F200010A88F4
:10C9C0004FF6FF739A4204D0D0B24FF00401FFF744
:10C9D0009FFE38BD70B543F2E800C2F200004DF68C
:10C9E000B411C0F60301FAF74DFF43F26003C2F23F
:10C9F00000034FF6FF721A8040F2A064C1F20004F7
:10CA00004FF0040684F820624FF00005C4F81C5271
:10CA10002846FBF771F9206084F86464C4F8605418
:10CA20004FF00100FBF768F9C4F8440284F8A866E7
:10CA3000C4F8A4564FF00200FBF75EF9C4F888046E
:10CA400084F8EC68C4F8E8584FF00300FBF754F999
:10CA5000C4F8CC0643F26800C2F200004DF6C011E3
:10CA6000C0F60301FAF70EFF43F2C400C2F2000061
:10CA70004EF28071C0F603012A462B46FFF70EF8EE
:10CA8000FDF730FE4FF00100FFF766FF70BD00BFFD
:10CA90002DE9F04F2DED048BABB01CAF26AC4DF261
:10CAA000E075C0F6030595E80F0084E80F00A76065
:10CAB0004AF27163C0F60203E36020462AA9F7F741
:10CAC0007BFB22AE95E80F0086E80F00B7604AF2C4
:10CAD0008D60C0F60200F06030462146F7F76CFB2F
:10CAE0004FF000041B9443F26800C2F2000021469C
:10CAF000FAF7E0FE43F2D801C2F200010C72FFF730
:10CB0000A1FE0AF0BFFC4FF00200FFF72DFE43F23A
:10CB10001822C2F2000215680DBB0FF009F8F0B937
:10CB2000F5F732F910F0C20F19D14FF00300FEF7FC
:10CB30004DFC4FF47A754FF032063046FBF700FBA0
:10CB4000F5F762FC05F1FF343046FBF7F9FAF5F72B
:10CB50005BFC651EF1D14FF00000FEF737FC43F29D
:10CB60001423C2F200034FF000041C604FF00100D8
:10CB7000187040F2A066C1F2000606F51965284655
:10CB8000214642F654220DF017FA41F26000C2F23B
:10CB9000000021464FF400520DF00EFA06F5116028
:10CBA00021464FF040020DF007FA43F21410C2F292
:10CBB000000021464FF0FC020DF0FEF921954FF0E8
:10CBC0000A01C6F8B41920462946FDF7EDFC43F2E8
:10CBD000A002C2F20002146043F2B003C2F20003EA
:10CBE0001C6043F21825C2F200054FF030042C609F
:10CBF00040F20004C0F6010494F82F0000F1010097
:10CC000094F82E1000EB0122101943F21023C2F207
:10CC100000031860FBF722FF0A902B68E15CFF29F4
:10CC200030D143F2D800C2F200004FF0010101728E
:10CC30000360219A106A18B100F1010052F8203007
:10CC400043F2D801C2F200014B604FF0FF024A727A
:10CC500043F2AC00C2F200004FF00003036043F265
:10CC60006001C2F20001088840F2A062C1F2000235
:10CC70004FF4117303FB0021D1F81C02FBF7CAF833
:10CC800005F08DBA06F098F84FF000070997BA46FC
:10CC90003C4601E04FF000042CB94FF00000FEF7D5
:10CCA00037FD4FF0640404F1FF3443F21426C2F25E
:10CCB0000006357805F0E7026FF34512327043F253
:10CCC0001820C2F200000368089343F21826C2F24B
:10CCD000000640F20007C0F6010743F21428C2F232
:10CCE00000084DF6EC39C0F6030931687D5C01F1AE
:10CCF0000101316098F8002012F0010F0ED10AF105
:10CD0000010A40F2FF30824508D943F2D803C2F24B
:10CD100000034FF03601197205F0F9B90DF1700CEE
:10CD200028464946FEF7FCF84EF23C33C0F60303B2
:10CD300053F825004DF6EC7BC0F6030B40F00101E3
:10CD4000084730683A5C0B9200F1010030600F2A0E
:10CD500005F2D5810DF1700C10465946FEF7E0F84A
:10CD60004DF63033C0F603030B9953F82100E5E785
:10CD700030683A5C0B9200F101003060102A02D951
:10CD8000154605F0BDB90DF1700C0B984EF23C71D3
:10CD9000C0F60301FEF7C4F84DF6A833C0F603034E
:10CDA0000B9953F82100C9E73268B85C0B9002F187
:10CDB000010232600F2802D9054605F0A1B90DF134
:10CDC000700C0B984EF65C11C0F60301FEF7A8F844
:10CDD0004EF2EC13C0F603030B9953F82100ADE7B4
:10CDE00030683A5C0B9200F1010030602F2A02D9C2
:10CDF000154605F085B90DF1700C0B984EF22C110B
:10CE0000C0F60301FEF78CF84EF28C73C0F60303F4
:10CE10000B9953F8210091E730683A5C0B9200F1CE
:10CE2000010030603B2A02D9154605F069B90DF1C1
:10CE3000700C0B984DF62C01C0F60301FEF770F84C
:10CE40004DF64023C0F603030B9953F8210075E714
:10CE50003268B85C0B9002F1010232603F2802D9BF
:10CE6000054605F04DB90DF1700C0B984EF69C116E
:10CE7000C0F60301FEF754F84EF22C03C0F603038C
:10CE80000B9953F8210059E730683A5C0B9200F196
:10CE900001003060432A02D9154605F031B90DF181
:10CEA000700C0B984EF22C21C0F60301FEF738F8F7
:10CEB0004EF64C03C0F603030B9953F821003DE7EF
:10CEC000219F97F846600DF1700CFDF7CFFA219D78
:10CED000331895F8502002F0010158181C9085F87D
:10CEE0004700FF2894BF0020012085F85000D3E6BA
:10CEF000219F97F846600DF1700CFDF7B7FA3518D1
:10CF00001C95219B83F84750FF2D94BF00250125D8
:10CF100083F85050C0E60DF1700CFDF7A7FA30B160
:10CF2000219A92F84700011C18BF012101E04FF03F
:10CF30000001219F87F84710AEE60DF1700CFDF758
:10CF400095FA219E96F84750284086F84700A3E6B8
:10CF50001D9BA3F1FB031C9319E11D99A1F1FB019A
:10CF60001C91A1E11D9AA2F1FB021C92D2E11D9835
:10CF7000A0F1FB001C906EE21D9EA6F1FB061C9624
:10CF80004FF002031B9306E21D99A1F1FB011C91D6
:10CF90001E9A1B9230E21D98A0F1FB001C902AE122
:10CFA0001D9EA6F1FB061C96ACE21D9BA3F1FB03A4
:10CFB0001C93E8E21D9FA7F1FB071C971E991B918C
:10CFC00025E31D9AA2F1FB021C921E981B904FF0C4
:10CFD00000068DF86A60D3E31D9BA3F1FB031C934D
:10CFE0001E991B914FF001028DF86A20C8E31D982D
:10CFF000A0F1FB001C9000F060BC1D9DA5F1FB059D
:10D000001C9500F0B5BC9DF874004FF00101FEF7CF
:10D0100025FE8DF86B0000283FF43EAE43F2D804A5
:10D02000C2F20004207205F072B81D9E1C964FF0EB
:10D0300001038DF86A301E46219991F8472013426A
:10D0400005D09DF870003146FEF708FE68B99DF8DE
:10D050006A304FEA43008DF86A001C9901F1010122
:10D060001C9110F0FE03E7D10CE09DF86A60012EE0
:10D0700008D19DF86B4043F2D802C2F2000214724C
:10D0800005F045B80DF1700CFDF7F0F904E69DF8D8
:10D09000740005F083FEFFE50DF1700CFDF7E6F975
:10D0A0001C9043F21823C2F200031E681C9906EB81
:10D0B00041021A60FDF7F0F91C9001F0DDBE43F269
:10D0C0001420C2F20000017811F0280F06D01D9B39
:10D0D000B3F5005F34BF0023012304E01D9BFA2B4E
:10D0E00094BF0023012343B143F2D804C2F20004E9
:10D0F0004FF01301217205F00AB841F26006C2F246
:10D1000000061D9AB05C1C90CBE7219B93F85260FF
:10D110001C96C6E7219A92F850001C90C1E74FF088
:10D12000000AB9E50DF1700CFDF7A0F91C90219FE4
:10D1300097F847101B91FDF74FFA87F84700ABE5CA
:10D14000219D95F8470095F84610FDF745FA85F8BA
:10D150005000A1E50DF1700CFDF7B0F91E9B41F2F6
:10D160006006C2F20006F05C1D9920EA0102F2544A
:10D1700092E543F21410C2F200004FF000014FF0AC
:10D18000FB020CF019FF87E54FF000031C930DF133
:10D19000A80C1CF8386DFDF769F90146304608F017
:10D1A00065FC8DF86B0000283FF476AD43F2D8049F
:10D1B000C2F20004207204F0AABF07F05DF86BE52C
:10D1C00007F062F88DF86B0000283FF465AD43F27C
:10D1D000D801C2F20001087204F099BF43F210278F
:10D1E000C2F200073D681D98281807F039F853E58A
:10D1F0004FF000021C921C9B40F2A066C1F2000698
:10D200004FF4117101FB036090F82022032A3FD1F3
:10D2100040F2A067C1F2000701FB03F303F5887633
:10D22000B919FB1803F104034FF00000D1F80021F5
:10D23000FE2A94BF551C0025D1F80471BD4214BFCD
:10D240000025012565F30000BA4214BF0022012227
:10D2500062F34100D3F80051FE2D94BF0135002543
:10D260000DF1A80C4CF8385DD3F80461B54214BF39
:10D270000025012565F38200D3F80811D1F10103DF
:10D2800038BF002363F3C300C0B2FDF7D7F803E54E
:10D2900043F2D804C2F200044FF04803237204F0B2
:10D2A00036BF4FF000001C901C9E40F2A062C1F2FD
:10D2B00000024FF4117101FB062393F820020328AA
:10D2C0001CD140F2A067C1F2000701FB0675D5F83A
:10D2D0001022D5F81412531AB3F5807F88BF03F5D6
:10D2E00080731C931C98FF2884BFFF201C900DF1B5
:10D2F000A80C1CF8380DFDF7A1F8CDE443F2D804D2
:10D30000C2F200044FF04806267204F000BF4FF04E
:10D3100000061C961C9B40F2A062C1F200024FF472
:10D32000117101FB032090F82062032E24D140F2FA
:10D33000A067C1F2000701FB037505F58876D6F8F2
:10D340000021D6F80411501AB0F5807F88BF00F58F
:10D3500080701C900DF1700CFDF788F88DF86A0054
:10D360001C9B984238BF1C90D6F804711C9DEA198A
:10D37000D1B2C6F804118FE443F2D804C2F200041B
:10D380004FF04803237204F0C2BE4FF000061C9613
:10D390004FF002001B901C9B40F2A062C1F2000201
:10D3A0004FF4117101FB032696F82002032815D1D2
:10D3B00040F2A067C1F2000701FB03750DF1700C8C
:10D3C0001B984AF2ED51C0F602014AF20162C0F622
:10D3D000020205F58873FDF783F85DE443F2D80493
:10D3E000C2F200044FF04803237204F090BE4FF0E5
:10D3F00000021C921D991B911C9E40F2A060C1F27C
:10D4000000004FF4117303FB060292F82012032967
:10D4100015D140F2A067C1F2000703FB06750DF1BC
:10D42000700C1B984AF2ED51C0F602014AF20162FB
:10D43000C0F6020205F58873FEF70AF92CE443F200
:10D44000D804C2F200044FF04806267204F05FBE12
:10D450004FF000001C901C9B40F2A062C1F2000241
:10D460004FF4117101FB032696F8200203283DD1E9
:10D4700040F2A067C1F2000701FB037505F588754E
:10D480000DF1700CFCF7F2FF8DF86A00D5F804215D
:10D490001C924FF000011B91D5F800711346974282
:10D4A00007D0AE5C864219D04FF001024FF0000E5B
:10D4B0000CE04FF0FF001B9010E002F10101EE5C68
:10D4C000864202D11C931B9208E00A46FF2B14BF30
:10D4D000013373469F42F0D11C93EAE70DF1700CC3
:10D4E0009DF86C00FCF7AAFFFFF7D6BB43F2D80407
:10D4F000C2F200044FF04803237204F008BE4FF05C
:10D5000000031C931C9E40F2A062C1F200024FF483
:10D51000117101FB062090F82032032B27D140F235
:10D52000A065C1F2000501FB065707F58875D7F81D
:10D530001462D7F81022964212D00DF1700CFCF74D
:10D5400095FF8319DFB21C970DF1700CE85DFCF7B5
:10D5500075FF4FF00005219E86F85050FFF79CBBE9
:10D560004FF00101219880F85010FFF795BB43F26E
:10D57000D804C2F200044FF04806267204F0C7BD7A
:10D580004FF000021C921C9840F2A063C1F200030D
:10D590004FF4117101FB003696F82022032A28D19E
:10D5A00040F2A067C1F2000701FB007505F588761F
:10D5B000D6F80431D6F800118B4213D00DF1700C5F
:10D5C000F05CFCF73BFFD6F80471FF2F14BF013766
:10D5D0000027C6F804714FF00005219E86F85050D0
:10D5E000FFF75ABB4FF00102219880F85020FFF757
:10D5F00053BB43F2D804C2F200044FF0480020723B
:10D6000004F085BD4FF000031C931D991B9143F25C
:10D610001022C2F20002D2F800801B9F08EB07061E
:10D6200040F20000C0F60200864208D943F2D80654
:10D63000C2F200064FF01F02327204F068BD1C9B5C
:10D64000032B08D943F2D801C2F200014FF0370092
:10D65000087204F05CBDF1780D2908D943F2D804B2
:10D66000C2F200044FF03703237204F050BD40F2C1
:10D67000A065C1F200054FF4117202FB035090F84F
:10D6800020323BB118F8071021B10FE04846FEF7F1
:10D690003FF805E04CF24F354FF09609DDF828B021
:10D6A000FBF7DCF9CBEB0002AA42EFD918F80770C0
:10D6B000032F3FF6F1AADFE807F002080F169DF8E6
:10D6C0007000FFF751F8FFF7E7BA9DF87000314698
:10D6D00008F0EEF9FFF7E0BA9DF87000314606F069
:10D6E00027FDFFF7D9BA9DF870504DF2F079C0F6DA
:10D6F000030996F8028008EB480809EB080728465A
:10D700004FF00301FFF704F84FF4117000FB05F32D
:10D7100040F2A061C1F20001C85800283FF4BCAA41
:10D72000F6784DF67032C0F6030252F8261019F85A
:10D7300008207B78BF7800974FF0000601964AF6E4
:10D74000BD17C0F6020702974AF6FD17C0F602079A
:10D7500003974AF62D27C0F6020704974AF64D476D
:10D76000C0F602070597069646682846B047FFF7B9
:10D7700093BA4FF000031C931D991B918DF86A30EA
:10D780001C9B40F2A060C1F200004FF4117101FB3C
:10D79000030696F82022032A79D140F2A065C1F24F
:10D7A000000501FB035707F5887943F21020C2F208
:10D7B00000000168219EB26B01EB020B885CFF2820
:10D7C0005CD0D8464FF001074FF0000B0894CDF81D
:10D7D0002CA0BA4698F8014004EB002343F2102035
:10D7E000C2F200000668F218D9F804111C919DF8E5
:10D7F0006A501DB1F75C02F1010200E05F4602F1E0
:10D80000FF349DF86A302BB177B9089C5546DDF896
:10D810002CA005E0607838B9089C5546DDF82CA0AE
:10D820001C99C9F804112BE01C99D9F800618E42AB
:10D8300018D014F8016F19F801501B9A3AB9304604
:10D840000BF028FFC6B228460BF024FFC5B2AE424B
:10D8500008D11C9BFF2B14BF01335B461C9307F1BF
:10D86000FF37CEE70AF1010A18F8020FFF28B1D1FD
:10D87000089CDDF82CA04FF0000501E04FF00005FA
:10D880000DF1700CE8B2FCF7D9FDFFF705BA43F2D1
:10D89000D804C2F200044FF04803237204F037BCEE
:10D8A0004FF000001C901E9E1B964FF001028DF859
:10D8B0006A2065E74FF000021C921C9E40F2A063B4
:10D8C000C1F200034FF4117000FB063191F82022E1
:10D8D000032A31D140F2A065C1F2000500FB0657D2
:10D8E00007F588750DF1700CFCF7C0FD8DF86A0026
:10D8F0004FF000031C93D5F80471D5F800118F4246
:10D9000012D0EA5D82420FD14FF00006FF2F14BF04
:10D91000013737468F4202D1C5F8047104E0EB5D50
:10D920008342F3D0C5F804710DF1700C4FF0000084
:10D93000FCF784FDFFF7B0B943F2D804C2F200044B
:10D940004FF04806267204F0E2BBFBF787F80A9D09
:10D95000401B0DF1700C4CF24F37B8428CBF0020C9
:10D960000120FCF76BFDFFF797B94FF000001C900A
:10D970001C9E40F2A062C1F200024FF4117101FB43
:10D98000062393F82052032D7FF486A940F2A06766
:10D99000C1F2000701FB067000F10406D0F808117F
:10D9A000D6F8002102F10102914238BF01F58071E1
:10D9B0008B1AFF2B34BF1D46FF250DF1700CE8B20A
:10D9C000FCF73CFDFFF768B91D9F41F26000C2F211
:10D9D0000000C65D06F1FF31C155FFF75DB943F2A6
:10D9E0001422C2F20002137813F0280F06D01D98FB
:10D9F000B0F5005F34BF0020012004E01D98FA2834
:10DA000094BF0020012040B143F2D804C2F20004C8
:10DA10004FF01301217204F07ABB1D9E41F26001A8
:10DA2000C2F200018A5D02F1FF33D8B288550028A6
:10DA30003FF432A91E9E1C9601F01EBA43F2142236
:10DA4000C2F20002137813F0280F06D01D98B0F52B
:10DA5000005F34BF0020012004E01D98FA2894BF25
:10DA60000020012040B143F2D804C2F200044FF07C
:10DA70001306267204F04BBB1D9E41F26001C2F2F8
:10DA800000018A5D02F1FF33D8B28855002842F0C8
:10DA90002087FFF701B943F21421C2F200010A788E
:10DAA00012F0280F06D01D9BB3F5005F34BF002392
:10DAB000012304E01D9BFA2B94BF0023012343B1F3
:10DAC00043F2D804C2F200044FF01300207204F0B5
:10DAD0001EBB1D9841F26006C2F20006315C01F1E6
:10DAE000FF32D3B23354002B02F0F386FFF7D4B8E1
:10DAF000219D95F8517007F1FF3685F85160FFF7C9
:10DB0000CBB8219991F8472002F1FF3381F84730D3
:10DB1000FFF7C2B82198C06C0BF036FC219DE86479
:10DB2000FFF7BAB8219F97ED137AD7ED127A37EE47
:10DB3000270A87ED130A2199C86C0AF001FF30B15A
:10DB40004FF00200219981F85000FFF7A5B8219EFF
:10DB5000F06C0AF005FF30B14FF00102219B83F811
:10DB60005020FFF799B84FF00007219D85F85070BD
:10DB7000FFF792B89DF87400219901F14C01FEF76E
:10DB8000EBF88DF86B0000283FF486A843F2D80428
:10DB9000C2F20004207204F0BABA9DF87400219E0B
:10DBA000F16CFEF70DF98DF86B0000283FF474A8B6
:10DBB00043F2D801C2F20001087204F0A8BA219A17
:10DBC000D06C0AF0CDFE20B9219B986C0AF0C8FEFB
:10DBD00030B14FF00302219B83F85020FFF75CB86F
:10DBE0002198D0ED138A90ED128A78EEC80A10EED3
:10DBF000900A0BF0C9FB09EE100A18EE900A18EE15
:10DC0000101A0BF03FF801464FF07E500BF03AF837
:10DC10009FEDCF1A01EE900A21EE812AB4EEC29A4E
:10DC2000F1EE10FA06D84FF00006219981F8506005
:10DC3000FFF732B8219DD5ED132A95ED123AF4EE97
:10DC4000C32AF1EE10FA05DD4FF0010785F8507098
:10DC5000FFF722B8F4EEC32AF1EE10FA4CBF02220D
:10DC6000032285F85020FFF717B82198D0ED133A1A
:10DC7000B7EE004A73EEC44AC0ED134A219EF06C21
:10DC80000AF06EFE30B14FF00305219B83F850502F
:10DC9000FFF702B82199D1ED138A9FEDAE8A38EED5
:10DCA000C89A19EE100A0BF06FFB09EE100A18EE75
:10DCB000900A18EE101A0AF0E5FF01464FF07E5068
:10DCC0000AF0E0FFDFEDA23A04EE100A64EE234A08
:10DCD000B4EEE49AF1EE10FA22D9219F97ED138A5F
:10DCE000DFED9C8A38EE285A15EE100A0BF04CFB3B
:10DCF00008EE900A18EE100A6FF052510AF0C2FFB7
:10DD000001464FF07E500AF0BDFFDFED915A06EE5E
:10DD1000100A66EE256AF4EEE68AF1EE10FA06D8ED
:10DD20004FF00407219A82F85070FEF7B5BF219A90
:10DD3000D56C28460BF028FB08EE100A28464FF059
:10DD400000010AF09FFF01464FF07E500AF09AFF53
:10DD5000DFED7F7A07EE100A27EE270AB4EEC08ABD
:10DD6000F1EE10FA06D84FF00006219981F85060C4
:10DD7000FEF792BF219BD3ED130AF5EEC00AF1EE38
:10DD800010FA05DD4FF0010083F85000FEF784BF64
:10DD9000F5EEC00AF1EE10FA4CBF0222032283F81E
:10DDA0005020FEF779BF219D95ED125AD5ED135AFB
:10DDB00085EE256A85ED136ABDE6219EF06C0AF0BA
:10DDC000BBFD002841F05680FEF766BF2199CE6C5E
:10DDD00030460BF0D9FA08EE100A30464FF0000139
:10DDE0000AF050FF01464FF07E500AF04BFFDFED86
:10DDF000586A07EE100A67EE267AB4EEE78AF1EE6B
:10DE000010FA01F33780FEF747BF219AD06C0AF071
:10DE100093FD002801F02E80FEF73EBF219B93ED7D
:10DE2000130AD3ED120AB4EEE00AF1EE10FA81F211
:10DE30002180FEF731BF219890ED131AD0ED121A10
:10DE4000B4EEE11AF1EE10FA01F31480FEF724BFEC
:10DE5000219991ED132AD1ED122AB4EEE22AF1EEC6
:10DE600010FA41F20780FEF717BF219E96ED133A94
:10DE7000D6ED123AB4EEE33AF1EE10FA00F1FA8779
:10DE8000FEF70ABF219AD66C30460BF07DFA08EEF9
:10DE9000100A30464FF000010AF0F4FE01464FF040
:10DEA0007E500AF0EFFE9FED2A4A04EE900A24EE1F
:10DEB000845AB4EEC58AF1EE10FA40F2DB87FEF721
:10DEC000EBBE219FF86CFCF709F9F8640DF1700CBA
:10DED0004FF00000FCF79EFBFEF7DEBE1D9BF62B0D
:10DEE00008D943F2D804C2F200044FF0120323729F
:10DEF00004F00DB9219DE86C0AF01EFD38B9219996
:10DF000091ED136AF6EE006A36EE268A06E0219855
:10DF100090ED138AF6EE005A38EE658A18EE100A74
:10DF20000AF00AFD00BB9FED0C7AB4EEC78AF1EE51
:10DF300010FA04DC18EE100A0AF002FDA0B14FF04E
:10DF40000106219F87F850606FF000463BE000BF5C
:10DF500000000034FFFF7F4BFEFFFF4AFEFFFFCAB9
:10DF600000008043000080C318EE100A0AF0E4FCB1
:10DF700098B15FED067AB4EEE78AF1EE10FA04D4B8
:10DF800018EE100A0AF0DCFC38B14FF001002199BC
:10DF900081F850004FF0004615E018EE100A0AF024
:10DFA000DFFC38B14FF00205219B83F850504FF051
:10DFB000000608E0BDEEC88A18EE106A4FF00007B0
:10DFC000219A82F850704FEA066242EA166506F41A
:10DFD0007F4345EA032006F47F0140EA112643F21D
:10DFE0001417C2F200071D9ABE50FEF755BE1D98C9
:10DFF000F62808D943F2D804C2F200044FF0120206
:10E00000227204F084B843F21415C2F200052E58AF
:10E010004FEA066141EA166706F47F4247EA0223A7
:10E0200006F47F0043EA102500EE105AF8EEC00A0D
:10E03000219EC6ED130A1FED381AF4EEC10AF1EE67
:10E0400010FA06DC5FED3B1AF4EEE10AF1EE10FA8D
:10E0500005D54FF0010786F85070FEF71DBE4FF052
:10E06000000186F85010FEF717BE0DF1700C4FF04E
:10E070000100FCF7CFFA219BD86CFCF759F8219DE1
:10E08000E864FEF709BE219890ED132AF7EE002A06
:10E0900032EE223A80ED133AF0E52198C06C0AF096
:10E0A0005FFC50B1219D4FF0000385F847304FF0E1
:10E0B000040085F85000FEF7EFBD219E96ED131A7F
:10E0C000B5EEC01AF1EE10FA23DB1FED5B3AB4EEA9
:10E0D000C31AF1EE10FA0FD5FCEEC13A13EE901A06
:10E0E0000DF1700CC8B2FCF7A9F94FF00007219AA6
:10E0F00082F85070FEF7D0BD0DF1700C4FF0FF00AC
:10E10000FCF79CF94FF00200219E86F85000FEF7C4
:10E11000C3BDB5EEC01AF1EE10FA7EF5BDAD5FEDF0
:10E120006F1AB4EEE11AF1EE10FA11DDB1EE412AE8
:10E13000FCEEC22A12EE902A0DF1700CD0B2FCF760
:10E140007DF94FF00105219B83F85050FEF7A4BDE7
:10E150000DF1700C4FF0FF00FCF770F94FF0030168
:10E16000219F87F85010FEF797BD43F21426C2F2A4
:10E170000006317811F0280F08D01D9A02F1010233
:10E18000B2F5005F34BF0022012206E01D9A02F1C1
:10E190000102FA2A94BF0022012242B143F2D804BC
:10E1A000C2F200044FF01303237203F0B0BF219FAB
:10E1B00097ED134AFDEEC44A14EE905A2BB21C930D
:10E1C00098B2C5F3072646EA002141F26002C2F286
:10E1D00000021D9FD153FEF75FBD43F21420C2F22F
:10E1E0000000067816F0280F08D01D9901F10101F2
:10E1F000B1F5005F34BF0021012106E01D9901F156
:10E200000101FA2994BF0021012141B143F2D80450
:10E21000C2F200044FF01302227203F078BF219D76
:10E2200095ED135AFCEEC55A15EE902A97B21C973D
:10E230004FEA172343EA072041F26006C2F20006C4
:10E240001D997052FEF728BD1D9D219FBD64FEF7EC
:10E2500023BD1D98219BD864FEF71EBD0DF1700CE7
:10E26000FCF704F906EE100AF8EE466A219EC6EDA8
:10E27000136AFEF711BD43F21421C2F200010A78BD
:10E2800012F0280F08D01D9800F10100B0F5005FD2
:10E2900034BF0020012006E01D9800F10100FA289B
:10E2A00094BF0020012040B143F2D804C2F2000420
:10E2B0004FF01303237203F02ABF41F26005C2F24C
:10E2C00000051D9FEB5B4FEA132646EA03218AB245
:10E2D00007EE902AB8EE670A219880ED130A9FEDA9
:10E2E000C97AB4EEC70AF1EE10FAFEF6D5ACDFED4E
:10E2F000C60A30EE601A80ED131AFEF7CDBC43F269
:10E300001426C2F20006317811F0280F08D01D9AA9
:10E3100002F10102B2F5005F34BF0022012206E0E3
:10E320001D9A02F10102FA2A94BF0022012242B191
:10E3300043F2D804C2F200044FF01300207203F03D
:10E34000E6BE41F26005C2F200051D9FE85B4FEAA0
:10E35000102343EA0026B1B201EE901AB8EE612A0A
:10E36000219A82ED132AFEF797BC1D98072808D939
:10E3700043F2D803C2F200034FF008061E7203F006
:10E38000C6BEFCF7C7FC02EE900AB8EE623A219DC9
:10E3900085ED133AFEF780BC219FD7ED133A97ED38
:10E3A000124A63EE844AC7ED134AFFF7C4BB2199B2
:10E3B00091ED135AF1EE455AC1ED135AFEF76CBCBC
:10E3C0004FF000004FF001010A46FDF789FC219A49
:10E3D00092ED136AF1EE046A66EE267A4FF00000C1
:10E3E0000090019043F22420C2F20000BCEEE70A44
:10E3F00010EE101A4FF0FF024BF64553C0F6020321
:10E40000FAF7F6FAFEF748BC43F21423C2F200030F
:10E410001E7816F0280F08D01D9901F10301B1F5FF
:10E42000005F34BF0021012106E01D9901F10301C5
:10E43000FA2994BF0021012141B143F2D804C2F26C
:10E4400000044FF01300207203F061BE41F260053A
:10E45000C2F200051D9FE859FBF76AFE219A9064FD
:10E46000FEF71ABC43F21423C2F200031E7816F022
:10E47000280F08D01D9901F10301B1F5005F34BFE9
:10E480000021012106E01D9901F10301FA2994BF41
:10E490000021012141B143F2D804C2F200044FF03F
:10E4A0001300207203F033BE41F26005C2F2000592
:10E4B0001D9FE859FBF73CFE219AD064FEF7ECBBA8
:10E4C0001D9B072B08D943F2D804C2F200044FF079
:10E4D0000806267203F01BBE219ED6ED130AF5EE48
:10E4E000C00AF1EE10FA0FDB9FED487AF4EEC70A8E
:10E4F000F1EE10FA08D8FCEEE01ACDED1C1A4FF040
:10E50000000586F8505021E09FED401AF4EEC10A54
:10E51000F1EE10FA07DD6FF07F431C934FF001011D
:10E5200086F8501012E04FF000011C9110EE900A96
:10E530000AF002FA28B14FF00202219880F8502028
:10E5400004E04FF00305219F87F850501D981C9957
:10E55000FCF7B2FBFEF7A0BB219FF86C0AF000FAB3
:10E5600000287EF499AB219890ED132AB5EEC02ACD
:10E57000F1EE10FA04DD4FF07E53C364FEF78CBB5E
:10E58000B5EEC02AF1EE10FA7EF586AB4FF0000230
:10E59000CBF68072C264FEF77FBB21998D6ACDB144
:10E5A000FAF75CFA219FBA6AC2F1040318184CF614
:10E5B000CD41CCF6CC41A1FB00154FEA95067A6A15
:10E5C000B6FBF2F302EE903AB8EE623A87ED133AF8
:10E5D000FEF762BB4FF6FF76C7F67F76CE64FEF796
:10E5E0005BBB43F21420C2F20000017811F0280F47
:10E5F00010D01D9E06F10306B6F5005F34BF00265D
:10E6000001260EE00000004700008047FFFF7F4B1F
:10E61000000000341D9E06F10306FA2E94BF00266A
:10E62000012646B143F2D804C2F200044FF01303AE
:10E63000237203F06CBD1D9F219DE86CFBF74EFD1E
:10E6400041F26002C2F20002D051FEF725BB2198D0
:10E65000D0ED123A90ED134A73EEC44AC0ED134A5E
:10E66000FFF769BA219EF76C1C97B56CF564B76427
:10E67000FEF712BB219AD06C0AF072F930B14FF05C
:10E680000306219981F85060FEF706BB219BD86CE8
:10E690000AF056F930B14FF00400219B83F8500086
:10E6A000FEF7FABA2198C66C30460AF06DFE08EE05
:10E6B000100A30464FF000010AF0E4FA01464FF02C
:10E6C0007E500AF0DFFA1FED2E5A05EE900A25EE75
:10E6D000856AB4EEC68AF1EE10FA06D84FF000054E
:10E6E000219A82F85050FEF7D7BA2199D1ED136ADA
:10E6F000F5EEC06AF1EE10FA05DD4FF0010781F882
:10E700005070FEF7C9BAF5EEC06AF1EE10FA4CBFD0
:10E710000222032281F85020FEF7BEBA219FD7EDD6
:10E72000138A97ED128A38EEC89A19EE100A0AF089
:10E730002BFE09EE100A18EE900A18EE101A0AF0D5
:10E74000A1FA01464FF07E500AF09CFA5FED507A34
:10E7500000EE100A60EE270AB4EEE09AF1EE10FA2D
:10E760000DF1700C8CBF00200120FBF767FEFEF757
:10E7700093BA219DEE6C30460AF006FE08EE100AB0
:10E7800030464FF000010AF07DFA01464FF07E500E
:10E790000AF078FA1FED621A07EE100A67EE011A06
:10E7A000B4EEE18AF1EE10FA0DF1700C8CBF00208E
:10E7B0000120FBF743FEFEF76FBA219A92ED132A70
:10E7C000D2ED122AB4EEE22AF1EE10FA0DF1700C3D
:10E7D000B4BF00200120FBF731FEFEF75DBA21989F
:10E7E00090ED133AB5EEC03AF1EE10FA0DF1700C5F
:10E7F000B4BF00200120FBF721FEFEF74DBA219B9C
:10E80000D3ED133A93ED124AF4EEC43AF1EE10FA56
:10E810000DF1700CD4BF00200120FBF70FFEFEF7B6
:10E820003BBA2199D1ED134A91ED125AF4EEC54A43
:10E83000F1EE10FA0DF1700C8CBF00200120FBF7F7
:10E84000FDFDFEF729BA219FD7ED135A97ED126A05
:10E85000F4EEC65AF1EE10FA0DF1700C54BF002020
:10E860000120FBF7EBFDFEF717BA219DD5ED136AEA
:10E87000F5EEC06AF1EE10FA0DF1700C54BF0020F5
:10E880000120FBF7DBFDFEF707BA219ED6ED138AC8
:10E8900096ED128A38EEC89A19EE100A0AF074FD45
:10E8A00009EE100A18EE900A18EE101A0AF0EAF9AA
:10E8B00001464FF07E500AF0E5F95FEDAB7A00EECD
:10E8C000100A60EE270AB4EEE09AF1EE10FA0DF1AC
:10E8D000700CD4BF00200120FBF7B0FDFEF7DCB9BF
:10E8E000219AD76C38460AF04FFD08EE100A3846D8
:10E8F0004FF000010AF0C6F901464FF07E500AF0D1
:10E90000C1F91FEDBD1A07EE100A67EE011AB4EE49
:10E91000E18AF1EE10FA0DF1700CD4BF0020012055
:10E92000FBF78CFDFEF7B8B943F21420C2F20000E9
:10E93000037813F0280F08D01D9901F10201B1F5F9
:10E94000005F34BF0021012106E01D9901F10201A1
:10E95000FA2994BF0021012141B143F2D804C2F247
:10E9600000044FF01300207203F0D1BBFAF776F8E1
:10E97000219F00F104004CF6CD45CCF6CC45A5FB1B
:10E9800000164FEA96007A6AB0FBF2F31D9D41F241
:10E990006000C2F2000041194E78425D4FEA024524
:10E9A00045EA0620897840EA01061B969B1B23F066
:10E9B0007F421C9202EE102AF8EE422AC7ED132A7B
:10E9C000FEF76AB9219FFD6CBD64FEF765B9219918
:10E9D00091F85160002E40F04D82FEF75DB9219B09
:10E9E00093F85120002A00F04582FEF755B943F212
:10E9F0001420C2F20000017811F0280F06D01D9EED
:10EA0000B6F5005F34BF0026012604E01D9EFA2EF5
:10EA100094BF0026012646B143F2D804C2F2000496
:10EA20004FF01306267203F072BB41F26002C2F28D
:10EA300000021D9BD05C00287EF42EA91E991C911B
:10EA40001AE243F21422C2F20002137813F0280FE4
:10EA500006D01D98B0F5005F34BF0020012004E00F
:10EA60001D98FA2894BF0020012040B143F2D80439
:10EA7000C2F200044FF01300207203F048BB41F2D1
:10EA80006001C2F200011D9E8A5D002A3EF404A9C5
:10EA90001E9B1C93F0E11D990F2908D943F2D8035E
:10EAA000C2F200034FF027021A7203F030BBC8B263
:10EAB000FCF762FC00283EF4EFA81E9E1C96DBE1EA
:10EAC0001D98F92808D943F2D804C2F200044FF087
:10EAD0001200207203F01BBB43F21411C2F20001BA
:10EAE0000E5C1E9B1E427EF4D7A81F9A1C92C3E1A7
:10EAF0001D99F92908D943F2D804C2F200044FF055
:10EB00001201217203F003BB43F21416C2F2000695
:10EB1000725C1E9B1A423EF4BFA81F981C90ABE18A
:10EB200043F21426C2F20006327812F0280F06D003
:10EB30001D9BB3F5005F34BF0023012304E01D9B40
:10EB4000FA2B94BF0023012343B143F2D804C2F24D
:10EB500000044FF01303237203F0D9BA41F26000AE
:10EB6000C2F200001D99465C002E7EF495A81E9A04
:10EB70001C92B2E143F21420C2F20000017811F0BD
:10EB8000280F06D01D9EB6F5005F34BF0026012673
:10EB900004E01D9EFA2E94BF0026012646B143F2E2
:10EBA000D804C2F200044FF01306267203F0AFBA85
:10EBB00041F26002C2F200021D9BD05C00283EF4CC
:10EBC0006BA81E991C9188E143F21422C2F2000244
:10EBD000137813F0280F06D01D98B0F5005F34BFEE
:10EBE0000020012004E01D98FA2894BF0020012095
:10EBF00040B143F2D804C2F200044FF01301217275
:10EC000003F085BA41F26001C2F200011D9E8A5DE7
:10EC10001E9B9A427EF640A81F981C902CE143F25E
:10EC20001426C2F20006327812F0280F06D01D9B7F
:10EC3000B3F5005F34BF0023012304E01D9BFA2BD2
:10EC400094BF0023012343B143F2D804C2F200046D
:10EC50004FF01300207203F05ABA41F26000C2F282
:10EC600000001D99465C1E9A9642FEF415A81F9B53
:10EC70001C9301E143F21421C2F200010E7816F058
:10EC8000280F06D01D9AB2F5005F34BF0022012282
:10EC900004E01D9AFA2A94BF0022012242B143F2F5
:10ECA000D804C2F200044FF01300207203F02FBA10
:10ECB00041F26000C2F200001D9BC15C1E9EB14289
:10ECC0007DF4EAAF1F9A1C92D6E043F21423C2F2FD
:10ECD0000003197811F0280F06D01D9EB6F5005FCD
:10ECE00034BF0026012604E01D9EFA2E94BF0026A4
:10ECF000012646B143F2D804C2F200044FF01302D9
:10ED0000227203F004BA41F26002C2F200021D98BE
:10ED1000115C1E9B99423DF4BFAF1F9E1C96ABE059
:10ED200043F21420C2F20000017811F0280F06D03F
:10ED30001D9BB3F5005F34BF0023012304E01D9B3E
:10ED4000FA2B94BF0023012343B143F2D804C2F24B
:10ED500000044FF01306267203F0D9B941F26006A1
:10ED6000C2F200061D9AB05C1E9988423DF694AF2F
:10ED70001F9B1C9380E043F21422C2F20002107821
:10ED800010F0280F06D01D99B1F5005F34BF0021A7
:10ED9000012104E01D99FA2994BF0021012141B10C
:10EDA00043F2D804C2F200044FF01306267203F0B7
:10EDB000AEB941F26006C2F200061D9BF25C1E98DD
:10EDC0008242BDF469AF1F991C9155E0219B93F8D5
:10EDD00047201D9882427DF45FAF1E991C917CE014
:10EDE000219E96F847201D9B9A423DF455AF1E98F0
:10EDF0001C9072E0219991F847601D9A96427DF629
:10EE00004BAF1E9B1C9368E0219890F847101D9E05
:10EE1000B142FDF441AF1E9A1C925EE0219B93F833
:10EE200047001D998842BDF437AF1E9E1C9654E0E2
:10EE3000219A92F847001D9B98423DF62DAF1E99EE
:10EE40001C914AE09DF874000DF16B01FCF764FE23
:10EE50008DF86A009DF86B6036B143F2D804C2F2B7
:10EE60000004267203F053B900283DF415AF1E9A32
:10EE70001C9201E01D981C901C9E40F20000C0F600
:10EE8000010090F82E1090F82F3043EA0122B24290
:10EE900008D243F2D804C2F200044FF009062672E9
:10EEA00003F035B943F21827C2F200073E60FDF7C0
:10EEB000F3BE0DF1700CFBF7D9FA1C900028D9D0E5
:10EEC000FDF7EABE0DF1700CFBF7D0FA1C9000289C
:10EED000D0D1FDF7E1BE1D9B1C93219A136A052B2F
:10EEE00008D943F2D804C2F200044FF00A03237297
:10EEF00003F00DB903F1020043F21821C2F2000140
:10EF00000E6842F8206003F10103219A1362B3E70F
:10EF10000DF1700CFBF7AAFA1C900028DBD0FDF76E
:10EF2000BBBE0DF1700CFBF7A1FA1C900028D2D1EA
:10EF3000FDF7B2BE0DF1700CFBF798FA1C901D990D
:10EF400088427DF4A9AE1E9E1C9695E70DF1700CCB
:10EF5000FBF78CFA1C901D9A90423DF49DAE1E98D2
:10EF60001C9089E70DF1700CFBF780FA1C901D9B3B
:10EF700098427DF691AE1E991C917DE70DF1700CC3
:10EF8000FBF774FA1C901D9EB042FDF485AE1E9AEC
:10EF90001C9271E70DF1700CFBF768FA1C901D9B39
:10EFA0009842BDF479AE1E981C9065E70DF1700C87
:10EFB000FBF75CFA1C901D9988423DF66DAE1E9ED3
:10EFC0001C9659E79DF874000DF16B01FCF772FD7A
:10EFD0008DF86A009DF86B3033B143F2D804C2F269
:10EFE0000004237203F093B800283DF455AE1E9A36
:10EFF0001C9241E79DF874000DF16B01FCF75AFD7E
:10F000008DF86A009DF86B1031B143F2D806C2F258
:10F010000006317203F07BB800287DF43DAE1E98E7
:10F020001C9029E70DF1700CFBF748FA41F26002E1
:10F03000C2F200021E9BD15C1D9801423DF42CAE31
:10F040001F9E1C9618E70DF1700CFBF737FA41F282
:10F050006002C2F200021E9BD15C1D9801427DF449
:10F060001BAE1F9E1C9607E70DF1700CFBF726FAEE
:10F0700041F26002C2F200021E9BD15C1D98014267
:10F080007DF40AAE1F9E1C9627E70DF1700CFBF76E
:10F0900015FA41F26002C2F200021E9BD15C1D987B
:10F0A00001423DF4F9AD1F9E1C9616E798F80050FA
:10F0B00045F0080088F80000FDF717BE0DF1700C50
:10F0C000FBF7D4F98DF86A00219991F851601D9AE7
:10F0D000B3181C9343F21421C2F200010E7816F00B
:10F0E000280F09D01E9E06F1FF32D318B3F5005F3A
:10F0F00034BF0023012307E01E9A02F1FF31CB1831
:10F10000FA2B94BF0023012343B143F2D804C2F287
:10F1100000044FF01303237202F0F9BF4FF0000711
:10F120001B971E9DE5B11C9941F26003C2F20003DA
:10F130005E5C864235D005F1FF3241F26007C2F2D3
:10F1400000077B1841F26005C2F20005C5F1010617
:10F15000C1F101014F1B12F0010F1AD003F042B8A8
:10F160004FF0FF001B901CE013F8019F02F1FF38E5
:10F17000484504D11C91CDF86CE01E9211E0424646
:10F18000F11807EB030E13F8015FA84243F0378034
:10F19000F0E7F11807EB030E002AE5D11C911E924F
:10F1A000DEE70DF1700C9DF86C00FBF747F9FDF7F9
:10F1B00073BD0DF1700CFBF759F943F2900BC2F2DD
:10F1C000000B8BF800004FF001061C96CDF830B014
:10F1D000BBE0219991F851201D9813181C9343F21C
:10F1E0001426C2F20006317811F0280F07D003F17F
:10F1F0000103B3F5005F34BF0023012305E003F1F1
:10F200000103FA2B94BF0023012343B143F2D80436
:10F21000C2F200044FF01302227202F078BF1E986F
:10F220001B900DF1700C26AF47F0010122AD45F0A7
:10F2300001024FF00003FBF753F9FDF72DBD2198B4
:10F2400090F851601D9BF1181C9143F21422C2F2F8
:10F250000002107810F0280F05D0B1F5005F34BF20
:10F260000021012103E0FA2994BF0021012141B1CD
:10F2700043F2D804C2F200044FF01303237202F0E9
:10F2800046BF1F9F1E98B84228BF38461B900DF1FD
:10F29000700C26AD45F0010122AE46F001024FF0A0
:10F2A0000003FCF7D5F9FDF7F7BC0DF1700CFBF787
:10F2B000DDF8034643F2900BC2F2000B58464FF0C4
:10F2C00010014DF6C812C0F603020AF03FFA1C9076
:10F2D000CDF830B039E01E991C911F9A1B924FF067
:10F2E00000000C9031E04FF0FF361C960C962CE09D
:10F2F000219BD86C9DF878109DF87C2043F29006F5
:10F30000C2F2000600964FF0100301934FF0010384
:10F31000FDF75CF84FF0FF311C910C9615E0219A37
:10F32000D06C9DF878109DF87C2043F29006C2F2D4
:10F33000000600964FF0100301934FF00003FDF715
:10F3400045F84FF0FF301C900C961D99A1F1FB0081
:10F3500086B20B96A1F1FB03032B23D840F2A060E9
:10F36000C1F200004FF411760B9906FB010393F8EC
:10F370002022032A08D043F2D806C2F200064FF03A
:10F380004803337202F0C3BE40F2A067C1F2000727
:10F390004FF411700B9E00FB067707F104074FF046
:10F3A000000605E0219F97F8512056184FF00007FE
:10F3B000DDF870B0BBF1FF3F11D14FF0FF0B4FF004
:10F3C0000009C84643F21421C2F200010D9141F236
:10F3D0006003C2F200030E930F950C9D05E0BBF194
:10F3E000000FECD14FF000096FE01D9AA2F1FB0273
:10F3F000032A10D8D7F80061FF2E14BF0136464605
:10F40000D7F80401864206D14046FCF781F9D7F8C7
:10F4100004118E42F8D0B5F1FF3F15D1219850F874
:10F42000341F0B68D3F800C0494610AA4FF00103FF
:10F43000E0478DF86B0080B10F9D43F2D804C2F213
:10F440000004207202F063BE25B115F809208DF882
:10F45000402002E01B9B8DF840301C98B0F1FF3F2C
:10F4600002D19DF8402082B31D99A1F1FB0103292F
:10F4700007D8D7F800319DF84000F854C7F800616C
:10F480001FE00D9B187810F0280F05D0B6F5005F2F
:10F4900034BF0020012003E0FA2E94BF0020012099
:10F4A00048B10F9D43F2D804C2F200044FF0130696
:10F4B000267202F02CBE9DF840200E998A5506F166
:10F4C000010609F10109D9458FD31D9FA7F1FB075B
:10F4D000032F05D80B99C8B2FBF758FAFDF7DCBB30
:10F4E000219D95F8512009EB020E85F851E0FDF7BA
:10F4F000D3BB1D9AA2F1FB01032958D88FB240F269
:10F50000A060C1F200004FF4117101FB070292F8F4
:10F510002032032B08D043F2D804C2F200044FF08B
:10F520004803237202F0F3BD40F2A066C1F2000668
:10F530004FF4117505FB076505F104051E9800F1F0
:10F54000FF311E9170B34FF0000843F21829C2F248
:10F55000000940F200029346C0F6010BD5F80061A5
:10F56000FF2E14BF01364646D5F804319E4206D11F
:10F570004046FCF7CDF8D5F804018642F8D0D9F81A
:10F580000030D5F800211BF80310A95403F1010342
:10F59000C9F80030C5F800611E9E06F1FF301E90CC
:10F5A000002EDBD1F8B2FBF7F1F9FDF775BB1E9B1E
:10F5B0001C93219991F8510082181B9243F2142652
:10F5C000C2F20006367816F0280F08D003F1FF3695
:10F5D000B218B2F5005F34BF0022012206E003F149
:10F5E000FF36B218FA2A94BF0022012242B143F238
:10F5F000D804C2F200044FF01306267202F087BD51
:10F60000C71881F851701C9A02F1FF351C95002A29
:10F610003DF442AB43F21823C2F200031E681B9F65
:10F6200041F26001C2F20001C91940F20000C0F6C7
:10F63000010030184FF0000305F0010910F803C075
:10F6400001F803C003F10103934242F0BC850DE0D1
:10F6500010F803E001F803E003F1010310F8039050
:10F6600001F8039003F101039342F1D1E819A919BC
:10F6700001F1010143F21822C2F2000211604FF0C1
:10F68000FF331C9300F101001B90FDF705BB4FF009
:10F6900000028DF86A20219E96F851001D9BC1182A
:10F6A0001C911E9A1B9243F21420C2F200000378B0
:10F6B00013F0280F08D002F1FF335818B0F5005F9F
:10F6C00034BF0020012006E002F1FF325018FA2872
:10F6D00094BF0020012040B143F2D804C2F20004DC
:10F6E0004FF01302227202F012BD41F26007C2F223
:10F6F000000707EB01099DF87CB043F21025C2F228
:10F7000000052A68B66B9119905DFF2859D088468C
:10F710004FF001070894CDF82CA0BA4698F80140A4
:10F7200004EB002343F21025C2F200052A68D61824
:10F730004FF000011C919DF86A00002802F0198525
:10F74000D75C06F1010602F016BD9DF86A402CB1A7
:10F750008FB9089C5046DDF82CA005E0727852B9AC
:10F76000089C5046DDF82CA0219F97F851609B190A
:10F7700087F8513027E016F8014F19F803B045B962
:10F78000204609F087FFC4B2584609F083FF5FFAAC
:10F7900080FB5C4508D11C9B03F101031C9307F11E
:10F7A000FF371B999942D0D2AB460AF1010A18F8EB
:10F7B000020FFF28B2D1089CDDF82CA04FF000000A
:10F7C00001E04FF000000DF1700CC0B2FAF736FE08
:10F7D000FDF762BA4FF001018DF86A105BE70DF199
:10F7E000700CFAF743FE034643F2900BC2F2000B93
:10F7F00058464FF010014DF6D012C0F6030209F042
:10F80000A5FF1C90CDF830B09FE50DF1700CFAF714
:10F810002DFE034643F2900BC2F2000B58464FF008
:10F8200010014DF6D812C0F6030209F08FFF1C90AC
:10F83000CDF830B089E50DF1700CFAF717FE0346EC
:10F8400043F2900BC2F2000B58464FF010014DF6F8
:10F85000DC12C0F6030209F079FF1C90CDF830B03D
:10F8600073E50DF1700CFAF701FE034643F2900BBD
:10F87000C2F2000B58464FF010014DF6E412C0F6EC
:10F88000030209F063FF1C90CDF830B05DE52198CC
:10F8900090F8517007F1010780F85170FDF7FCB93D
:10F8A0001D9D41F26002C2F20002515D01F10101B1
:10F8B0005155FDF7F1B9219E96F8473003F1010348
:10F8C00086F84730FDF7E8B99DF874000DF16B013B
:10F8D000FCF7F0F80DF1700CFAF7B0FD9DF86B0035
:10F8E00000283DF4D9A943F2D804C2F200042072E2
:10F8F00002F00DBC9DF874000DF16B01FCF746F9A8
:10F900000DF1700CFAF79AFD9DF86B1000293DF48B
:10F91000C3A943F2D802C2F20002117202F0F7BB8F
:10F920001D9E1C964FF000031B934FF001008DF8B5
:10F930006A009DF870000DF16B01FCF7BBF89DF8B3
:10F940006B1099B920B19DF86A201B9E16431B9637
:10F950009DF86A304FEA43008DF86A001C9901F166
:10F9600001011C9110F0FE0FE3D10AE09DF86A201E
:10F97000012A06D143F2D804C2F20004217202F037
:10F98000C6BB0DF1700C9DF86C00FAF757FDFDF742
:10F9900083B91D9E1C964FF000031B934FF001008E
:10F9A0008DF86A009DF870000DF16B01FCF7EEF820
:10F9B0009DF86B1099B920B19DF86A201B9E1643E3
:10F9C0001B969DF86A304FEA43008DF86A001C9937
:10F9D00001F101011C9110F0FE0FE3D10AE09DF846
:10F9E0006A20012A06D143F2D804C2F2000421722F
:10F9F00002F08DBB0DF1700C9DF86C00FAF71EFD46
:10FA0000FDF74AB99DF874000DF16B01FCF784F81D
:10FA10008DF86A009DF86B6036B143F2D803C2F2EC
:10FA200000031E7202F073BB0DF1700CFAF706FDB5
:10FA3000FDF732B91D981C904FF000011B914FF05B
:10FA400001008DF86A00219A92F8476030420ED08A
:10FA50009DF870000DF16B01FCF75EF89DF86B30BE
:10FA60009BB920B19DF86A001B9901431B919DF839
:10FA70006A204FEA42068DF86A601C9B03F101037D
:10FA80001C9316F0FE00DED10AE09DF86A100129F1
:10FA900006D143F2D804C2F20004237202F037BB4D
:10FAA0001B9F219D85F84770FDF7F6B89DF87400FF
:10FAB0000DF16B01FCF79CF80DF1700CFAF7BEFC30
:10FAC0009DF86B60002E3DF4E7A843F2D802C2F225
:10FAD0000002167202F01BBB1D9B1C93D8B20DF1E5
:10FAE0006B01FCF785F81B909DF86B0030B143F279
:10FAF000D804C2F20004207202F009BB4FF00101E9
:10FB00008DF86A101C9F7A181C92D0B20DF16B010F
:10FB1000FCF76EF89DF86A5000FA05F01B9E06434C
:10FB20001B9605F101058DF86A501C9A02F101023D
:10FB30001C92EBB2072BE8D90DF1700C9DF86C000C
:10FB4000FAF77CFCFDF7A8B80DF1700C219890F83D
:10FB50005100FAF773FCFDF79FB8FDF79DB843F22B
:10FB6000C001C2F200014FF001070F70FDF794B819
:10FB700043F2C005C2F200054FF000062E70FDF7FB
:10FB80008BB821984FF000014FF054020AF014FA9C
:10FB90004FF00002219243F2A003C2F200031C685E
:10FBA00004F1FF30186002F01EBA43F2A002C2F264
:10FBB000000213687F2B08D943F2D804C2F2000474
:10FBC0004FF03000207202F0A2BA4FF001071C97EC
:10FBD00040F2A065C1F20005D5F8E809002842F01E
:10FBE000D58205E0D6F8AC20002A4ED11C9301E066
:10FBF0004FF001031D9840F2A066C1F200064FF0DD
:10FC0000540505FB03F3F218C2F89009C2F89409F1
:10FC10001E9982F8E2194FF00A07C2F8B47906F586
:10FC20001967F81800F13400219901F134014FF0FF
:10FC300010020AF09DF91C9B05FB037000F14400C3
:10FC4000219901F144014FF004020AF091F91C9846
:10FC500005FB007000F14800219901F148014FF0C7
:10FC600008020AF085F9219A92F851101C9F05FBB1
:10FC7000076686F8E11943F2A005C2F200052B6879
:10FC800003F101032B60FDF707B803F101073B46C1
:10FC900006F15406D6F8AC50002D42F08B82A5E751
:10FCA0001C93FCF7F9BF219991F852601E967CE7EE
:10FCB0000DF1700CFAF7DAFB1E9076E71D9A219988
:10FCC00081F85120FCF7E8BF0DF1700C9DF874002D
:10FCD000FAF7B4FBFCF7E0BF219EB36A002B3CF4BB
:10FCE000DBAFF8F7BBFE219B9A6A861A586A1D9B08
:10FCF00003FB00F008F086F94FF000024FF000031C
:10FD0000C4F2040308F0EAFB08F010FA8642BCF4DF
:10FD1000C3AF1E981C90FFF7AFB8F8F79FFE219F66
:10FD2000B862FCF7B9BF43F21412C2F2000292F8B3
:10FD3000FB201E9E9119FB2908D943F2D800C2F27C
:10FD400000004FF01201017202F0E1B943F21423F6
:10FD5000C2F20003187810F0280F09D01D9953182B
:10FD600003F1FF30B0F5005FB4BF0020012007E0D1
:10FD70001D99531803F1FF30FA28D4BF0020012049
:10FD800040B143F2D804C2F200044FF013022272D1
:10FD900002F0BDB943F21415C2F20005A81941F2F0
:10FDA0006007C2F200071D9EB9190AF0E1F8FCF7DE
:10FDB00073BF98F8003043F0100588F80050FCF746
:10FDC00094BF219F97F84760002E0CBFFF220022AE
:10FDD00087F84720FCF760BF219890F847106FEA3A
:10FDE000010380F84730FCF757BF0DF1700CFAF7AC
:10FDF00065FB1E9D41F26007C2F200077E5D1D9A01
:10FE000072407A55FCF748BF2198816B1D9B5E18A4
:10FE10001C96BDE12198C26B816B53181C93B7E10E
:10FE2000219E306C40B943F2D804C2F200044FF076
:10FE30002002227202F06BB900F1FF353564FCF745
:10FE40002BBF21990B6C03F101030B64002B7CF495
:10FE500023AF43F2D806C2F200064FF02000307202
:10FE600002F055B9219A516B0B685E6846B943F2AE
:10FE7000D800C2F200004FF01E03037202F047B92F
:10FE80000DF1700CFAF7F2FA1C90219850F8342F0B
:10FE900011684E681D991CAA4FF00103B0478DF8F8
:10FEA0006B0000283CF4F8AE43F2D804C2F2000420
:10FEB000207202F02CB90DF1700CFAF7D7FA1C90F1
:10FEC00054E10DF1700CFAF7D1FA219FF863FCF7B9
:10FED000E3BE0DF1700CFAF7C9FA219D2864FCF716
:10FEE000DBBE219850F8342F11680E681D991CAAAA
:10FEF0004FF00103B0478DF86B0030B143F2D804E6
:10FF0000C2F20004207202F002B90DF1A80C1CF834
:10FF1000380DFAF793FAFCF7BFBE2198436B0DF149
:10FF2000700C187AFAF78AFAFCF7B6BE0DF1700C6D
:10FF3000219F97F83C00FAF781FAFCF7ADBE219AB1
:10FF4000116CFF2908D943F2D806C2F200064FF01F
:10FF50002004347202F0DBB80DF1700CC8B2FAF76D
:10FF60006DFAFCF799BE219850F8345F2B689F68B2
:10FF7000B84703EE100AF8EE433A2198C0ED133A61
:10FF8000FCF78ABE219A92ED0E4AF8EE444AC2ED81
:10FF9000134AFCF781BE219991ED105AF8EE455AAB
:10FFA000C1ED135AFCF778BE219E96ED136AFCEE64
:10FFB000C66ACDED1C6AEBE0219BD3ED137A9FED71
:10FFC000B40AF4EEC07AF1EE10FA08DB43F2D8047A
:10FFD000C2F200044FF02000207202F098B8FCEE4C
:10FFE000E70AC3ED100AFCF757BE219850F8342FEA
:10FFF00011680E681D991CAA4FF00403B0478DF8D4
:020000040803EF
:100000006B0030B143F2D803C2F20003187202F061
:100010007EB81C98FAF78CF8219DA864FCF73CBECA
:10002000219850F8342F11680E681D991CAA4FF0C2
:100030000403B0478DF86B0030B143F2D804C2F22C
:100040000004207202F063B81C98FAF771F8219F3F
:10005000F864FCF721BE2198436B1A68516841B9D6
:1000600043F2D800C2F200004FF01E02027202F00A
:100070004EB8C06CFAF732F81C90219850F8346FE3
:1000800033685E681D991CAA4FF00403B0478DF8D1
:100090006B0000283CF400AE43F2D804C2F2000426
:1000A000207202F034B843F21421C2F200010B783E
:1000B00013F0280F0BD0219EF06B1D9A111801F13F
:1000C000FF33B3F5005F34BF0023012309E0219E15
:1000D000F06B1D9A111801F1FF33FA2B94BF002326
:1000E000012343B143F2D800C2F200004FF01301E4
:1000F000017202F00CB8219B184650F8347F3E681C
:1001000036684FF0000141F26007C2F200071D9A05
:10011000BA18DB6BB0478DF86B0000283CF4BCAD1F
:1001200043F2D804C2F20004207201F0F0BF21981B
:1001300050F8343F1E6836681D991BAA4FF004031F
:10014000B0478DF86B0030B143F2D804C2F200041E
:10015000207201F0DCBF1B9882B2C0F3072141EA94
:1001600002239EB21C9613E01D981C901C982199A6
:10017000FAF71AFA8DF86B0000283CF48DAD43F2C3
:10018000D802C2F20002107201F0C1BF1D991C9189
:100190001C9BB3F5803F08D343F2D804C2F200049D
:1001A0004FF01F00207201F0B2BF219DAB63FCF73E
:1001B00073BD1D9D219FFD63FCF76EBD1D9E219BA0
:1001C0001E64FCF769BD2198826B1D99561A1C9616
:1001D000DEE71E9A219BD96B8E18FB2E08D943F2BD
:1001E000D800C2F200004FF01202027201F08FBF7D
:1001F00043F21417C2F2000787F8FB10184650F8B4
:10020000341F0E6836681D99BA18DB6BB0478DF83D
:100210006B0000283CF440AD43F2D804C2F2000465
:10022000207201F074BF219B596B0E68766846B945
:1002300043F2D801C2F200014FF01E00087201F033
:1002400066BF43F21420C2F20000027812F0280FB9
:100250000AD0DA6B1D99881800F1FF30B0F5005F05
:1002600034BF0020012008E0D86B1D990A1802F164
:10027000FF30FA2894BF0020012058B143F2D80380
:10028000C2F200034FF013061E7201F040BF00BF20
:100290000000804703F134004FF0000141F2600795
:1002A000C2F200071D9ABA18DB6BB0478DF86B00DD
:1002B00000283CF4F1AC43F2D804C2F200042072EE
:1002C00001F025BFF6F7E2FA00287CF4E5AC1D9AB0
:1002D0001C92FEF7D1BDF6F7D9FA00283CF4DCAC4D
:1002E0001D9B1C93FEF7C8BD1D9E0C2E08D943F222
:1002F000D804C2F200044FF00501217201F007BFDB
:10030000F0B24FF00001F6F77FFA01EE100AB8EEF6
:10031000417A219F87ED137AFCF7BEBC1D980C280B
:1003200008D943F2D803C2F200034FF005021A7253
:1003300001F0EDBEC0B24FF00101F6F765FA01EE33
:10034000900AB8EE612A219D85ED132AFCF7A4BC22
:100350001D9E0C2E08D943F2D804C2F200044FF0BF
:100360000501217201F0D3BEF0B24FF00001F6F7A3
:10037000BBF9FCF791BC1D980C2808D943F2D803AF
:10038000C2F200034FF005021A7201F0C0BEC0B203
:100390004FF00101F6F7A8F9FCF77EBC1D9E0C2E6C
:1003A00008D943F2D804C2F200044FF005012172CB
:1003B00001F0ADBEF0B24FF00001F6F7E5F9FCF741
:1003C0006BBC1D980C2808D943F2D803C2F2000375
:1003D0004FF005021A7201F09ABEC0B24FF001014F
:1003E000F6F7D2F9FCF758BC9DF87400F1F7E6FB7C
:1003F00000287CF451AC43F2D806C2F200064FF05C
:100400002804347201F083BE9DF87400219901F133
:100410004C01F1F7F3FB00287CF43EAC43F2D80129
:10042000C2F200014FF02800087201F070BE219B5B
:10043000D3ED132A9DF87400BCEEE23A13EE101AC5
:10044000F1F70EFC00287CF427AC43F2D806C2F288
:1004500000064FF02802327201F059BEFCF71CBCB6
:100460000DF1700CFAF702F830B9219F97F8475058
:10047000291C18BF012101E04FF00101219880F8EB
:100480004710FCF709BC9DF874600DF1700CF9F78A
:10049000EDFF014630464FF00102FBF721FC8DF8DD
:1004A0006B0000283CF4F8AB43F2D804C2F200041D
:1004B000207201F02CBE0DF1700CF9F7D7FF014648
:1004C0008DF86A009DF87400FBF7C8FB8DF86B008F
:1004D00000283CF4E1AB43F2D803C2F200031872E7
:1004E00001F015BE1D9A1C924FF001038DF86A3081
:1004F0001E46219890F847100B420AD090F84610FB
:100500009DF8700019403246FBF7EAFB8DF86B004E
:1005100068B99DF86A304FEA43008DF86A001C9A6A
:1005200002F101021C9210F0FE03E2D10AE09DF8F4
:100530006A60012E06D143F2D804C2F20004207290
:1005400001F0E5BD4FF000078DF86B700DF1700CF8
:10055000F9F78CFF0DF1700CF9F788FFFCF79CBBE5
:100560009DF874004FF001010A46FBF7B9FB8DF8C6
:100570006B0000283CF490AB43F2D801C2F20001BA
:10058000087201F0C4BD9DF874004FF000014FF0F7
:100590000102FBF7A5FB8DF86B0000283CF47CAB57
:1005A00043F2D802C2F20002107201F0B0BD0DF1A8
:1005B000700CF9F75BFF219D95F84730184385F8DB
:1005C0004700FCF769BB1D980DF1A80C4CF8380DDD
:1005D000FAF7FAFB00287CF45FAB43F21826C2F26C
:1005E00000060898306001F015BD10A8FAF77EFAF1
:1005F000014640B19DF84070022F04D0C2484FF030
:100600000D0209F0B5FC0DF1700C9DF84000F9F7F2
:1006100015FFFCF741BBFAF79BFFFCF73DBB0DF163
:10062000700CF9F723FFFCF737BB1D9EFA2E08D993
:1006300043F2D804C2F200044FF01202227201F019
:1006400066BD0DF1700CF9F711FF43F21411C2F2FF
:1006500000018855FCF720BB0DF1700CF9F706FF7F
:1006600043F21415C2F2000585F8FB00FCF714BB39
:100670000DF1700C219B93F84700F9F7DFFEFCF7B2
:100680000BBB1D98FA2808D943F2D806C2F200061F
:100690004FF01201317201F03ABD0DF1700C43F2CE
:1006A0001417C2F20007385CF9F7C8FEFCF7F4BA79
:1006B0000DF1700C43F21412C2F2000292F8FB002A
:1006C000F9F7BCFEFCF7E8BA1D9EF62E08D943F2F6
:1006D000D804C2F200044FF01200207201F017BDDE
:1006E000219DA86CF9F7FAFC43F21413C2F200033F
:1006F0009851FCF7D1BA43F21421C2F200010A78F2
:1007000012F0280F06D01D9EB6F5005F34BF0026FC
:10071000012604E01D9EFA2E94BF0026012646B154
:1007200043F2D803C2F200034FF013041C7201F02D
:10073000EEBC0DF1700C41F26007C2F200071D9D86
:10074000785DF9F77BFEFCF7A7BA0DF1700CF9F7AD
:10075000B5FE41F26000C2F200001E99425C1D9E8F
:1007600032420DF1700C0CBF0020FF20F9F766FE3D
:10077000FCF792BA43F21423C2F20003187810F087
:10078000280F08D01D9901F10101B1F5005F34BFB8
:100790000021012106E01D9901F10101FA2994BF10
:1007A0000021012141B143F2D800C2F200004FF014
:1007B0001301017201F0ABBC1D9A41F26006C2F256
:1007C0000006B05CB318597841EA00221C92002A56
:1007D0003CF462AAFEF750BB43F21423C2F20003BA
:1007E0001A7812F0280F06D01D9EB6F5005F34BFB0
:1007F0000026012604E01D9EFA2E94BF0026012645
:1008000046B143F2D804C2F200044FF01302227240
:1008100001F07DBC41F26000C2F200001D99435C12
:10082000002B56D1FCF738BA43F21426C2F2000668
:10083000307810F0280F06D01D99B1F5005F34BF55
:100840000021012104E01D99FA2994BF0021012112
:1008500041B143F2D804C2F200044FF013002072F9
:1008600001F055BC41F26002C2F200021D9BD65C51
:100870007EB3FCF711BA0DF1700CF9F7F7FD1C907F
:1008800038BBFCF709BA0DF1700CF9F717FE41F20D
:100890006001C2F200011E9A8E5C1D9B1E4218D0A0
:1008A000FCF7FAB90DF1700CF9F708FE41F260009F
:1008B000C2F200001E99425C1D9E324209D1FCF733
:1008C000EBB90DF1700CF9F7D1FD1C9000287CF408
:1008D000E3A9219B1E6A46B943F2D804C2F2000480
:1008E0004FF00300207201F012BC06F1FF351D62CB
:1008F00006F1010653F8267043F21821C2F20001F6
:100900000F60FCF7C9B900BF6610002098F80050CE
:1009100045F0200388F80030FCF7E7B9219F97F8ED
:1009200047004FEAD01141EA400287F84720FCF720
:10093000B3B9219E96F847504FEA550343EAC517CD
:1009400086F84770FCF7A8B9FAF7A2F9FCF7A4B942
:1009500041F25800C2F20000C2784FF0010101FAE2
:1009600002F1067926EA01060671FCF795B943F211
:100970001415C2F2000541F25807C2F200073B7895
:1009800078780090BA78019228464FF0FB014DF636
:10099000E812C0F6030208F0D9FE85F8FB00FCF768
:1009A0007BB941F25803C2F20003D97841B941F250
:1009B0005807C2F200074FF00600F870FCF76CB958
:1009C00001F1FF3641F25805C2F20005EE70FCF766
:1009D00063B941F25802C2F20002137803F1FF3109
:1009E000CEB216701579FF2D0BD1632E7CF654A96B
:1009F00041F25803C2F200034FF063021A70FCF791
:100A00004BB9172E7CF648A941F25807C2F20007ED
:100A10004FF017003870FCF73FB941F25801C2F2AD
:100A200000014E7806F1FF35EFB24F700879FF28CC
:100A30000BD1002F7CF430A941F25801C2F2000121
:100A40004FF00C064E70FCF727B93B2F7CF624A91B
:100A500041F25803C2F200034FF03B025A70FCF718
:100A60001BB941F25805C2F20005AF7807F1FF301B
:100A7000C2B2AA702B79FF2B17D141F25805C2F2EE
:100A800000052F78687807F5FA61F7F7E5F88DF833
:100A90006A00AA7812B19042BCF4FEA841F2580351
:100AA000C2F200039870FCF7F7B83B2A7CF6F4A872
:100AB00041F25801C2F200014FF03B068E70FCF784
:100AC000EBB843F21410C2F200004FF0000180F8BE
:100AD000FB1041F25806C2F20006F57845703779EE
:100AE0000770FCF7D9B843F21416C2F2000641F2BF
:100AF0005802C2F200021378507800909178019168
:100B000030464FF0FB014DF6F812C0F6030208F034
:100B10001DFE86F8FB00FCF7BFB843F21415C2F2C5
:100B2000000541F25807C2F200073B787E78009634
:100B300028464FF0FB014DF60822C0F6030208F0EC
:100B400005FE85F8FB00FCF7A7B841F25803C2F296
:100B50000003D878052808D941F25801C2F20001F3
:100B60004FF00005CD70FCF797B800F1010041F29D
:100B70005802C2F20002D070FCF78EB841F258075A
:100B8000C2F200073E7806F10106F3B23B703879F5
:100B9000FF280BD1632B7CF67FA841F25805C2F2E7
:100BA00000054FF000072F70FCF776B8172B7CF686
:100BB00073A841F25801C2F200014FF000020A701E
:100BC000FCF76AB841F25806C2F20006737803F1E6
:100BD0000103D8B270703179FF290BD10C287CF653
:100BE0005BA841F25807C2F200074FF001067E7081
:100BF000FCF752B83B287CF64FA841F25805C2F2E8
:100C000000054FF000026A70FCF746B841F2580345
:100C1000C2F20003987800F10100C5B29D70197905
:100C2000FF291DD15DB141F25802C2F200021778CE
:100C3000507807F5FA61F7F70FF8854208D941F2C5
:100C40005807C2F200074FF00106BE70FCF724B847
:100C500041F25806C2F200063379FF2B3CF41CA87F
:100C600041F25800C2F2000085783B2D7CF614A8B2
:100C700041F25801C2F200014FF000028A70FCF705
:100C80000BB841F25803C2F20003D8784FF00105C7
:100C900005FA00F5197985EA01021A71FBF7FCBF24
:100CA0000DF1700CF9F7E2FB41F25807C2F20007B0
:100CB0003871FBF7F1BF0DF1700CF9F7D7FB06287F
:100CC00041F25806C2F2000692BFF0700023F370A2
:100CD000FBF7E2BF0DF1700CF9F7C8FB41F25805C4
:100CE000C2F200052870FBF7D7BF0DF1700CF9F7C1
:100CF000BDFB41F25801C2F200014870FBF7CCBFC6
:100D00000DF1700CF9F7B2FB41F25802C2F2000289
:100D10009070FBF7C1BF0DF1700C41F25800C2F2A8
:100D200000000079F9F78AFBFBF7B6BF0DF1700CF4
:100D300041F25807C2F20007F878F9F77FFBFBF79A
:100D4000ABBF0DF1700C41F25806C2F200063078CC
:100D5000F9F774FBFBF7A0BF0DF1700C41F25803DB
:100D6000C2F200035878F9F769FBFBF795BF0DF164
:100D7000700C41F25805C2F20005A878F9F75EFB45
:100D8000FBF78ABF11A8F1F769F841F25803C2F2E4
:100D90000003169D48F21F50C5F2EB1080FB0502C0
:100DA0004FEAE577C7EB62164FF0640101FB165579
:100DB0001D70159800F101005870149A9A70179BD5
:100DC0001BB103F1FF36F7B201E04FF0060741F225
:100DD0005801C2F20001CF704FF0FF050D71FBF713
:100DE0005BBF1D9A0F2A08D943F2D804C2F200044F
:100DF0004FF02700207201F08AB9C64800EB82014B
:100E000041F25807C2F2000710F822603E704B789A
:100E10007B704FF00005BD70FD708A783A71FBF76A
:100E20003BBF41F25800C2F20000FAF789FAFBF723
:100E300033BF41F25807C2F20007FE784FF00101BC
:100E400001FA06F13B7941EA03053D71FBF724BF46
:100E500011A8F1F703F841F25800C2F2000002783D
:100E600002F164021692477807F1FF3615968178F1
:100E7000149111A8F1F758F884E71D980F2808D9A4
:100E800043F2D804C2F200044FF02702227201F0AC
:100E90003EB9C0B2FAF770FA0DF1700CF9F7CEFA5C
:100EA000FBF7FABE4FF000031393129311931993BB
:100EB00041F25807C2F200073E7806F16406169622
:100EC000797801F1FF351595B878149011A808F0DC
:100ED00075FE179A1AB102F1FF37FBB201E04FF02D
:100EE000060341F25806C2F20006F370FBF7D4BEC7
:100EF0001D9A0F2A08D943F2D804C2F200044FF019
:100F00002702227201F003B9824800EB820141F20C
:100F10005803C2F200031D7800F822505F784F702A
:100F20001E798E70FBF7B8BE11A8F0F797FF41F25B
:100F30005800C2F20000017813914378129385782B
:100F4000119511A8F0F7F0FFFBF7A6BE0DF1700C9C
:100F5000219F97F85000F9F771FAFBF79DBE43F215
:100F60001426C2F20006347814F0010F08D143F2BF
:100F7000D806C2F200064FF03004347201F0C7B850
:100F800043F2A002C2F20002106840B943F2D80155
:100F9000C2F200014FF031030B7201F0B8B843F216
:100FA0001421C2F200010B7803F0FE0646F004049F
:100FB0000C7043F2B000C2F200004FF00002026079
:100FC00001F011B843F21420C2F20000027812F0CE
:100FD000010F08D143F2D800C2F200004FF03002F6
:100FE000027201F094B843F2A001C2F200010B6852
:100FF00043B943F2D806C2F200064FF0340434720B
:1010000001F085B843F21426C2F20006347804F0E9
:10101000FE0040F00202327043F2B001C2F2000161
:101020004FF000030B6000F0DEBF219D95F8467085
:101030000DF1700CF9F71AFA21993B1A91F85060EA
:1010400006F001001A1A1C9281F84720FF2A94BF6B
:101050000022012281F85020FBF71EBE43F214212A
:10106000C2F200010B7813F0280F06D01D9EB6F5D2
:10107000005F34BF0026012604E01D9EFA2E94BFB7
:101080000026012646B143F2D804C2F200044FF014
:101090001302227201F03BB841F26005C2F2000572
:1010A0001E9F1D982F54FBF7F7BD4FF000011C91B8
:1010B0001AE04FF001031C9316E04FF002061C9655
:1010C00012E04FF003051C950EE04FF004071C974B
:1010D0000AE04FF005001C9006E04FF006021C925B
:1010E00002E04FF007011C911D991B911C98F9F724
:1010F000E3FDFBF7D1BD0DF1700CF9F7DFF91E9B95
:1011000041F26006C2F20006F55C1D9F2F43F754C2
:10111000FBF7C2BDF00F00101D98F92808D943F263
